:020000040000FA
:10000000F83B002011040000190400003102000038
:100010001D0400001F040000210400000000000077
:1000200000000000000000000000000023040000A9
:10003000250400000000000027040000290400003F
:10004000D10A00002B040000550F00002B04000013
:100050002B0400002B040000810700002B0400008B
:100060002B0400002B0400002B0400002B040000D4
:100070002B0400002B0400002B0400002B040000C4
:100080002B040000E10A00002B0400002B040000F8
:100090002B0400002B0400002B0400002B040000A4
:1000A0002B0400002B0400002B0400002B04000094
:1000B0002B0400002B0400000000000000000000E2
:1000C0002B0400002B0400002B0400002B04000074
:1000D0002B0400002B0400002B0400000000000093
:1000E0000000000000000000000000000000000010
:1000F0000000000000000000000000000000000000
:1001000000000000000000000000000000000000EF
:1001100000000000000000000000000000000000DF
:1001200000000000000000000000000000000000CF
:1001300000000000000000000000000000000000BF
:1001400000000000000000000000000000000000AF
:10015000000000000000000000000000000000009F
:10016000000000000000000000000000000000008F
:10017000000000000000000000000000000000007F
:10018000000000000000000000000000000000006F
:10019000000000000000000000000000000000005F
:1001A000000000000000000000000000000000004F
:1001B000000000000000000000000000000000003F
:1001C000000000000000000000000000000000002F
:1001D000000000000000000000000000000000001F
:1001E000000000000000000000000000000000000F
:1001F00000000000000000000000000000000000FF
:10020000DFF80CD000F070FA00480047B151000050
:10021000F83B002000B583B002900091019244F2B7
:10022000010071466A4600F0F9FF03B000BD00000E
:10023000094B1EF0040F1CBFEFF309801847EFF3C2
:1002400008800649064A884201D8904202D88D4665
:100250004FF0000018470000ED080000F83B0020B8
:10026000F81B002030B450E8012F93B2C489234416
:100270008489A34228BF1B1B0489A34202BFBFF38A
:100280002F8F002007E0C3EA020340E80134002C6E
:10029000E9D14FF001000A6030BC704750E8012FEF
:1002A000C2EA024240E801210029F7D1704730B488
:1002B00050E8022F1FFAA2F3C488A34202BFBFF383
:1002C0002F8F00200DE0C48923448489A34228BFD6
:1002D0001B1BC2EA034340E80234002CE8D14FF074
:1002E00001000A6030BC704750E8022FC2EA224287
:1002F00040E802210029F7D17047034653E8022F56
:10030000D988B2EB324F4FF0000017BF92B241EAEA
:10031000014142EA014104E05A68B2EB324F08BFA2
:10032000012043E80212002AE8D1704730B40446A5
:1003300054E8000F0D4644E80053002BF8D1156037
:1003400030BC704730B4044654E8000F40EA010561
:1003500044E80053002BF7D1156030BC704730B42F
:10036000044654E8000F00EA010544E80053002B5E
:10037000F7D1156030BC704730B4044654E8000F24
:1003800080EA010544E80053002BF7D1156030BC2A
:10039000704730B4044654E8000F00EB010544E810
:1003A0000053002BF7D1156030BC704730B40446C1
:1003B00054E8000FA0EB010544E80053002BF7D1EF
:1003C000156030BC704770B404464FF0000054E82C
:1003D000006F0D68AE4207BF44E80023012044E8E7
:1003E00000630E60002B1CBF0020F0E770BC70475C
:1003F00030B4044654E8000F88422CBF451A054625
:1004000044E80053002BF5D1156030BC7047000064
:100410000648804706480047FEE7FEE7FEE7FEE79E
:10042000FEE7FEE7FEE7FEE7FEE7FEE7390C000029
:100430000102000000487047D8B30000A0F141015C
:10044000192900D8203070472DE9FE4399461546FA
:100450008846074601AC022942D3002D40D0002037
:100460000290A8F101004FF0FF36009022E000FB5F
:10047000057201FB057011464A469047002805DCCD
:1004800054F82600304444F8260013E060682A46F9
:1004900000FB057154F8040C00FB057007E00B78B5
:1004A00090F800C001F801CB00F8013B521E002A71
:1004B000F5D1764254F8040C61688842D7DC4B468B
:1004C0002A463846FFF7C0FF54F8040C4B46A8EB09
:1004D0000001401C00FB05702A46491EFFF7B4FFCF
:1004E000BDE8FE8310B5431A934209D283188818D9
:1004F00003E010F8011D03F8011D521EF9D210BDD2
:1005000040EA01039B0703D009E008C9121F08C095
:10051000042AFAD203E011F8013B00F8013B521E15
:10052000F9D210BDD2B201E000F8012B491EFBD276
:1005300070470022F6E710B513460A4604461946EE
:10054000FFF7F0FF204610BD30B505462A460B46A2
:1005500012F8010B13F8014B08B1A042F8D01CB1FE
:10056000002802D06D1CF1E7284630BDCAB2401EFB
:1005700010F8011F8A4202D00029F9D100207047EB
:10058000421C10F8011B0029FBD1801A704710B5DE
:10059000002200E0521C835C8C5CA34201D1002B42
:1005A000F8D1D8B2E1B2401A10BD034611F8012BC0
:1005B00000F8012B002AF9D11846704730B50546DE
:1005C0000020034600E05B1C934205D2EC5CC85C53
:1005D000201A01D1002CF6D130BD2DE9F04791460B
:1005E0000F4680460446002614F8015B2DB1FFF744
:1005F00021FF0068405DC007F6D12B2D02D02D2DC4
:1006000018D0641E4A463946204600F01EF827B12D
:100610003968A14201D1C7F8008071054FF002048A
:100620000BD54042002803DD00F062FD0460A00706
:10063000BDE8F08746F48066E4E70028F8DA00F0C9
:1006400057FD04606FF00040F2E72DE9F05F82464D
:100650000078002715468B460AF10104B946302878
:1006600001D09DB113E014F8010B0127782803D0C5
:10067000582801D045B10AE00DB1102D07D100274F
:10068000102514F8010B02E0082500E00A250026D9
:10069000B0460EE005FB080005FB06F1012701EB63
:1006A00010461FFA80F8B6F5803F00D3B94614F81B
:1006B000010B294600F02AF80028EBDABBF1000F05
:1006C00005D00FB1641E00E05446CBF80040B9F1EC
:1006D000000F06D000F00CFD02210160C81EBDE82D
:1006E000F09F48EA0640FAE7064C074D06E0E0684E
:1006F00040F0010394E8070098471034AC42F6D369
:10070000FFF782FD40D1000060D100003A2800D2FE
:10071000303820F02002412A01D3A2F1370088426C
:1007200001D34FF0FF30704770B58C1810F8015BA3
:1007300015F0070301D110F8013B2A1106D110F87A
:10074000012B03E010F8016B01F8016B5B1EF9D17E
:100750002B0705D40023521E0DD401F8013BFAE704
:1007600010F8013BCB1A921C03E013F8015B01F86F
:10077000015B521EF9D5A142D8D3002070BD000004
:100780002DE9F04700268AB0DFF85891B0464FF4C3
:100790008075012437460596284606F079FE38B163
:1007A000D9F80403204203D0284606F067FE26430A
:1007B0002D1D64007F1CADB2082FEDD34FF4BE7425
:1007C000204606F065FE48B1204606F057FE46F08A
:1007D000004605AA0121002006F01CFE424D16F03D
:1007E000FF0F15D00127002437420DD009EB8401FB
:1007F000D1F81005D1F81015C0F3042055F82420C5
:10080000C1F3014102B190477F00641C082CEBD377
:10081000002E63DA4FF0FF30CDF8108058E0281931
:1008200010F8507F90F9000027F0C008401C3FD01E
:1008300008A9404605F04AF930B34FEA97194046F7
:1008400000F07CFF55F820701FB1B9F1030F03D001
:1008500006E0B9F1030F2BD104A9404605F03EF99B
:1008600002A8CDF8088006F055FD029900EB810042
:10087000D0F8000705A9C0F3014A404605F026F963
:1008800018B1BAF1020F03D012E0BAF1030F0FD181
:10089000B9F1030F08D1BAF1020F1DD00221404671
:1008A00006F020FD761CF6B217B149464046B8471F
:1008B000641C042CB3D3002E10D06A460121002002
:1008C00006F0A8FD05990098884207D00590049885
:1008D000002634460890A2E70321E0E70AB0BDE80D
:1008E000F087000000600040B81100201CB5814670
:1008F00007F0CAF906F062FF0028FBD137484E46E0
:100900000768374C01256068002821D0208835A170
:1009100005EB0040B26907F07FF86068002817D047
:10092000D6E90201CDE900012088D6E9002305EBD4
:10093000004032A107F088F8606848B1F069009083
:10094000D6E9042320883BA105EB004007F073F8AB
:100950002248001D0068800707D5606828B12088FC
:100960003E4905EB004007F053F8DFF8F48000261D
:1009700005FA06F038420AD058F826203AB16068E5
:1009800028B1208837A105EB004007F045F8761C18
:100990001A2EEDD338060AD5606840B10F480C30E6
:1009A0000268208832A105EB004007F035F83804D2
:1009B0000AD5606840B1094810300268208834A127
:1009C00005EB004007F028F80448C8300068C0076D
:1009D00000D000BE484600F069F8000028ED00E0B5
:1009E0001404002048415244204641554C54206193
:1009F0007420307825303858000000002020523014
:100A00003A2020307825303858202052313A2020A2
:100A1000307825303858202052323A20203078253E
:100A2000303858202052333A20203078253038583A
:100A30000000000020205231323A20307825303832
:100A40005820204C523A2020307825303858202029
:100A50005053523A203078253038580000BE0000FC
:100A60009801002043617573653A2025732E0000BC
:100A70004D656D4D616E616765204661756C7420D2
:100A8000416464726573733A2030782530385800B9
:100A9000427573204661756C74204164647265739D
:100AA000733A20307825303858000000BFF34F8F5C
:100AB00005480168054A01F4E06111430160BFF394
:100AC0004F8F00BFFDE700000CED00E00400FA05C9
:100AD00010B508F067FABDE8104008F0D1B9000081
:100AE00002490248091F0968006808479001002070
:100AF000044900EB400001EBC000416D806D081A15
:100B0000704700007019002000F050BA70B506461A
:100B100014460D46002000F0C3FC2246294630460C
:100B200000F006F80446002000F0E8FC204670BD06
:100B30002DE9F0471B4D0746164628780C4608B9A4
:100B400000F034FA07EB470005EBC007A046D7E9F1
:100B50001595002448374D4511D9B868441BB44257
:100B600000D334467868224641194046FFF7BAFC64
:100B7000B868361B2544A044A84200D10025A9EB43
:100B80000500B04200D206463EB1786832464119AF
:100B90004046FFF7A7FC3444354404B13D6120468C
:100BA000BDE8F0877019002070B50B4B064614465F
:100BB00018780D4608B900F0F9F9002000F070FC33
:100BC00022462946304600F009F80446002000F08D
:100BD00095FC204670BD00007019002070B50E46CF
:100BE000144900EB400001EBC0051446E86A1835D3
:100BF00020B101280FD0022805D113E0284600F0CB
:100C000009FAA04201D2002411E0224631462846CA
:100C100000F038FA0BE0284600F0FCF9A042F4D2CC
:100C20000446F2E73146284600F0FFF90446204624
:100C300070BD000070190020F0B5B5480023021DFA
:100C40000178101D01254FF0805406290BD116782C
:100C5000360708D10678C6F30316032E06D0042EF5
:100C600004D0052E02D0062907D00EE0B4F8246384
:100C7000A84FC6F304263E6002E01678360704D17A
:100C80000678C6F30316032E02D0062904D00FE01F
:100C9000A24FA14E7E670EE01678360708D106787F
:100CA000C6F30316032E06D0042E04D0052E02D060
:100CB000062907D00EE0D4F84462994FC6F34236B5
:100CC0003E6002E01678360704D10678C6F30316B4
:100CD000032E02D0062906D011E0924E376827F085
:100CE000807737600EE01678360708D10678C6F3AD
:100CF0000316032E06D0042E04D0052E02D006299A
:100D00000AD011E04FF08046C6F80C31C6F8103119
:100D1000834E361F336002E01678360704D106781A
:100D2000C6F30316032E02D0062905D00CE07C4F33
:100D3000032664373E600AE01678360704D1067849
:100D4000C6F30316032E02D006290DD014E0764F09
:100D500005263E60744E78363560734E0836336033
:100D60003F263F1D3E6002E01678360704D1067824
:100D7000C6F30316052E02D0062957D062E06B4E4B
:100D800036686B4F3E60694E361D36683F1D3E60CB
:100D9000664E083636683F1D3E60644E0C36366837
:100DA0003F1D3E60614E103636683F1D3E605F4E0F
:100DB000143636683F1D3E605C4E183636685C4F10
:100DC00020373E60594E1C3636683F1D3E60574EF8
:100DD000203636683F1D3E60544E243636683F1D2F
:100DE0003E60524E283636683F1D3E604F4E2C36D0
:100DF00036683F1D3E604D4E303636684C4F4037AA
:100E00003E604A4E343636683F1D3E60474E3836A7
:100E100036683F1D3E60454E3C3636683F1D3E609D
:100E2000424E403636683F1D3E6002E01678360777
:100E300008D10678C6F30316032E06D0042E04D07C
:100E4000052E02D0062907D019E0D4F85812394AE5
:100E500001F04F01116002E0117809070FD100780D
:100E6000C0F30310032803D0042801D0052806D1BD
:100E700031480168C90702D06FF001010160D4F860
:100E80003001062808D1D4F83401062804D12B48B3
:100E9000016841F48061016022487438016841F4BE
:100EA00070010160BFF34F8FBFF36F8F4FF01021C0
:100EB000D1F80002002803DBD1F80402002822DA6E
:100EC0001F4A15601F480468002CFCD01524C1F887
:100ED00000420568002DFCD0C1F8044201680029D9
:100EE000FCD0136001680029FCD0BFF34F8F0D4880
:100EF000F0380168144A01F4E06111430160BFF366
:100F00004F8F00BFFDE7124910480860F0BD000098
:100F1000E00F00F0403501400DF0ADBA00C00740D1
:100F20003C050040FCED00E01056004004040010B9
:100F300020C50040E40E0040000400403C17004083
:100F400004E5014000E401400400FA050090D003EC
:100F5000B402002010B5054C206818B904A12B205C
:100F600000F082FB2068BDE81040004758010020D7
:100F70002E2E5C2E2E5C2E2E5C2E2E5C2E2E5C2EAB
:100F80002E5C6D6F64756C65735C6E7266785C6404
:100F90007269766572735C7372635C7072735C6E97
:100FA0007266785F7072732E6300000010B5124C89
:100FB00002202061606111A0A06104F17800E0616D
:100FC0004FF4007020620020A06260620BA1A16457
:100FD000E06204F51E71E1641021A065C4E91410FB
:100FE000E06509A1E01DFFF7E0FA08A12046FFF740
:100FF000DCFA2020A07110BD701900205465726DBC
:10100000696E616C0000000052545400534547471C
:10101000455200000269C1688A4203D88068401ABC
:10102000104400E0501A401E70472DE9F047C46894
:101030001746894606464FF000083069A04201D99C
:10104000051B02E0B168201A0D1AB0686D1E001B66
:10105000A84200D80546BD4200D33D4670682A46E6
:1010600020444946FFF73EFAB0687F1B2C44A84451
:10107000A944A04200D10024F460002FDDD14046F5
:10108000BDE8F0872DE9F04104468846D4E902071F
:10109000C51BE168606816460844B54206D941465A
:1010A000FFF720FAB819E060BDE8F0812A46414612
:1010B000FFF718FA761B08EB050132466068FFF768
:1010C00011FAE660F0E700000FB4084B10B504A970
:1010D00002AA039800F01FF8044602A9002000F0BD
:1010E00085F8204610BC5DF814FB0000ED110000EF
:1010F00000487047B802002002E008C8121F08C16B
:10110000002AFAD170477047002001E001C1121F88
:10111000002AFBD170472DE9F84F99469246884640
:101120000546002706E025280AD051464A46904742
:101130006D1C7F1C28780028F5D13846BDE8F88F53
:10114000002315F8011F18462E2915D115F8011F87
:1011500004232A290DD06FF02F022978A1F1300441
:10116000092C09D800EB800002EB400008446D1CFC
:10117000F3E758F8040B6D1C2A78002ADDD0632AA7
:1011800007D0732A0FD0104651464A4690477F1C1D
:101190002AE018F8042B8DF8002000218DF80110AA
:1011A0006E46012103E058F8046B4FF0FF315A07F7
:1011B0004FF0000401D409E0641C84420BDA8C4235
:1011C000FADB325D002AF7D105E0641C8C42FCDBBF
:1011D000305D0028F9D1274404E016F8010B514690
:1011E0004A469047641EF8D26D1CA3E70A68531C58
:1011F0000B6010707047800701D0002070470120FD
:101200007047C3688B4206D811440069491E814269
:1012100001D8012070470020704700002DE9FE43EF
:1012200015460F46804672B606F02EFD06F0C6FA49
:101230000028FBD16FF48041224C18EB01004FF0E5
:10124000010622D00128606814D030B120883A46C7
:1012500006EB00401CA106F0DFFB21480068C00738
:1012600000D000BE2A4603B039464046BDE8F043F0
:1012700000F064B80028F0D020882B8806EB0040EE
:1012800018A16A6806F0CFFBE7E760680028E4D0A1
:10129000A86807F06BFD0346D5E90001CDE9001011
:1012A0000297208816A106EB0040AA6806F0D6FB3C
:1012B00060680028D1D020881BA106EB004006F012
:1012C000A7FBCAE774040020554E4B4E4F574E20E3
:1012D0004641554C542061742030782530385800F0
:1012E000F0ED00E0415353455254494F4E204641E2
:1012F000494C45442061742025733A25750000004F
:101300004552524F52202575205B25735D20617434
:101310002025733A25750D0A50432061743A203018
:101320007825303878000000456E64206F662065AF
:1013300072726F72207265706F72740008B501234B
:101340008DF800309DF80030144B186059609A6099
:101350006FF48041401807D001280FD1DA60D868B7
:1013600000889861D86807E01A6118698068586138
:1013700018690068986118694068D86118685868E9
:101380009868D868186958699869D86972B600BFB2
:101390009DF800000028FBD162B608BD6412002051
:1013A000014802F0FCBC00006801002070B5144642
:1013B0000E46050004D10B4940F2C51000F054F967
:1013C0003CB12868012EC4600AD000218160002051
:1013D00070BD04494FF4E37000F046F9072070BD7A
:1013E0000121F3E7D4BB000038B50E48082358228A
:1013F000416800910C49006804F063F900280FD19E
:101400000A4A69460A4802F0CFFC040008D10121CB
:10141000074802F0A0FD064901200839087020465F
:1014200038BD000068AD000084120020E59C00007B
:101430006801002070B516460D46040004D10C4921
:1014400040F2D51000F010F90A48854201D9072072
:1014500070BD0948266102F0A2FC28446060A068C3
:1014600000B1A5602146BDE87040002009F014B825
:10147000D4BB000017FCFF006801002010B5040079
:1014800004D106494FF4F57000F0EEF80020214633
:101490002076BDE81040012008F0FEBFD4BB00005C
:1014A00010B508F085FB012803D004A11D2000F031
:1014B000DBF8BDE8104000F04FB800002E2E5C2E87
:1014C0002E5C2E2E5C2E2E5C2E2E5C2E2E5C636FE0
:1014D0006D706F6E656E74735C6C69627261726957
:1014E00065735C7574696C5C6170705F7574696C50
:1014F0005F706C6174666F726D2E630010B508F0DA
:1015000057FB012803D004A12B2000F0ADF8BDE863
:10151000104000F029B800002E2E5C2E2E5C2E2EDE
:101520005C2E2E5C2E2E5C2E2E5C636F6D706F6EAB
:10153000656E74735C6C69627261726965735C7507
:1015400074696C5C6170705F7574696C5F706C61FC
:1015500074666F726D2E630072B602480168491C92
:10156000016070478801002003490868401E086038
:1015700000D162B6704700008801002070B50546B2
:1015800008680C46411C04D005F030FF206805F0C7
:1015900095FE6068411C02D0002105F07DFE29689F
:1015A000A069C1F82405607D227D29681043C1F837
:1015B0006C05D4E900122868C0F81425C0F80C1591
:1015C000207D012814D1A068411C02D0002105F023
:1015D00063FEE068411C04D005F008FFE06805F0F8
:1015E0006DFED4E902122868C0F80825C0F810156D
:1015F00070BD70B5054608680C46411C04D005F066
:10160000FFFE206805F064FE6068411C02D00021E6
:1016100005F04BFE2968A069C1F82405607D217D95
:101620002A680843C2F86C05D4E900122868C0F89B
:101630000C15C0F81425207D012814D1A068411C88
:1016400002D0002105F031FEE068411C04D005F015
:10165000D7FEE06805F03CFED4E902122868C0F825
:101660000825C0F8101570BD1CB56A46ADF800001D
:101670000191002144F20200FFF7D0FD1CBD0000E3
:101680002DE9F0470546C61C90460F464FF001096C
:101690000020FFF705FF1B4C20683860D4E90001EB
:1016A000401AA16804F21C47081A0EE001213846CE
:1016B00004F052F803F08AFC0146384604F04CF876
:1016C000D4E90001401AA168081A401C8642EDD8EE
:1016D000B8F1000F03D0052065F3891002E0062061
:1016E00065F39F50A2682168114004EB8101C86036
:1016F0002068304420600020FFF700FF4846BDE826
:10170000F08700004C15002030B482680468531C38
:101710008360A154D0E901128A4202D330BC05F0A3
:101720003FBA30BC70470000034803C8814201D172
:1017300001207047002070474C15002002490844E2
:1017400090F9300070470000B811002070B5816832
:1017500004464A8B002A4DD0888B00284AD0121AA2
:10176000084495B200F120016A1C1F30FEF7BAFE52
:10177000A068818B491E8183A068418B491E4183EB
:101780008DB308221C49206905F0CAF9204603F0F0
:1017900070FF8188C088814211D1A06817A2818B17
:1017A000431808212046203304F068FD204600F04D
:1017B0003FF929462046BDE8704002F0B5B9204601
:1017C00000F0A2F9204600F033F9A0680BA2818B4B
:1017D000431808212046203304F050FD2046BDE880
:1017E000704000F05BB92069BDE87040044A03A175
:1017F00005F096B970BD00002C1A0000257300009A
:10180000C4AF000070B504468068428B818B521AC9
:1018100015042D0C48D0084400F121012A4620303F
:10182000FEF760FEA068418B491E4183204603F00D
:1018300020FF8188C08881420CD1A0681BA2818BC7
:10184000431808212046203304F018FD4FF4707629
:10185000C4B913E0204600F057F9204600F0E8F83C
:10186000A06812A2818B431808212046203304F07F
:1018700005FD2046BDE8704000F010B90CA13046CF
:10188000FFF7F2FE206918B909A13046FFF7ECFE18
:10189000154A06A1206905F043F96D1EA9B220463C
:1018A000BDE8704002F040B970BD00002573000033
:1018B0002E2E5C2E2E5C2E2E5C2E2E5C2E2E5C2E62
:1018C0002E5C636F6D706F6E656E74735C6C6962B5
:1018D0007261726965735C636C695C6E72665F638A
:1018E0006C692E6300000000C8AF00002DE9F041D4
:1018F000044680680F46D0F84813828B11F0010629
:10190000418BA1EB02039DB24FF4BF730BD0994200
:1019100001D9002D7ED0A068818B0844002180F879
:10192000207066B113E099427CD8002DF3D0831863
:1019300003F120012A46481CFEF7D4FDEBE7A0681E
:10194000428B521C92B24283A068203281544DB324
:10195000204603F08EFE8188C08881420ED1A068A7
:1019600031A2818B431808212046203304F086FCE5
:10197000A81B81B2204602F0D7F821E0204600F0F3
:10198000C3F8A06828A2818B431808212046203381
:1019900004F074FC204600F081F80121204602F09A
:1019A000D5F90DE03EB1A068428B521C92B2428341
:1019B000A068203281543A461CA1206905F0B0F895
:1019C000A168888B401C8883204602F09AF8002882
:1019D000204603D0BDE8F04102F0B2B802F0C6FEE6
:1019E00000281FD0204603F044FE0546C088A98881
:1019F000401A401E81B2204602F024F8204602F030
:101A00009FF8E888A988401A81B2204602F0AAF916
:101A1000288800E006E0401E81B22046BDE8F04183
:101A200002F094B9BDE8F081257300002563000041
:101A300070B504004FF4B27503D108A12846FFF732
:101A400013FE206918B905A12846FFF70DFE20698D
:101A5000BDE870400F4A10A105F062B82E2E5C2E32
:101A60002E5C2E2E5C2E2E5C2E2E5C2E2E5C636F3A
:101A70006D706F6E656E74735C6C696272617269B1
:101A800065735C636C695C6E72665F636C692E6320
:101A900000000000BCAF00002573000070B504001A
:101AA0004FF4B87503D108A12846FFF7DDFD206982
:101AB00018B905A12846FFF7D7FD2069BDE8704099
:101AC0000F4A10A105F02CB82E2E5C2E2E5C2E2E67
:101AD0005C2E2E5C2E2E5C2E2E5C636F6D706F6EF6
:101AE000656E74735C6C69627261726965735C6364
:101AF0006C695C6E72665F636C692E630000000047
:101B0000B3AF00002573000070B504004FF4B57545
:101B100003D108A12846FFF7A7FD206918B905A140
:101B20002846FFF7A1FD2069BDE870400F4A10A1CB
:101B300004F0F6BF2E2E5C2E2E5C2E2E5C2E2E5C1C
:101B40002E2E5C2E2E5C636F6D706F6E656E7473DF
:101B50005C6C69627261726965735C636C695C6E0E
:101B600072665F636C692E6300000000B0AF000016
:101B7000257300002DE9F04F4FF000099FB0054696
:101B80004E464C46CDF8509001F004FE284602F037
:101B90001DFFA868CA464FF4C07100F5D070FEF76B
:101BA000C8FCA86800F12001428B00F5D070FEF758
:101BB00099FCA86800F5D07008F0FCF9A86800F559
:101BC000D07000F067FCA968401CC883284601F06B
:101BD00045FF284601F095FF10B9284601F0B0FFF7
:101BE000AA680C2304A912A8203203F099FB03462B
:101BF000129840B15BB170A20221284604F03EFB6E
:101C00001FB0BDE8F08F284601F09AFFF8E7704951
:101C100070480027A1EB00080DF1100B13E008D36A
:101C20006DA0009071A202212846049B04F026FBBF
:101C3000E6E700EBC704606801685BF82900FEF77F
:101C4000A6FC20B17F1C6348B7EBD80FE7D92078FA
:101C500020B168A140F68200FFF706FD4FF00008B2
:101C6000CDF870806068C7680FB1A9684860606887
:101C700009F101044FF00009806803901298844232
:101C80005CD25BF8240069A1FEF781FCD0B15BF85F
:101C9000240067A1FEF77BFCA0B15BF8240008F0EC
:101CA0000BFFB8B10020139013A800905BF824300C
:101CB00022462846039901F0F3FD02283ED01399ED
:101CC0008A4439E0A868D0F8481341F00201C0F80E
:101CD000481333E018A84A46009009F101091CABEB
:101CE0002146039801F0C8FAB9F1000F26D01C98DC
:101CF00020B301685BF82400FEF749FC0028BDD141
:101D00001C98C168A1B1BAF1000F0BD0284601F0B0
:101D1000A5FE284601F0F5FE10B9284601F010FF97
:101D200045A23CE0A9F10101DDF80C8026461491A2
:101D300080684FF000090390641C9FE7BAF1000F20
:101D400010D0A86800F5D071C28B2030FEF7CAFB16
:101D5000A9680C23C88B4883AA6804A912A820325A
:101D600003F0DEFAB8F1000F12D018A800901CABF7
:101D700031464046149A01F07FFAA9681C980BEB93
:101D8000860248601299C368891B284698470AE072
:101D900027B104AA28461299B84704E032A20221CA
:101DA000284604F06BFAA868D0F8481321F0020125
:101DB000C0F8481324E700006E6F74207465726DDC
:101DC000696E617465643A2025630D0A00000000A5
:101DD000F0D1000060D100003A20636F6D6D616E3C
:101DE00064206E6F7420666F756E640025732573B2
:101DF0000D0A00002E2E5C2E2E5C2E2E5C2E2E5CEC
:101E00002E2E5C2E2E5C636F6D706F6E656E74731C
:101E10005C6C69627261726965735C636C695C6E4B
:101E200072665F636C692E63000000002D6800001D
:101E30002D2D68656C7000004572726F723A2072C9
:101E40006571756573746564206D756C7469706C0B
:101E5000652066756E6374696F6E2065786563755D
:101E600074696F6E730D0A00506C65617365207341
:101E7000706563696679206120737562636F6D6D4B
:101E8000616E642E0D0A00008068D0F84803C0F32C
:101E9000C000704710B58AB02022144901A8FEF78F
:101EA00021FB062001900820029000208DF81800E8
:101EB0000E48032401231A4601A93838009404F07F
:101EC000B7FB18B10A4ABE21FEF7A4F9074801235F
:101ED0001A4600211C38009404F0AAFB002803D005
:101EE000034AC221FEF796F90AB010BD9CAC00006F
:101EF000A45200002DE9F0410446C0688EB00D46A2
:101F00000026C068324601A906F06CFA18B100201C
:101F10000EB0BDE8F0816DB1019805F084FFA168B5
:101F2000D1F83803401CC1F8380300F0070001283D
:101F300079D10126204603F09CFB054680880128C4
:101F400004D9401E81B2204601F00CFF28880128E8
:101F500004D9401E81B2204601F0E6FD2046FFF77D
:101F600067FD2EB131A20221204604F087F95AE024
:101F70004FF0010800230C2202A9019805F062FF2E
:101F800004980590BDF80C00ADF81800BDF80E00DF
:101F9000ADF81A008DF81D8002980C2700F00300A0
:101FA000012802D0022818D032E002983B46860A67
:101FB000C0F3C2008DF81C00029808A9C0F3831575
:101FC000AA00019805F03EFF2069009005AB2A4663
:101FD00008A9304605F06CFE1AE00298850DC0F3A2
:101FE000C2008DF81C00082D01D22E4600E0082604
:101FF0003B46324608A9019805F024FF3744AD1B43
:1020000005AA314608A8236905F036FD002DEAD15E
:10201000019805F008FFE068002201A9C06806F0F9
:10202000E1F90028A6D0012072E700004C6F73741C
:10203000206C6F6773202D20696E63726561736514
:10204000206C6F67206261636B656E6420717565DB
:1020500075652073697A652E0D0A00002DE9F0413F
:102060001E4617460D46040000D01DB909A1EA20FE
:10207000FFF7FAFA606818B906A1EB20FFF7F4FA47
:10208000606833463A4601680C692946A446BDE8B3
:10209000F04160472E2E5C2E2E5C2E2E5C2E2E5C88
:1020A0002E2E5C2E2E5C636F6D706F6E656E74737A
:1020B0005C6C69627261726965735C636C695C6EA9
:1020C00072665F636C692E630000000070B50446A1
:1020D00040680E460025007A38B1A0680068FFF716
:1020E000CDF908B108281AD10025BEB96068007A78
:1020F00050B90B4A0021A068FFF758F96168050044
:102100004FF00100087209D1A068224640F6CD4187
:102110000068FFF78FF90546FEF7F6FC284670BD0C
:10212000CDA2000010B541680A6041684B6040686C
:1021300000210172FEF7E8FC02490120087000202E
:1021400010BD00000402002070B51C0015460E46AC
:1021500003D106A16620FFF787FA2A463146002000
:10216000FEF7D4FC2060002070BD00002E2E5C2EF7
:102170002E5C2E2E5C2E2E5C2E2E5C2E2E5C636F23
:102180006D706F6E656E74735C6C6962726172699A
:1021900065735C636C695C7274745C6E72665F63B9
:1021A0006C695F7274742E630000000080680068C0
:1021B000FFF764B92DE9F05F5FEA030815460E46A4
:1021C00003D11DA17420FFF74FFA2B480068C00708
:1021D0000FD0DFF8A8B000244FF0050AB14600BFC9
:1021E00009EB04012A460020FEF7DEFC060003D0BE
:1021F00011E0C8F8005018E09BF8000088B10A27E9
:102200001F494FF47A4088477F1EF9D1AAF1010097
:102210005FEA000A0CD001218BF800103444AD1B9A
:10222000DED1002CE5D0C8F800400020BDE8F09FCA
:1022300000218BF80010F4E72E2E5C2E2E5C2E2E43
:102240005C2E2E5C2E2E5C2E2E5C636F6D706F6E7E
:10225000656E74735C6C69627261726965735C63EC
:102260006C695C7274745C6E72665F636C695F72D9
:1022700074742E6300000000F0ED00E00402002002
:1022800011B000007CB500260446019601AB012286
:1022900069462046FFF7E2FE019800281CD09DF811
:1022A00000007F28F2D806F09BF8A068417821B1A1
:1022B000012964D0022966D16AE0217E9DF8005090
:1022C000A9420DD1408B0028204606D0FFF752FCD2
:1022D0000221204600F0CAF87CBD01F031FCF7E78E
:1022E000092D1CD004DC002DD0D0082D04D11FE016
:1022F0001B2D12D07F2D24D0FEF79CF80068405D86
:1023000010F03E0FC2D02046FFF7BEFD9DF8001032
:1023100000B32046FFF7EAFAB8E7012136E020468D
:10232000FFF7B2FD0028B1D0204600F0B9F8ADE7C4
:102330002046FFF7A9FD0028A8D02046FFF706FA9F
:10234000A4E72046FFF7A0FD00289FD02046FFF716
:1023500059FA9BE7A268508BB0F5BF7F96D8908B57
:102360001318401C908383F82010A068818B0844C8
:1023700080F82060A068418B491C418386E79DF866
:1023800000105B2901D0002100E0022141707DE7AF
:10239000002141702046FFF777FD00289CD09DF872
:1023A000000041380C28B7D2DFE800F007090E2DF5
:1023B000064C06500606065468E7012100E000219D
:1023C000204602F0E7F961E7204603F052F905469E
:1023D00000886988884203D1A988EA8891429BD005
:1023E000698988424FF00101204606D101F02AFB9D
:1023F0006989204601F098FB01E001F0A7FCA06884
:10240000818B491C15E0204603F033F9054600880E
:10241000297B491C884202D1A988012987D001283B
:102420004FF00101204606D001F07EFBA068818BB1
:10243000491E81832AE701F095FC6989204601F055
:1024400085FCF3E7204601F009FB1FE7204601F079
:102450002EFB1BE7A068D0F8482301219143D0F858
:10246000482361F30002C0F848230FE7826802297D
:1024700011700CD18268002182F82010826891834B
:102480008268518302A20321036803F0F7BE7047FC
:1024900025730000002801D0FEF772B870470000D5
:1024A0002DE9F04FA5B04FF000080546CDF8348077
:1024B000CDF8308080684746418BA1F27F114942B8
:1024C00089B25FEA010B71D0828B00F1200100F527
:1024D000D070FEF707F8A8680024818B084480F8C4
:1024E000A041FDF7A7FF20900168A8680C23828B0C
:1024F0000244D27F895CC0F84443AA6801F0010914
:102500000EA91FA802F5D07202F00AFF0E98FFF77D
:10251000C1FF86B2A2460A9407941F9921B101EB2C
:102520000900401EB8426BD8B9F1000F01D0002657
:1025300005E00EA850F82700FFF7ACFF86B2002494
:102540001BA822460090641C0AAB3946504600F096
:1025500093FE0A9800287CD001680EA8324650F8F5
:102560002700FEF72BF80028079802D00028E7D0B4
:102570006FE0E0B10A980068FFF78CFF0C9980B219
:10258000884200D90C90BBF1000F2BD021A80090FD
:1025900007AB42463946504600F06EFE0A98006886
:1025A0008319079800688119002015E042E0601E39
:1025B0000D900A980068FFF76DFF80B20C90801BA9
:1025C00058450FDA80B20CE011F800C0624506D120
:1025D000401C0004000C10D01A5C002AF4D1834582
:1025E00000D983460A98B4F101080790A8D267A2DF
:1025F0000421284603F042FE2BE04FF6FF70EEE781
:1026000000241BA822460090641C0AAB39465046A1
:1026100000F032FE4CB10A9800280BD00EA850F8FA
:10262000270008F049FAA0B907E058A2042128467B
:1026300003F024FE25B0BDE8F08F0A9801680EA8CB
:1026400050F82700FDF7A3FF0028DAD10A98D0F848
:1026500008A0BAF1000F09D00A9838B11F997F1C61
:10266000BFB201EB09008742FFF457AF079800287B
:10267000E0D00D984146404556D19AF8000038B157
:102680001BA80A46009007AB3946504600F0F4FDFF
:1026900007980068FFF7FEFEB04206D007985A463A
:1026A00000688119284601F061F920980368A8683C
:1026B000818B421892F820209A5CD20715D0408B6B
:1026C0008142B7D2284602F0D4FFA9688488888B5B
:1026D000401C8883284602F0CCFF8088A0421FD18E
:1026E0000121284601F032FBA4E7D0F84813C907BE
:1026F00011D0D0F8481321F00101C0F8481320216F
:102700002846FFF7F3F8A868D0F8481341F0010114
:10271000C0F848138EE720212846FFF7E7F889E73D
:10272000284601F00DFA85E7002128460C9A07F0AB
:1027300089F90DF16C090D9C0EE00AAB2246394671
:102740005046CDF8009000F097FD0A980C9A016869
:10275000284607F077F9641C4445EED917A20321F7
:1027600028462B6803F08AFDAB6816A2082128468C
:10277000203303F083FD284601F0B2FA07985A4649
:1027800000688119284601F0F1F853E7546162208E
:1027900066756E6374696F6E3A20636F6D6D616EFE
:1027A000647320636F756E746572206F76657266F0
:1027B0006C6F7765642E0D0A000000000D0A25730A
:1027C000000000002573000070B505460C0004D120
:1027D00007A14FF41260FEF747FF002D06D0A06856
:1027E000D0F8481341F02001C0F8481370BD000034
:1027F0002E2E5C2E2E5C2E2E5C2E2E5C2E2E5C2E13
:102800002E5C636F6D706F6E656E74735C6C696265
:102810007261726965735C636C695C6E72665F633A
:102820006C692E630000000000238B540A46006888
:10283000194603F023BD000070B5044640680D46FC
:1028400090F8280030B1A0680068FEF717FE08B1C4
:1028500008280CD1012685B1606904F055F961683A
:1028600000220831606904F00BF908B1062070BD40
:10287000606880F82960002070BD606890F82800CA
:1028800048B9074A0021A068FEF790FD616800285A
:1028900081F82860F0D12046BDE8704007F014BBF5
:1028A0004DA3000070B5044640680D4602606068A4
:1028B00000224360606880F82820606880F8292042
:1028C000606820220830FDF70DFE2C61074A29467A
:1028D000606904F0D5F8050005D1E06806F00AF952
:1028E000206906F007F9284670BD0000E1A5000048
:1028F0002DE9F0411C0016460F46054603D106A1FE
:10290000D220FEF7B1FE266022463946E868BDE8CF
:10291000F04106F005B800002E2E5C2E2E5C2E2E07
:102920005C2E2E5C2E2E5C2E2E5C636F6D706F6E97
:10293000656E74735C6C69627261726965735C6305
:102940006C695C756172745C6E72665F636C695F02
:10295000756172742E63000010B50446406904F07E
:10296000D3F8A0680068BDE81040FEF787BD0000FE
:102970002DE9FC411D0016460F46044603D11AA15D
:10298000E620FEF771FE2E602A463946206906F0E1
:1029900013F8050025D16069234A0178515C19B10B
:1029A000001D06F063FF02E00C3006F057FDC0B9D1
:1029B000FF20009001236A4601A9206906F056F81D
:1029C00078B900980199C2B2606904F08DF80546A3
:1029D000606890F8290020B11DB92069009906F0BF
:1029E00031F82846BDE8FC812E2E5C2E2E5C2E2E62
:1029F0005C2E2E5C2E2E5C2E2E5C636F6D706F6EC7
:102A0000656E74735C6C69627261726965735C6334
:102A10006C695C756172745C6E72665F636C695F31
:102A2000756172742E630000340100202DE9F843B3
:102A30001F4614468846050002D0B8F1000F03D1A6
:102A40001EA1BB20FEF710FE6868006818B91BA124
:102A5000BC20FEF709FE002628E000BF686808EBEE
:102A600006016B460268D2F80CC02246E04718B156
:102A700012A1C620FEF7F8FD0098844203D20FA1F0
:102A8000C720FEF7F1FD00980644241A70B9A86823
:102A9000017803290AD000BFD0F848138906FBD576
:102AA000D0F8481321F02001C0F84813002CD5D1EC
:102AB000002F01D000983860BDE8F8832E2E5C2EE0
:102AC0002E5C2E2E5C2E2E5C2E2E5C2E2E5C636FCA
:102AD0006D706F6E656E74735C6C69627261726941
:102AE00065735C636C695C6E72665F636C692E63B0
:102AF0000000000070B5084C050009D010342168B2
:102B0000002907D008682060496828468847F6E70A
:102B10000834F4E770BD0000A4110020054A01212B
:102B200020B1012805D19170FFF7E4BF517000205A
:102B3000FAE77047A41100203EB5044603F072FD89
:102B400038B103B02046BDE830400022114603F002
:102B5000F3BB06490648CDE900010346029105A2F0
:102B60000821204603F08AFB3EBD0000B0D40000DF
:102B7000000000004170706C69636174696F6E20C1
:102B8000616464726573733A256420283078253057
:102B90003858292C2073697A653A2025642028301A
:102BA0007825303858290D0A00000000F8B5144681
:102BB0000E46050004D121A14FF48770FEF754FDA5
:102BC000A86818B1686808B1286820B91BA140F24C
:102BD0000F10FEF749FD012E03D0284603F01CFD1F
:102BE00030B12846BDE8F84001221B4903F0A4BBE0
:102BF000022E08D0236801B02846BDE8F04017A295
:102C0000022103F03BBB1CA16068FDF7C0FC68B16A
:102C10001AA16068FDF7BBFC40B16068009019A282
:102C200002212846236803F029FBF8BD2846BDE8A9
:102C3000F8401BA2082103F021BB00002E2E5C2EC1
:102C40002E5C2E2E5C64656D6F5F636C695F636DD7
:102C500064732E630000000054AC000025733A201A
:102C600062616420706172616D6574657220636F6A
:102C7000756E740D0A0000002D7400002D2D746512
:102C80007374000025733A20756E6B6E6F776E203B
:102C9000706172616D657465723A2025730D0A006A
:102CA00044756D6D792074657374206F7074696FED
:102CB0006E2E0D0A00000000012904D0136804A242
:102CC000022103F0DBBA0949002048607047000088
:102CD00025733A2062616420706172616D6574656C
:102CE0007220636F756E740D0A00000000000020F2
:102CF000012904D0136804A2022103F0BFBA0949D4
:102D0000012008707047000025733A20626164203A
:102D1000706172616D6574657220636F756E740D9C
:102D20000A00000000000020012904D0136804A25A
:102D3000022103F0A3BA094900200870704700007F
:102D400025733A2062616420706172616D657465FB
:102D50007220636F756E740D0A0000000000002081
:102D600070B514460D460646012902D003F054FC06
:102D700030B13046BDE870400022114603F0DCBAA5
:102D80002368022D01D904A200E00AA23046BDE862
:102D90007040022103F072BA25733A206261642008
:102DA000706172616D6574657220636F756E740D0C
:102DB0000A00000025733A20706C6561736520730A
:102DC00070656369667920737562636F6D6D616E9E
:102DD000640D0A002DE9F04714460D46814603F0C4
:102DE0001BFC30B14846BDE8F0470022114603F015
:102DF000A3BA022D07D048462368BDE8F04728A2B1
:102E0000022103F03BBADFF8B48098F801001428DF
:102E100001D32BA206E06068FDF7B2FB86B2212E3B
:102E200002D32DA2022132E0002567680AE000BF2C
:102E3000FDF700FB0068795D405C10F0380F2BD087
:102E40006D1CEDB2B542F3D3284E002505EB4510BD
:102E500030446168FDF79BFB00281FD06D1CEDB26C
:102E6000142DF3D398F80110454601EB4110491C8D
:102E700088F8011030441EA16268FEF725F91D4B49
:102E8000212269781948FDF7DFFA1BA2082148467C
:102E9000BDE8F04703F0F2B91FA2C3E72EA2C1E7D5
:102EA00025733A2062616420706172616D6574659A
:102EB0007220636F756E740D0A0000000000002020
:102EC000636F6D6D616E64206C696D6974207265ED
:102ED00061636865640D0A00746F6F206C6F6E67C4
:102EE00020636F6D6D616E640D0A00008004002028
:102EF00025730000D9A00000636F6D6D616E6420C2
:102F00006164646564207375636365737366756C6F
:102F10006C790D0A0000000062616420636F6D6DC2
:102F2000616E64206E616D65202D20706C6561732B
:102F30006520757365206F6E6C7920616C706861B7
:102F40006E756D65726963616C206368617261633F
:102F5000746572730D0A00006475706C6963617446
:102F6000656420636F6D6D616E640D0A0000000082
:102F70002DE9F84314460D46804603F04DFB30B171
:102F80004046BDE8F8430022114603F0D5B9022DB2
:102F900003D014A2022123681DE00025184F194E0A
:102FA00009E000BF05EB451038446168FDF7EFFA12
:102FB00070B16D1CEDB270788542F3D360680090FB
:102FC00011A202214046236803F058F9BDE8F883B6
:102FD000636814A2082101B04046BDE8F04303F045
:102FE0004DB9000025733A206261642070617261FE
:102FF0006D6574657220636F756E740D0A00000054
:10300000800400200000002025733A20756B6E6F4D
:10301000776E20706172616D657465723A202573F8
:103020000D0A000064796E616D696320636F6D6DD8
:10303000616E643A2025730D0A0000002DE9F0410D
:1030400017460C468046012902D003F0E5FA30B15C
:103050004046BDE8F0410022114603F06DB9022C54
:1030600002D01BA23B6811E00024204E204D08E056
:1030700004EB441030447968FDF789FA60B1641CB0
:10308000E4B268788442F3D37B681AA24046BDE874
:10309000F041022103F0F2B8132C14D06878001B21
:1030A00000EB401204EB4410304400F12101FDF725
:1030B00019FA687816A2401E68704046BDE8F041D3
:1030C000082103F0DBB8002086F87302F1E7000066
:1030D00025733A2062616420706172616D65746568
:1030E0007220636F756E740D0A000000800400206A
:1030F00000000020646964206E6F742066696E644D
:1031000020636F6D6D616E643A2025730D0A0000B7
:10311000636F6D6D616E642072656D6F766564209E
:103120007375636365737366756C6C790D0A000063
:10313000F8B514460D46074603F06EFA30B138462E
:10314000BDE8F8400022114603F0F6B8012D08D082
:10315000236801B03846BDE8F04013A2022103F015
:103160008DB8184D687838B117A20821384603F099
:1031700085F800241A4E13E03846BDE8F84019A23D
:10318000042103F07BB800BF04EB441030440090EE
:1031900023461DA20821384603F070F8641CE4B2EF
:1031A00068788442F0D3F8BD25733A2062616420C8
:1031B000706172616D6574657220636F756E740DF8
:1031C0000A0000000000002044796E616D696320F0
:1031D000636F6D6D616E64206C6973743A0D0A00E3
:1031E00080040020506C6561736520616464207305
:1031F0006F6D6520636F6D6D616E647320666972BB
:1032000073742E0D0A0000005B2533645D20257366
:103210000D0A000010B5044603F004FA30B1204650
:103220000022BDE81040114603F086B81F21BDE81A
:10323000104002A20320FCF7EDBF00002E2E5C2EF2
:103240002E5C2E2E5C2E2E5C2E2E5C2E2E5C636F42
:103250006D706F6E656E74735C6C696272617269B9
:1032600065735C636C695C636C695F7574696C73CE
:103270005F636D64732E63002DE9F05F1C000A9F8D
:1032800015468846064603D121A1FF20FEF7ECF93A
:1032900027B91FA14FF48070FEF7E6F94FF000093F
:1032A000B8F1000F0BD026B3307840B372683946BE
:1032B000284690473868E0B12760BDE8F09F224972
:1032C0002248A1EB0008B5EBD80F15D2DFF880A09B
:1032D000002683460AE000BF0BEBC607786801684A
:1032E0005AF82500FDF753F920B1761CB6EBD80F3C
:1032F000F2D301E0786808E0C4F80090DDE7706878
:1033000000EB051001680029F6D02060D5E7000029
:103310002E2E5C2E2E5C2E2E5C2E2E5C2E2E5C2EE7
:103320002E5C636F6D706F6E656E74735C6C69623A
:103330007261726965735C636C695C6E72665F630F
:103340006C692E6300000000F0D1000060D1000025
:10335000BC0200202DE9F04115460F46044603F05B
:1033600061F930B12046BDE8F0410022114602F07B
:10337000E3BF0126214C7F1E0ED0012F14D06068C0
:10338000022F22D0002837D020881DA106EB004054
:10339000BDE8F04104F03CBB606800282CD02088D8
:1033A00023A106EB0040F3E76068002824D00A223E
:1033B00000216868FDF711F90246208821A106EB7B
:1033C0000040BDE8F04104F027BB002814D00A22D9
:1033D0000021A868FDF701F907460A220021686864
:1033E000FDF7FBF8024620883B4606EB0040BDE8AF
:1033F000F0411AA104F017BBBDE8F081740400206D
:1034000074657374206572726F72206D6573736179
:1034100067652077697468206D6F726520746861D4
:103420006E203320617267756D656E7473000000E5
:1034300074657374206572726F72206D6573736149
:103440006765000074657374206572726F72206D19
:103450006573736167653A20256400007465737451
:10346000206572726F72206D6573736167653A20B3
:1034700025642025640000002DE9F04115460F4623
:10348000044603F0CFF830B12046BDE8F0410022F9
:10349000114602F051BF0226214C7F1E0ED0012F93
:1034A00014D06068022F22D0022837D320881DA1B3
:1034B00006EB0040BDE8F04104F0AABA60680228BB
:1034C0002CD3208823A106EB0040F3E76068022894
:1034D00024D30A2200216868FDF77FF8024620887D
:1034E00022A106EB0040BDE8F04104F095BA0228A5
:1034F00014D30A220021A868FDF76FF807460A22B4
:1035000000216868FDF769F8024620883B4606EB13
:103510000040BDE8F0411CA104F085BABDE8F0818F
:103520007404002074657374207761726E696E672D
:10353000206D6573736167652077697468206D6FAE
:103540007265207468616E203320617267756D65E5
:103550006E74730074657374207761726E696E6740
:10356000206D657373616765000000007465737496
:10357000207761726E696E67206D65737361676530
:103580003A2025640000000074657374207761722E
:103590006E696E67206D6573736167653A20256497
:1035A0002025640010B5044603F036F830B12046FB
:1035B0000022BDE81040114602F0BEBE054A0721B8
:1035C000204602F05BFE2046BDE8104002A2082122
:1035D00002F054BE8CB600002020202020202020A5
:1035E00020202020202020204E6F72646963205309
:1035F000656D69636F6E647563746F72202020203F
:10360000202020202020202020200D0A0D0A00004C
:10361000F8B515460E46040003D117A12520FEF784
:1036200023F8A06818B1606808B1206818B912A121
:103630002620FEF719F8012E03D0204602F0ECFFF9
:1036400030B12046BDE8F8400022114602F074BEB9
:10365000022E08D02B6801B02046BDE8F0400DA234
:10366000022102F00BBE6868009011A202212046E0
:103670002B6802F003FEF8BD2E2E5C2E2E5C2E2E43
:103680005C64656D6F5F636C695F636D64732E630B
:103690000000000025733A2062616420706172614D
:1036A0006D6574657220636F756E740D0A0000009D
:1036B00025733A20756E6B6E6F776E207061726144
:1036C0006D657465723A2025730D0A002DE9F0418D
:1036D00016460D460746012408E000BF56F8243080
:1036E00007A20821384602F0C9FD641CAC42F5D39C
:1036F0003846BDE8F04103A2082102F0BFBD00003A
:10370000257320000D0A0000F8B516460D46074641
:10371000012409E056F824000090234604A2082161
:10372000384602F0ABFD641CAC42F3D3F8BD000098
:10373000617267765B25645D203D2025730D0A006C
:1037400001A2022102F09ABD4E696365206A6F6B87
:1037500065203B290D0A000010B5044602F062FF07
:1037600030B120460022BDE81040114602F0E4BD11
:10377000BFF34F8F05480168054A01F4E06111432A
:103780000160BFF34F8F00BFFDE700000CED00E0CC
:103790000400FA052DE9F04185680646002495F8F5
:1037A0002000002811D0A046FCF744FE0746006820
:1037B00004F1200104F10104695CA4B2415CC90771
:1037C00005D0002CF4D185F82080BDE8F081641E7E
:1037D0002404240C0FD0688B021B04F1200029184C
:1037E00005F12000521CFCF77DFEB168488B001BE0
:1037F0004883B1688883B2683D68538BD0181F3006
:103800000446002102E0491C89B2401E0778EF5DA2
:10381000FF07F8D18442D8D05B1A203302F8038026
:10382000B268508B401A5083B1688883CDE700009E
:103830002DE9F0410746154688460846FEF72AFE60
:1038400084B2B868661CC18B3144B1F5C07F07D91A
:10385000124A0421384602F011FD0020BDE8F08133
:10386000294600F5D070FCF76FFE051EF6D0FEF776
:1038700011FE82B228192946401C521CFCF732FE68
:10388000224641462846FCF72DFE20202855B868E0
:10389000C18B3144C1830120E0E70000C8C50000AE
:1038A0002DE9FF4F002787B09A46DDF850B0064655
:1038B0003C46B84602250DF108090197DDE90801EB
:1038C0003A467F1C01ABCDF80090FFF7D5FC01987C
:1038D00088B101680022504600F0D4FD48B9019833
:1038E000524601683046FFF7A3FF5FEA000802D0A6
:1038F000641C002FE2D15CB3CBF80040B0685546A1
:10390000514600F5D070FCF71FFE04462846FEF72E
:10391000C1FD85B2C4B1B06800F5D070A04206D236
:1039200014F8010C202802D16D1CADB2641E204693
:10393000FEF7B0FD421BB068521CC18B491BC1830E
:1039400061192046FCF7CEFDB8F1000F01D000252B
:1039500000E001250BB02846BDE8F08F40684968BB
:10396000884201D801207047002070472DE9F041BE
:1039700015460F00044604D123A140F28650FDF7FE
:1039800073FEA068418B828B8B1A29449EB2B1F5DD
:10399000C07F37D2002D35D0104400F1200105F151
:1039A00020021044721CFCF79DFDA0682A46818B02
:1039B000084439462030FCF795FDA0682030FEF71A
:1039C00069FDA1681EA24883A068818B4318082165
:1039D0002046203302F052FCA068818B2944818369
:1039E000204600F08EF818B9204600F0BFFE10B156
:1039F000204600F0A5F8002E04D02046BDE8F04196
:103A000000F06EB9BDE8F0812E2E5C2E2E5C2E2EBD
:103A10005C2E2E5C2E2E5C2E2E5C636F6D706F6E96
:103A2000656E74735C6C69627261726965735C6304
:103A30006C695C6E72665F636C692E6300000000E7
:103A400025730000002904D00A46006901A103F093
:103A500067B870471B5B25644200000070B50546DF
:103A600001F007FE044600886188884203D1A088DF
:103A7000E18888421AD0E188A088814204D9081AD6
:103A800081B22846FFF7DEFF20886188884205D989
:103A9000401A81B2284600F047F804E0081A81B2C3
:103AA000284600F053F9A868418B818370BD70B53A
:103AB000054601F0DEFD04460188007B401C814282
:103AC00002D1A08801281BD0A088012804D9401E5B
:103AD00081B2284600F046F92088217B884206D929
:103AE000401A401E81B2284600F01EF805E0081A70
:103AF000401C81B2284600F029F9A968002088837B
:103B000070BD10B504460068FEF7C4FC0146A0680D
:103B1000828B408A1144B1FBF0F200FB121008B115
:103B2000002010BD012010BD002904D00A46006904
:103B300001A102F0F5BF70471B5B25644400000043
:103B400070B504004FF4BB7503D108A12846FDF7FA
:103B50008BFD206918B905A12846FDF785FD206970
:103B6000BDE870400F4A10A102F0DABF2E2E5C2E85
:103B70002E5C2E2E5C2E2E5C2E2E5C2E2E5C636F09
:103B80006D706F6E656E74735C6C69627261726980
:103B900065735C636C695C6E72665F636C692E63EF
:103BA00000000000B6AF0000257300002DE9FC47BF
:103BB000002604468DF8046080684FF4C07A3546CC
:103BC000B146B046514600F5D070FCF7B2FC43490F
:103BD000206902F0A5FF206902F0E2FF00276B4692
:103BE000012201A92046FEF739FA0098D8B19DF8C4
:103BF00004001B2806D0A16891F8A0111B29EED162
:103C000052281FD0A26808F5D071505408F1010065
:103C10001FFA80F8B8F1090F0AD9A168042081F8C9
:103C2000A091BDE8FC872D494FF6C0100D318847A3
:103C300000980028D3D17F1CBFB2B7F57A7FCED3CE
:103C40000D20EEE7A16808F5D0704A4601F8009013
:103C5000A16891F8A1015B2803D081F8A0210B2075
:103C6000DFE7022057466FF02F0309E005EB8505DB
:103C700003EB4505401C654480B2ADB2B8420AD2A0
:103C800000F5D07C11F80CC0BCF13B0FEED1401C0C
:103C900080B2B84209D30C20C3E700BF06EB86060A
:103CA00003EB46066644B6B2F1E700F5D07C11F8A6
:103CB0000CC0BCF1000FF1D1FA20FA2E01D9088115
:103CC00000E00E81FA2D02D9A168888101E0A06888
:103CD0008581A06880F8A0210020A2E7D4AF000071
:103CE00070B5054601F0C5FC04468088E18888422D
:103CF00001D1012600E000262846FFF702FF18B98F
:103D0000284600F033FD10B12846FFF719FF1EB119
:103D100060882188401A12E0E088A188401A81B2A8
:103D2000284600F01FF820886188884206D9401A8A
:103D300081B22846BDE8704000F008B8081A81B288
:103D40002846BDE87040FFF7EFBE0000002904D010
:103D50000A46006901A102F0E3BE70471B5B2564BF
:103D600043000000002904D00A46006901A102F0C6
:103D7000D7BE70471B5B25644100000010B50021D1
:103D8000024801F0FFFC80F3100010BD681900200C
:103D90004FF4A07202EB810189B200F06FBA0068A3
:103DA000D0F80405704700002DE9F04715460E468F
:103DB000040003D138492F20FDF756FC1EB93649BF
:103DC0003020FDF751FC1DB933493120FDF74CFC83
:103DD00060793249DFF8C480DFF8C49041F82050A0
:103DE000617908F1040808EBC100007958B1D9F8ED
:103DF0000400082402284CD3B9F80000022101EB8A
:103E0000004028A143E035882768B5F5805F03D3DB
:103E10002DA1FD20FDF728FCC7F80855B67894F9C8
:103E20000450082E03D334A14520FDF71DFC002DBE
:103E30004FEA461006DA05F00F0101F1E02181F8A2
:103E4000140D03E005F1E02585F8000494F9041051
:103E5000012201F01F0302FA03F04909890001F170
:103E6000E021C1F88002C1F80001617908EBC101CD
:103E70000A71617948F83140D9F804000024032818
:103E800007D3B9F80000032101EB004026A103F09D
:103E9000BFFD2046BDE8F087E4BC00008C01002097
:103EA000FC03002052544320696E7374616E636595
:103EB00020616C726561647920696E697469616CF6
:103EC000697A65642E0000002E2E5C2E2E5C2E2E4C
:103ED0005C2E2E5C2E2E5C2E2E5C6D6F64756C65D8
:103EE000735C6E7266785C68616C2F6E72665F726E
:103EF00074632E68000000002E2E5C2E2E5C2E2E89
:103F00005C2E2E5C2E2E5C2E2E5C696E74656772A4
:103F10006174696F6E5C6E7266785C6E7266785FF3
:103F2000676C75652E6800005254433A20696E69CB
:103F30007469616C697A65642E00000090F9040070
:103F4000012100F01F0291404009800000F1E020B3
:103F5000C0F8001270470A46022100F07BB94FF406
:103F6000827100F08BB9000010B5040003D1044940
:103F70006120FDF779FB20680121016010BD000080
:103F8000E4BC000010B5040003D104496720FDF72C
:103F90006BFB20680121416010BD0000E4BC000003
:103FA0002DE9F843994616460F46050003D12E49E0
:103FB0008620FDF759FB29684FF480344FF4A07038
:103FC000BC4000EB870080B226F07F46C1F8084372
:103FD0002968C1F84843296800220A50085800900F
:103FE000286800EB8701D1F84005C1F840652968D1
:103FF000D1F804151D4F401A20F07F404FF00408FF
:1040000001280CD17868042805D3398808EB0140D1
:1040100017A103F0FDFC23494FF40460884728688A
:10402000C0F844432968D1F80435F01A20F07F40E5
:10403000020201D540F07F40C9F1000290420EDD3E
:1040400002280CDC7868042806D33988324608EB4D
:10405000014015A103F0E7FC0D20BDE8F883C1F88D
:1040600004430020F9E70000E4BC0000FC0300204A
:104070005254433A2044656C617920696E74726FC2
:1040800064756365642064756520746F207269735C
:104090006B206F66207072652D666972696E672E7F
:1040A0000000000001AE00005254433A2057696EF0
:1040B000646F77656420636F6D70617265207365EE
:1040C000742074696D656F757420286162735F7602
:1040D000616C75653A25642C20636F756E7465722A
:1040E0003A2564292E00000070B50C00054604D165
:1040F0000AA140F27510FDF7B7FA0F484178002089
:104100008D4209D20D4AE06005EB4511A0601144D3
:104110000BA0C4E9001070BD206070BD2E2E5C2E77
:104120002E5C2E2E5C64656D6F5F636C695F636DE2
:1041300064732E6300000000000000208004002053
:1041400053686F772064796E616D696320636F6D6A
:104150006D616E64206E616D652E00001FB51446A2
:104160001A4AD06100200190029003908868019063
:104170008888ADF80800086800F00302012A07D01B
:10418000022A15D0124940F27720FDF76DFA1FBDC3
:10419000C0F3C2008DF80C000C4801AB2030009039
:1041A00008682146C0F38312800A03F081FD1FBD19
:1041B000C0F3C2008DF80C000868044B810D203359
:1041C00001AA204603F058FC1FBD00000C0200208D
:1041D000E8CB00002DE9FC4180461F4615460E46FF
:1041E00000240D4801F0B5FA38B11120BDE8FC817A
:1041F00006EB043004F0B0F8641CAC42F8D1064879
:1042000001F09EFACDE900573346002202214046D4
:1042100000F004F80020E9E7080200202DE9F0434F
:1042200087B00446DDE90E8980681D4616460F46B4
:1042300000280BD018216846FCF77BF902A88DF8FE
:10424000007080E86003A1686846884707B0BDE851
:10425000F083000070B516460C46050003D10649F0
:10426000B920FDF701FA2868C0F84443002E02D0B7
:104270002868C0F8044370BDE4BC000038B50C46A3
:10428000050003D10749CA20FDF7EEF92868015956
:1042900029B10021015100590090012038BD0020B2
:1042A00038BD0000E4BC000010B58168D1F84813A7
:1042B000C1F3400119B10022114602F03DF8BDE8FA
:1042C000104003F0CFB9000010B5134803F0E0F937
:1042D00018B1124AFD21FBF79DFF0221104803F09F
:1042E000DFF8012414EBE07003D10C4A2102FBF744
:1042F00091FF0B48032144720C3003F0D1F814EB0A
:10430000E07004D1054A40F20711FBF783FF04482F
:104310000C30447210BD0000A8B00000A452000090
:10432000080000203EB505468068D0F84803C0F379
:10433000400020B100221146284601F0FDFF002078
:104340000290012400906A4601A902A803F0C6F970
:1043500038B1002C04D006A20221284601F08EFFBD
:104360003EBDDDE900212846FFF7F8FE0024EAE71C
:10437000466C617368206C6F6720656D7074790D91
:104380000A0000007CB505468068D0F84803C0F3F9
:10439000400020B100221146284601F0CDFF14A2B2
:1043A0000821284601F06AFF164C4FF48056230B73
:1043B0001B0315A208212846009601F05FFF200B81
:1043C0001D4C40421DA2216901EB0031CDE90016D0
:1043D000642041430B0B0821284601F04FFFA369DD
:1043E00002B02846BDE8704020A2082101F046BF77
:1043F000466C617368206C6F6720737461747573A9
:104400003A0D0A00AFE4000009092D204C6F6361EA
:1044100074696F6E2028616464726573733A20302A
:1044200078253038582C206C656E6774683A2025E2
:1044300064290D0A000000000C02002009092D204B
:1044400043757272656E742075736167653A256491
:10445000252520282564206F662025642062797434
:1044600065732075736564290D0A000009092D2004
:1044700044726F70706564206C6F67733A202564B6
:104480000D0A00004023AFF300802DE9F0471646E7
:104490000C4605005BD0ACB3B3F1010902D2032096
:1044A000BDE8F087884615F8010B314600F0A3F807
:1044B000C7B23F2F11D003DC3FB12A2F7DD122E0BC
:1044C0005B2F69D05C2F78D182E0F00602D520788E
:1044D0002F283ED02078A8B9E2E7207890B12F2885
:1044E00002D02E2803D06DE0B00730D46AE0700708
:1044F00068D544452BD0B00764D514F8010C2F289B
:1045000025D05FE023E0287801E015F8010F31465F
:1045100000F071F8C0B22A28F7D021782E2909D1ED
:10452000710707D5444512D0B10703D514F8011C13
:104530002F290CD010B12F280DD023E0B00708D5BB
:10454000F00606D42F212046FCF710F808B1012010
:10455000A6E70020A4E7B00714D52F212046FCF7DA
:1045600005F804009FD1F2E74B4642462146284613
:10457000FFF78BFF012893D12F2F01D1B007E6D48D
:10458000641C01E026F004082078314600F033F87E
:1045900010F0FF07E8D1DAE720780028D7D02F28DD
:1045A00001D1B107D3D4314600F025F80146324697
:1045B000284605F035FB002800E014E0C7D0411C78
:1045C00002D00546641C6EE720785B28BFD1F9E76E
:1045D000F00708D115F8010B314600F00CF810F087
:1045E000FF0700D16D1E14F8010B314600F003F8EF
:1045F000B842E8D0ABE710B5044608070AD5FBF788
:1046000019FF0068005DC00604D52046BDE81040D3
:10461000FBF714BF204610BD2DE9F05F17460E00D2
:10462000814670D013B1B9B2FFF790FB0024FBF7BD
:1046300001FF8246006800E0641C315D415CC907EF
:10464000FAD100253046FDF725FFD9F80810001BE8
:104650004A8AD11B814228D306EB040805E000BF3B
:1046600018F805100A290CD06D1C8542F8D33119B1
:10467000D9F8100002F054FA4846BDE8F05FFFF7A1
:104680005FBAD9F8100002F08BFA414600232A469F
:104690004846FEF7CBF92C444846641CFFF750FA15
:1046A000B9B24846FFF752FBE1E78B46DAF8001053
:1046B00006EB040818F805000B5CDB0702D0AB46DC
:1046C0000A2804D0E819904201D26D1CF2E7D9F80B
:1046D000100002F065FA414600235A464846FEF7AC
:1046E000A5F95C44DAF8000000E0641C315D415C2F
:1046F000C907FAD14846FFF723FAB9B24846FFF78F
:1047000025FB9EE7FFE7BDE8F09F000010B50446DB
:1047100014480021027862B1012A09D12278022AC4
:1047200006D1114AA3686FF30B02934200D10170C6
:1047300010BD2278012AFBD162684AB18169491C07
:10474000816160690028F3D0BDE8104003F06BBBC5
:10475000D0E904231A44C0E904210021406800F094
:10476000E7FBEEE70C020020AFE4000010B50446C2
:104770000068FDF78FFE0146A068428B408A114415
:10478000B1FBF0F200FB121008B1002010BD0120B7
:1047900010BD0000FEB50026044600960196029664
:1047A0008068E9B3D0E9D0128A4273D0D0F83C03D4
:1047B00000286FD02046FFF77AF9A068D0F844535C
:1047C000002D6AD000230A226946284603F03AFBEE
:1047D000A168BDF808500098C1F84403A068002300
:1047E0000A22D0F84403694603F02CFBA168BDF807
:1047F00008200A23D1F844032031521C03F022FB85
:10480000A168BDF808008883A168BDF80800488346
:10481000BDF80800A84202D22046FDF709F900E0E1
:104820000BE0A3682CA208212046203301F026FDCE
:104830002046FFF766F970BB45E0D0F84403002836
:1048400049D02046FFF733F9A06800230A22D0F8A8
:104850004403694603F0F6FAA0680199C0F84413CE
:10486000A0680029458BB9D100F5D070FDF712FE84
:104870000028A06805D000F5D0712030FBF795FE28
:1048800001E080F82060A0682030FDF703FEADF85D
:104890000800B5E71FE01BE0FFE72030FDF7FAFD59
:1048A0000504A0682D0CD0F83C13C0F84413A06890
:1048B00006D000F1200100F5D070FBF776FE8DE701
:1048C00080F8A0618AE72046FFF750FF002802D059
:1048D0002046FFF735F9FEBD25730000FEB50D003B
:1048E000044604D11E4940F2DD40FCF7BDFEA1683C
:1048F0000026D1F83C0338B300230A22694603F0AE
:10490000A1FA0195A06800230A22D0F83C03694669
:1049100003F09EFA0196A068D0F83C130091408BFA
:10492000ADF80800A068C0F83C5300230A2269468D
:10493000284603F08DFAA1680A2328464A8B2031C5
:10494000521C03F085FAFEBDC1F83C53A068C0F8C4
:10495000405300960196A068408BADF80800E4E74C
:10496000FCA10000FEB504468068D0F84063002E2C
:1049700028D000230A226946304603F063FAA16872
:1049800001980025C1F84003009501952B460A22A5
:1049900069463046029503F05BFA304603F024FA8C
:1049A000A168D1F8400370B100230A22694603F0E0
:1049B00049FA0095A06800230A22D0F8400369460E
:1049C00003F046FAFEBDC1F83C53FEBDFEB50446F9
:1049D00080682030FDF75EFD0504A0684FF00006FA
:1049E0002D0CC0F8446333D0A068D0F83C03E0B18C
:1049F00000230A22694603F025FABDF80820AA42DE
:104A000013D1A0680A2300F5D071D0F83C03521CE2
:104A100003F018FAA06800F5D0712030FBF7B7FD5D
:104A20000028A06880F8A06112D000260B35294626
:104A3000606903F0A9F90100204604D003B0BDE885
:104A4000F040FFF74BBFFFF78DFF761C082EEED32B
:104A5000FEBD000001494160002070479CB000008D
:104A60002DE9FC5F0E008346DDE90C47C6F100002E
:104A700098469246814600D40846012503E000BFCF
:104A800090FBFAF06D1C5045FADAA84500D945466E
:104A900024B1002E01DB780700D5641EB80702D5CB
:104AA000B8F1000F0AD0F80708D13CB1A54205D2F1
:104AB00020215846641EFCF727FEF6E7002E02DA96
:104AC0004E462D2102E0780703D52B215846FCF7EE
:104AD0001BFE07F0030002280BD1B8F1000F08D12C
:104AE0003CB1A54205D230215846641EFCF70CFEAD
:104AF000F6E7CDE90047434652463146584605F0B1
:104B00003BFFBDE8FC9F000070B50E4605460068FF
:104B10004FF48E7104F039F94FF4A271286804F053
:104B200034F928681549C0F804132868000B44B20A
:104B3000082E03D312A14520FCF796FD7007000E46
:104B4000002C06DA04F00F0101F1E02181F8140DC8
:104B500003E004F1E02484F8000428680121000B3C
:104B600040B200F01F0291404009800000F1E020B7
:104B7000C0F88012C0F8001170BD00008000020073
:104B80002E2E5C2E2E5C2E2E5C2E2E5C2E2E5C2E5F
:104B90002E5C696E746567726174696F6E5C6E72AB
:104BA00066785C6E7266785F676C75652E6800006B
:104BB00070B50E46044600684FF4887104F0F6F8AC
:104BC0004FF49071206804F0F1F84FF4927120686E
:104BD00004F0ECF84FF4A271206804F0E7F82068C4
:104BE0001549C0F804132068000B45B2082E03D302
:104BF00012A14520FCF738FD7007000E002D06DAE3
:104C000005F00F0101F1E02181F8140D03E005F139
:104C1000E02585F8000420680121000B40B200F077
:104C20001F0291404009800000F1E020C0F880128E
:104C3000C0F8001170BD0000100302002E2E5C2E83
:104C40002E5C2E2E5C2E2E5C2E2E5C2E2E5C696E23
:104C5000746567726174696F6E5C6E7266785C6EA3
:104C60007266785F676C75652E68000010B5024645
:104C700000201268930702D0530702D410BD5007DA
:104C800019D502F00300012807D002280BD00D49E6
:104C90004FF49170FCF7E8FC0BE0C2F383100B6853
:104CA000C01C184404E00323086803EB925210442C
:104CB0000860012010BD086800EB9253C2F3891010
:104CC000401CEEE73CCC000002480068002800D001
:104CD00001207047080200200268134602E08A4261
:104CE00004D01268002AFAD10B60016070470000FE
:104CF0001CB5012905D08168D1F84813C1F34001E2
:104D000031B102B00022BDE81040114601F014BBE1
:104D1000536804A1CDE90013136808A2022101F031
:104D2000ADFA1CBD20756E6B6E6F776E2070617270
:104D3000616D657465723A200000000025733A25A4
:104D40007325730D0A0000002DE9F74F82B0154658
:104D500002980F004FF00006C068007A009058D00B
:104D6000072248A12868FBF729FC78B1082247A14F
:104D70002868FBF723FC002830D02B6845A2029856
:104D800005B00221BDE8F04F01F078BA012F02D042
:104D9000022F08D008E0029805B044A2BDE8F04F09
:104DA000022101F06BBA0126DFF81881002400BF50
:104DB00058F824100A226868FBF700FC10B1641C44
:104DC000052CF5D3052C06D004F0FF090224002E93
:104DD00054D0002419E03CA26B68D0E7012F4FF0BB
:104DE0000009F6D0012449E04A462146009800F027
:104DF000CAFB48B90021204602F038FF03463AA218
:104E00000221029801F03AFA641C02F0DDFEA04291
:104E1000EAD805B0BDE8F08F4FF0000A55F824B08D
:104E200002F0D2FE8046002609E00021304602F062
:104E30001DFF20225946FBF7C1FB90B1761C464569
:104E4000F3D3464506D155F8243030A2022102980A
:104E500001F014FA4A465146009800F094FB10B154
:104E60000BE0B246EDE70021504602F0FFFE03469C
:104E70001DA20221029801F001FA641CBC42CBD3AE
:104E8000C7E70000656E61626C650000646973616C
:104E9000626C6500556E6B6E6F776E206F70746913
:104EA0006F6E3A2025730D0A0000000042616420F5
:104EB000706172616D6574657220636F756E742EBA
:104EC0000D0A000044020020556E6B6E6F776E2055
:104ED0007365766572697479206C6576656C3A20C5
:104EE00025730D0A000000004C6576656C20756E18
:104EF000617661696C61626C6520666F72206D6FAE
:104F000064756C653A2025730D0A0000556E6B6E52
:104F10006F776E206D6F64756C653A25730D0A00AE
:104F2000C068012141727047C0680021417270471A
:104F30007CB50D460646214C26E040201F4A6061A4
:104F400014321F49019800F059FBE8B10198009014
:104F5000D4E904131A4A1B4802F062F808B155B1AB
:104F60000BE0002D1BD0D4E9040108442061019816
:104F700002F059FF08E0042812D0102817D0124977
:104F800040F21710FCF770FB002201A9304603F035
:104F900029FA0028D1D009480C3000F0D1FB7CBDA3
:104FA000019802F040FFA069401CA061F3E701985E
:104FB00002F039FF01202070E6E700000C0200201B
:104FC0003C13002004030020E8CB00002DE9FF4142
:104FD0000026264800F0BAFB2448001F074600F0D0
:104FE000B5FB234C60680090A56800E00098694616
:104FF000284004EB80000C30FFF738FE0028F5D184
:1050000001AA009901EA050304EB8303491CDB684C
:1050100042F82030401C00910328F2D3019800F0A0
:10502000030001281AD002280ED012494FF4AF70A5
:10503000FCF71AFB384600F086FB08B10098606068
:1050400004B03046BDE8F0810198032101EB905097
:105050000099BDF80A6001EB900005E00198BDF8E9
:105060000A60C0F3831008440090E3E7641900204D
:105070004C1500203CCC00002DE9FE4F814602F08B
:10508000A3FD0746D9F80C0090F80880407A20B9B3
:105090001FA20221484601F0F1F822A324A2082110
:1050A000484601F0EBF82AA20821484601F0E6F84C
:1050B000002429E001231A462146404602F08EFDD5
:1050C0008246002301222146404602F087FD054624
:1050D000042801D2064600E004260121204602F001
:1050E000C5FD0346AE4201D229A200E027A229480D
:1050F00050F8261050F82A008DE8070026A2082153
:10510000484601F0BBF8641CBC42D3D3BDE8FE8F17
:105110004C6F6773206172652068616C74656421EF
:105120000D0A00006D6F64756C655F6E616D6500E2
:10513000252D343073207C2063757272656E742067
:105140007C206275696C742D696E200D0A00000068
:105150002D2D2D2D2D2D2D2D2D2D2D2D2D2D2D2D7F
:105160002D2D2D2D2D2D2D2D2D2D2D2D2D2D2D2D6F
:105170002D2D2D2D2D2D2D2D2D2D2D2D2D2D2D2D5F
:105180002D2D2D2D2D2D2D2D2D2D0D0A0000000046
:105190002A00000044020020252D343073207C209A
:1051A000252D3773207C20257325730D0A00000000
:1051B0004FF400442146344802F0B4FC20B133A23D
:1051C00040F22111FBF726F801F0F0FB20B12FA2ED
:1051D0004FF49371FBF71EF8002001F001FCFCF77F
:1051E00003F920B129A24FF49571FBF713F82B4A6C
:1051F00001212B48FCF7DAF820B124A240F22D114E
:10520000FBF708F82648002221460068FCF712F94F
:1052100020B11EA24FF49871FAF7FCFFFCF73AFE9A
:105220001F48001D01F062FB18B11EA2A821FAF769
:10523000F1FF1B48203001F059FB18B119A2AC2135
:10524000FAF7E8FFFFF740F81A4C606803280FD31D
:105250002088052505EB004017A102F0D9FB606806
:10526000032805D320881FA105EB004002F0D0FBE6
:1052700002F0A4FA0A48001D01F0D2FA08482030D2
:1052800001F0CEFAF4E70000A11300002E2E5C2EF0
:105290002E5C2E2E5C6D61696E2E630089A200006B
:1052A00060AC00002E2E5C2E2E5C2E2E5C6D616993
:1052B0006E2E630074040020436F6D6D616E642078
:1052C0004C696E6520496E74657266616365206520
:1052D00078616D706C6520737461727465642E0DF5
:1052E0000A000000506C656173652070726573730D
:1052F0002074686520546162206B657920746F208A
:1053000073656520616C6C20617661696C61626CAB
:105310006520636F6D6D616E64732E0D0A00000071
:105320002DE9FF4F4FF0000881B014468B468146AF
:10533000C246C0F800802578002D71D0FBF77AF8BE
:1053400000900068405DC00702D004F801AB84E023
:10535000D9F800008300401CC9F800004BF8034056
:1053600015E02678002E78D0B8F1000F05D1222E56
:1053700010D0272E0ED05C2E1ED0B04514D1204662
:10538000FDF788F80246611C2046FBF7ABF84FF0AA
:105390000008E6E72046FDF77DF80246611C20463E
:1053A000FBF7A0F8B046DCE7B8F1000F50D05C2E58
:1053B0006AD16078404508D12046FDF76BF8024677
:1053C000611C2046FBF78EF85EE030281CD10027D8
:1053D0000225605DA0F13001072906D86D1C41EA65
:1053E000C701EDB2CFB2052DF3D3022D0CD9204663
:1053F000FDF750F8421B61192046491E921CFBF72D
:1054000071F804F8017BACE778281ED1002702254B
:10541000605DA0F13001092903D841EA07100DE0D1
:1054200021E0A0F16101052901D8573804E0A0F17D
:105430004101052907D8373840EA07106D1CEDB245
:10544000C7B2042DE4D3022DD1D8B8F1000F1BD17F
:1054500000980068805DC00716D0D9F80010049845
:105460008142FFF468AFD9F800000C2804D907A1E5
:1054700040F25B40FCF7F8F8D9F8002040464BF8C2
:1054800022A005B0BDE8F08F641C6AE72E2E5C2ECA
:105490002E5C2E2E5C2E2E5C2E2E5C2E2E5C636FD0
:1054A0006D706F6E656E74735C6C69627261726947
:1054B00065735C636C695C6E72665F636C692E63B6
:1054C000000000002DE9F05FC7888A46191D1646C6
:1054D000B1FBF7F2B1FBF7F507FB12199919394443
:1054E000C91CB1FBF7F104464079C9B2DDF828B018
:1054F000884206D217499420FCF7B6F801E02468E8
:105500006D1E002DFBD1A846A7EB0905B5421AD8A0
:105510001CE000BFBBF1000F06D004EB09010AEB51
:1055200008002A46091D05E004EB09000AEB080102
:105530002A46001DFAF7D6FF2468761B4FF00009B3
:10554000A844B74201D9354600E03D46002EE1D1DE
:10555000BDE8F09F6CC6000033B581B0054600245D
:1055600009E000226946284602F03CFF18B900987D
:1055700002F059FC641C02A9284603F069F80028CF
:10558000EFD120463EBD70B5144600230D460646B9
:105590001A4602F023FB844201D9002070BD224646
:1055A0002946304602F040FB012070BD30B502466E
:1055B00069B102F009FB0021084C0BE001EB41034B
:1055C00004EB830315685B88AB4202D111600020B5
:1055D00030BD491C8142F1D3052030BD18030020A5
:1055E00010B50C460021E16061600349A160012112
:1055F00002F03CFB206010BDCCB200002DE9FE4360
:10560000002416460D460C2780460094019423463C
:105610003A466946029402F015FC009845F8040BDE
:10562000019845F8040B029845F8040B009800F027
:105630000300012803D0022806D0346017E0009848
:10564000C0F38310840004E00098800D04F08CFC0B
:1056500004463B4622462946404602F0F3FB3068AA
:105660000C34A04203D301203460BDE8FE83002047
:10567000FBE770B58468006804F10805FCF70AFFD1
:10568000C1B22973A08B6A890844B0FBF2F302FB14
:1056900013035B1C2B80A08B0844B0FBF2F35B1C54
:1056A000AB80608B0844B0FBF2F35B1CEB80608B3B
:1056B0000844B0FBF2F102FB1101491C6980284645
:1056C00070BD10B531B1B2FBF3F403FB14241CB16F
:1056D000092010BD0E2010BD0160002141608160D5
:1056E0008281C381084610BD70B50C460546FAF7A5
:1056F000B9FD002802D021882868084470BD10B583
:105700000A8849888A4203D1FAF7EEFD012010BDCC
:10571000002010BD70B50C460546FAF7C8FD0028FC
:1057200002D061882868084470BD10B50A8849888D
:105730008A4203D1FAF7B2FD012010BD002010BD4E
:10574000002100F00FB8002100F012B8012100F094
:105750001EB8012100F011B808B56A46FAF719FE23
:10576000009808BD08B56A46FAF7F9FD009808BD2B
:1057700008B56A46FAF7F3FD08BD08B56A46FAF7B8
:10578000E1FD08BD08B56A46FAF7D0FD08BD08B5C9
:105790006A46FAF7D7FD009808BD08B56A46FAF7D9
:1057A00005FE009808BD000070B5040003D113A1E8
:1057B000FE20FBF759FF00252846FBF771FE206805
:1057C00062680168914214D9491E01600D781CB9C4
:1057D00019A1C220FBF748FF208BE16805FB0015EB
:1057E0002068217A0278891A0279C9B28A4200D2E5
:1057F00001710020FBF782FE284670BD2E2E5C2E24
:105800002E5C2E2E5C2E2E5C2E2E5C2E2E5C636F5C
:105810006D706F6E656E74735C6C696272617269D3
:1058200065735C62616C6C6F635C6E72665F626113
:105830006C6C6F632E6300002E2E5C2E2E5C2E2E61
:105840005C2E2E5C2E2E5C2E2E5C636F6D706F6E48
:10585000656E74735C6C69627261726965735C62B7
:10586000616C6C6F635C6E72665F62616C6C6F63BF
:105870002E63000070B50C46050004D110A140F263
:105880002110FBF7F1FE24B90DA14FF49170FBF745
:10589000EBFE0020FBF704FE1DB91849CF20FBF7F3
:1058A000E3FEE8682A68211A288BB1FBF0F1106842
:1058B000431C13600170BDE870400020FBF71EBE62
:1058C0002E2E5C2E2E5C2E2E5C2E2E5C2E2E5C2E12
:1058D0002E5C636F6D706F6E656E74735C6C696265
:1058E0007261726965735C62616C6C6F635C6E722D
:1058F000665F62616C6C6F632E6300003858000055
:1059000010B5040002D0206830B901E00E2010BDAF
:1059100017A1D920FBF7A8FE606818B914A1DA20F6
:10592000FBF7A2FEA06818B911A1DB20FBF79CFED3
:10593000E06818B90EA1DC20FBF796FE208B18B9A1
:105940000BA1DD20FBF790FE207A61682268401AE7
:10595000C0B2116004E0226811684B1C136008702B
:10596000401EC0B2F7D221680020087110BD0000AF
:105970002E2E5C2E2E5C2E2E5C2E2E5C2E2E5C2E61
:105980002E5C636F6D706F6E656E74735C6C6962B4
:105990007261726965735C62616C6C6F635C6E727C
:1059A000665F62616C6C6F632E6300002DE9F04FDF
:1059B0008146806889B0D0F84803C0F3400038B110
:1059C00009B04846BDE8F04F0022114600F0B4BCD3
:1059D000012907D909B04846BDE8F04F24A20221A9
:1059E00000F04CBC27492848081A1C21B0FBF1F8EC
:1059F000002538E02448C5EBC50110EB81044FF0C9
:105A0000000AB4F818B0D4E90101A1EB000604D1F2
:105A10001EA140F21F10FBF727FE2068077924B96A
:105A20001AA140F22F10FBF71FFE2068217A0078A0
:105A3000081AC0B2642117FB01F1B1FBF6F2642130
:105A400010FB01F1B1FBF6F16369CDE90210CDE97C
:105A50000462CDE90676CDE900BA1B4A0821484622
:105A600000F00CFC6D1C4545C4D309B0BDE8F08FB7
:105A700042616420617267756D656E7420636F7535
:105A80006E74000034D30000E0D200002E2E5C2E95
:105A90002E5C2E2E5C2E2E5C2E2E5C2E2E5C636FCA
:105AA0006D706F6E656E74735C6C69627261726941
:105AB00065735C62616C6C6F635C6E72665F626181
:105AC0006C6C6F632E68000094C20000C20800F086
:105AD00007030120895C98400840704710B5C20850
:105AE00000F00703885C01249C402043885410BDCB
:105AF00070B515468268D2F84843C4F3400424B117
:105B00001A46294600F018FC06E039B1516804A293
:105B10000B68022100F0B2FB012070BD002070BDB7
:105B200025733A2077726F6E6720706172616D65C0
:105B300074657220636F756E740D0A0070B50D4642
:105B4000040004D122A140F65640FBF78DFDA06869
:105B500018B1606808B1206820B91DA140F657400F
:105B6000FBF782FD022D0CD1A068D0F84803C0F3EA
:105B7000400030B12046BDE870400022114600F0E0
:105B8000DBBB40F65F451CB911A12846FBF76CFD55
:105B9000206918B90EA12846FBF766FD1A4A1BA119
:105BA000206900F0BDFF4FF446651CB908A12846E6
:105BB000FBF75AFD206918B905A12846FBF754FDEB
:105BC0002069BDE87040104A10A1093200F0A8BF5A
:105BD0002E2E5C2E2E5C2E2E5C2E2E5C2E2E5C2EFF
:105BE0002E5C636F6D706F6E656E74735C6C696252
:105BF0007261726965735C636C695C6E72665F6327
:105C00006C692E6300000000D0AF00002573000017
:105C100070B50D46040004D113A140F66540FBF7B2
:105C200023FDA06818B1606808B1206820B90EA1F2
:105C300040F66640FBF718FD012D07D0022D0CD170
:105C4000A068D0F84803C0F3400030B12046BDE85A
:105C500070400022114600F06FBB2046BDE8704046
:105C60000FA2022100F00ABB2E2E5C2E2E5C2E2EDF
:105C70005C2E2E5C2E2E5C2E2E5C636F6D706F6E14
:105C8000656E74735C6C69627261726965735C6382
:105C90006C695C6E72665F636C692E630000000065
:105CA000506C656173652073706563696679206106
:105CB00020737562636F6D6D616E642E0D0A000056
:105CC0001CB5012905D002290BD014D94FF00101D0
:105CD00012E002B04FF00002BDE81040114600F0A3
:105CE0002BBB536808A1CDE9001313680CA2022155
:105CF00000F0C4FA1CBD002102B00023BDE8104032
:105D00001A46FFF7F5BE000020756E6B6E6F776E5A
:105D100020706172616D657465723A200000000048
:105D200025733A257325730D0A00000010B504464B
:105D3000012901D0012100E0002100231A46FFF7CC
:105D4000D7FE002808D1A168C1F83803E068C06810
:105D5000BDE8104002F040BC10BD00003EB5044656
:105D6000012901D0012100E0002100231A46FFF79C
:105D7000BFFE002818D1E068C06802F003FCC0B282
:105D8000642110FB01F2E168C9688968B2FBF1F295
:105D9000D2B20092CDE90101A06804A20821D0F896
:105DA0003833204600F06AFA3EBD00004C6F737431
:105DB000206C6F67733A2025750D0A4D6178206C51
:105DC0006F67207175657565207574696C697A6196
:105DD00074696F6E3A2025752525205B25752F2562
:105DE000755D0D0A000000007CB515460E460400E6
:105DF00004D118A140F68640FBF736FCA06818B124
:105E0000606808B1206820B912A140F68740FBF70E
:105E10002BFC012E03D0022E09D0012108E002B094
:105E20002046BDE870400022114600F085BA0021EE
:105E300000231A462046FFF75BFE002809D1696857
:105E400012A0CDE9000117A2022120462B6800F024
:105E500015FA7CBD2E2E5C2E2E5C2E2E5C2E2E5C1A
:105E60002E2E5C2E2E5C636F6D706F6E656E74737C
:105E70005C6C69627261726965735C636C695C6EAB
:105E800072665F636C692E630000000020756E6BA4
:105E90006E6F776E20706172616D657465723A2005
:105EA0000000000025733A257325730D0A000000D9
:105EB00010B50446012901D0012100E00021002392
:105EC0001A46FFF715FE002806D1A068D0F848133F
:105ED00021F00401C0F8481310BD10B50446012993
:105EE00001D0012100E0002100231A46FFF700FE47
:105EF000002806D1A068D0F8481341F00401C0F88A
:105F0000481310BD7CB514460D460646022901D93A
:105F1000012100E0002100231A46FFF7E9FD0028D7
:105F200011D1022D05D03046FBF7AEFF60B10BA3B7
:105F30000BE061680AA0CDE900010FA20221304602
:105F4000236800F09BF97CBD0EA302B03046BDE88B
:105F500070400DA2082100F091B900006F6E0000A2
:105F600020756E6B6E6F776E20706172616D6574F7
:105F700065723A200000000025733A257325730DE1
:105F80000A0000006F6666004563686F20737461E5
:105F90007475733A2025730D0A00000010B504468D
:105FA000012901D0012100E0002100231A46FFF75A
:105FB0009FFD002806D1A068D0F8481321F0080101
:105FC000C0F8481310BD10B50446012901D00121C5
:105FD00000E0002100231A46FFF78AFD002806D1C1
:105FE000A068D0F8481341F00801C0F8481310BD6C
:105FF0007FB50D46040004D123A140F6CC40FBF749
:1060000033FBA06818B1606808B1206820B91EA1F0
:1060100040F6CD40FBF728FB012D01D0012100E027
:10602000002100231A462046FFF762FD002829D1EF
:10603000A0680026D0F8405305B301E0082E1DD219
:1060400000230A2201A9284601F0FCFEBDF80C201D
:10605000A1680A23284601F5D071521C01F0F2FE16
:10606000A068334600F5D0700090029D761C14A203
:106070000821204600F002F9002DDFD1A1680020A0
:1060800081F8A0017FBD00002E2E5C2E2E5C2E2EEE
:106090005C2E2E5C2E2E5C2E2E5C636F6D706F6EF0
:1060A000656E74735C6C69627261726965735C635E
:1060B0006C695C6E72665F636C692E630000000041
:1060C0005B2533645D2025730D0A00007CB5154601
:1060D0000E46040004D120A140F63250FBF7C4FA6A
:1060E000A06818B1606808B1206820B91AA140F60C
:1060F0003350FBF7B9FA012E03D0022E18D9012133
:1061000017E0A168204601F11002123104F038F8BE
:1061100000281FD0A16850201DA24882A168182025
:10612000088202B02046BDE87040042100F0A6B805
:10613000002100231A462046FFF7DAFC002809D187
:10614000696822A0CDE9000126A2022120462B6821
:1061500000F094F87CBD00002E2E5C2E2E5C2E2EBE
:106160005C2E2E5C2E2E5C2E2E5C636F6D706F6E1F
:10617000656E74735C6C69627261726965735C638D
:106180006C695C6E72665F636C692E630000000070
:106190004E6F20726573706F6E73652066726F6DDF
:1061A00020746865207465726D696E616C2C206165
:1061B0007373756D65642038307832342073637280
:1061C00065656E2073697A650D0A000020756E6B37
:1061D0006E6F776E20706172616D657465723A20C2
:1061E0000000000025733A257325730D0A00000096
:1061F00070B50446012901D0012100E000210023EF
:106200001A46FFF775FC002817D140F62B551CB92C
:106210000AA12846FBF728FA206918B907A12846E1
:10622000FBF722FA134A14A1206900F079FCA16857
:1062300050204882A1681820088270BD2E2E5C2E46
:106240002E5C2E2E5C2E2E5C2E2E5C2E2E5C636F12
:106250006D706F6E656E74735C6C69627261726989
:1062600065735C636C695C6E72665F636C692E63F8
:1062700000000000E6AF0000257300000FB4F8B581
:10628000044608980E4620B91DA140F65120FBF7A0
:10629000EBF924B91AA140F65220FBF7E5F9A06802
:1062A00018B1606808B1206820B915A140F65320E4
:1062B000FBF7DAF909A80090A068D0F8481349075D
:1062C00017D5817DB14214D0C58A3146204604F0ED
:1062D000CBFB6A462069089900F08EFCE9B22046A3
:1062E00004F0C2FB290A204604F0A0FBF8BC5DF8CC
:1062F00014FB6A462069089900F07EFCF6E700006E
:106300002E2E5C2E2E5C2E2E5C2E2E5C2E2E5C2EC7
:106310002E5C636F6D706F6E656E74735C6C69621A
:106320007261726965735C636C695C6E72665F63EF
:106330006C692E63000000002DE9F04F89B0904693
:106340000D46040004D191A140F6D220FBF78CF950
:10635000A06818B1606808B1206820B98BA140F628
:10636000D320FBF781F99748FCF794F80646954847
:106370003338FCF78FF8301A1FFA80F9914892A24F
:1063800020380090A0680821406803682046FFF785
:1063900075FFA06840680068FCF77CF806468948ED
:1063A0002038FCF777F8304482B2A06800234068B8
:1063B00041682046FEF730F985A208212046FFF704
:1063C0005DFFB8F1000F22D00DB300261DE000BF25
:1063D00006EB460A05EB8A0BDBF80400FCF75AF8DB
:1063E000074655F82A00FCF755F8391849450BD9E6
:1063F000DBF80400FCF74EF8074655F82A00FCF7D6
:1064000049F838441FFA80F9761C4645E0D36D48B8
:106410003338FCF73FF84844801C1FFA80F969487C
:1064200000904B466DA208212046FFF727FF09F197
:10643000030087B2079000233A466AA12046FEF780
:10644000EBF8002D51D000264DE000BF06EB460AC8
:1064500005EB8A0B55F82A00DBF8043063B348B328
:10646000584965A23339CDE9001008212046FFF7CD
:1064700005FF09F102000090DBF80400FCF70AF8C0
:10648000074655F82A00FCF705F807444D4833380D
:10649000FCF700F839180098401A801E81B2204697
:1064A000FDF754FC3A225749206900F039FB009867
:1064B000401C0AE0009301E040B100904B4647A227
:1064C00008212046FFF7DAFE079887B2DBF80810AC
:1064D00029B100233A462046FEF79EF802E0204606
:1064E000FDF72EFB761C4645B0D3A0684068806857
:1064F000002847D0814600200646054603AF02909B
:106500002A466D1C02AB012148460097FCF7B4FEF9
:10651000029850B10068FBF7BDFFB042F0D9029875
:106520000068FBF7B7FF86B2EAE7012D2AD036A252
:1065300008212046FFF7A2FE0025B8462A466D1C1A
:1065400002AB01214846CDF80080FCF795FE029889
:10655000002817D0B11C8FB2006800903B461FA2E4
:1065600008212046FFF78AFE0298FF1CBAB2416854
:1065700021B100232046FEF74FF8DFE72046FDF764
:10658000DFFADBE709B0BDE8F08F00002E2E5C2EAD
:106590002E5C2E2E5C2E2E5C2E2E5C2E2E5C636FBF
:1065A0006D706F6E656E74735C6C69627261726936
:1065B00065735C636C695C6E72665F636C692E63A5
:1065C00000000000ECAF0000257325730000000000
:1065D0004F7074696F6E733A0D0A00002020252DEC
:1065E0002A733A0053686F7720636F6D6D616E6434
:1065F0002068656C702E000020202573257325739C
:10660000000000002C1A0000537562636F6D6D610D
:106610006E64733A0D0A00008068D0F84803C0F336
:10662000400070478068D0F84803C0F340007047CE
:106630002DE9F0411E46DDF8188015460F4604008E
:1066400004D10DA140F69410FBF70EF82A46394606
:10665000204600F02DF805000CD15EB14146E068FF
:1066600000F01EFF002802DA0420BDE8F081E06897
:10667000012141722846F8E72E2E5C2E2E5C2E2E2C
:106680005C2E2E5C2E2E5C2E2E5C636F6D706F6EFA
:10669000656E74735C6C69627261726965735C6368
:1066A0006C695C6E72665F636C692E63000000004B
:1066B0002DE9F04715460E46040004D143A140F6EB
:1066C0003610FAF7D1FFA06818B1606808B12068E9
:1066D00020B93EA140F63710FAF7C6FF207E0A28FF
:1066E00006D00D2804D039A140F63810FAF7BCFFC7
:1066F000E0682346434A4461606801680F68314698
:10670000B84700285FD1606920B930A140F6471032
:10671000FAF7AAFF606901F084FB002853D1A16851
:10672000C1F83C03A168C1F840034FF45371A0685D
:10673000F9F7FFFEA068D0F8481341F02001C0F837
:106740004813A068D0F8481365F38201C0F84813D5
:10675000A068D0F8481341F00801C0F84813A168B8
:106760000120294F0870A168502040F66319488223
:10677000A1681820002408822448254940F6641A9C
:106780000D1A804613E000BF18EBC40603D10FA119
:106790004846FAF769FF7068006818B90BA15046BF
:1067A000FAF762FF7068006847F82400641CB4EBD5
:1067B000D50FE9D3072D05D9E908164B0422384631
:1067C000F9F742FE0020BDE8F08700002E2E5C2E77
:1067D0002E5C2E2E5C2E2E5C2E2E5C2E2E5C636F7D
:1067E0006D706F6E656E74735C6C696272617269F4
:1067F00065735C636C695C6E72665F636C692E6363
:1068000000000000C9270000BC02002060D1000089
:10681000F0D100001DA100000023FCF707B9000023
:1068200010B5040004D122A140F61B20FAF71CFF8A
:10683000A06818B1606808B1206820B91CA140F6B2
:106840001C20FAF711FFA068102100F55270FEF726
:106850009EFFA0680078F8B101281DD002281BD146
:106860002046FBF70FFD00212046FBF743FB98B1C4
:106870001DA2032120462368FFF700FD2046FBF7F9
:1068800003FB48B1A36818A2082120462033FFF774
:10689000F5FC2046FDF724FA206900F081F9A06894
:1068A000BDE810406FF0100100F55270FEF75ABFBE
:1068B0002E2E5C2E2E5C2E2E5C2E2E5C2E2E5C2E12
:1068C0002E5C636F6D706F6E656E74735C6C696265
:1068D0007261726965735C636C695C6E72665F633A
:1068E0006C692E63000000002573000070B5040081
:1068F00004D117A140F6EA10FAF7B6FEA06818B165
:10690000606808B1206820B911A140F6EB10FAF7D1
:10691000ABFEA0680078012801D0082070BD606837
:1069200001688A680021904705000FD108212046A0
:1069300004F09AF80121204604F078F812A12069A9
:1069400000F0EEF802212046FBF790FD284670BDCE
:106950002E2E5C2E2E5C2E2E5C2E2E5C2E2E5C2E71
:106960002E5C636F6D706F6E656E74735C6C6962C4
:106970007261726965735C636C695C6E72665F6399
:106980006C692E63000000000D0A0A0000F18040CF
:106990000068002800D00120704708B500F1804051
:1069A000002101600068009008BD000070B50A4C2D
:1069B000207808B185250CE00020A060606020618F
:1069C000E060064802F02AFA054602F0F5F90120D7
:1069D0002070284670BD0000A41100201D2B00006F
:1069E00070B5174C0546207818B916A1C120FAF7E2
:1069F0003BFEA07838B115B16968012088470020B6
:106A0000FAF74EFD0CE00020FAF74AFD25B10C48DC
:106A100029461030FEF760F9E06808B902F05CFA28
:106A2000E068401CE0600020FAF768FDE06800289C
:106A300005D1BDE8704003A1DD20FAF715BE70BD99
:106A4000A41100202E2E5C2E2E5C2E2E5C2E2E5C91
:106A50002E2E5C2E2E5C696E746567726174696F90
:106A60006E5C6E7266785C6C65676163795C6E7291
:106A7000665F6472765F636C6F636B2E6300000009
:106A8000F0B505460478154889B0164640F824202C
:106A9000124A0869121DA2F1080742F82400487F33
:106AA000385520226846F9F71DFD04942878385C93
:106AB00048B10EB10A4A00E000226946281D02F0E2
:106AC0003FFD09B0F0BD0EB1064A00E00022694664
:106AD00005F10C0002F032FBF3E700003801002062
:106AE00045A80000EDA6000030B40378054CE35C37
:106AF0001BB130BC001D02F03BBE30BC0C3002F0BC
:106B00002BBC0000340100200178044A515C11B113
:106B1000001D02F0B9BE0C3002F0B0BC3401002000
:106B20000FB438B5040003D110A11C20FAF79CFD66
:106B3000606918B90DA11D20FAF796FD206818B9F3
:106B40000AA11E20FAF790FD606818B907A11F205E
:106B5000FAF78AFD0599002905D006A800906A4633
:106B6000204600F049F838BC5DF814FB2E2E5C2E50
:106B70002E5C2E2E5C2E2E5C2E2E5C2E2E5C6578CE
:106B80007465726E616C5C667072696E74665C6E60
:106B900072665F667072696E74662E630000000034
:106BA00010B5040003D107A10B20FAF75DFDA26820
:106BB000002A05D0D4E90403216898470020A0608A
:106BC00010BD00002E2E5C2E2E5C2E2E5C2E2E5C18
:106BD0002E2E5C2E2E5C65787465726E616C5C6620
:106BE0007072696E74665C6E72665F667072696EF2
:106BF00074662E63000000002DE9FC4791460C46A8
:106C00005FEA000804D183A14FF49F70FAF72CFDCE
:106C1000D8F8140020B97FA14FF4A070FAF724FD32
:106C2000D8F8000020B97BA140F24110FAF71CFD12
:106C3000D8F8040020B977A14FF4A170FAF714FD39
:106C4000002C76D014F8011B39B125290ED040460E
:106C5000FAF75AFD20780028F4D198F80C000028A3
:106C600067D04046BDE8FC47FFF79ABF00200122ED
:106C700021782B291BD02D2902D0302908D102E000
:106C800040F0010001E040F00200641C002AEFD156
:106C900000252A290ED02178A1F130020A2A11D22A
:106CA00005EB850201EB4205641C303DF1E740F045
:106CB0000400EAE7D9F800100B1DC9F80030096894
:106CC000641C0D44217800232E290BD114F8011FD8
:106CD000A1F130020A2A05D203EB830201EB420341
:106CE000303BF3E76C290DD068290BD0692921D0FE
:106CF0000BDC252918D0582931D063290ED06429FE
:106D000015D117E014F8011FECE7702969D0732939
:106D100032D075291BD0782909D120E0D9F800009C
:106D2000011DC9F8001001784046FAF7EDFC641C1B
:106D300090E76CE0D9F800100A1DC9F80020096836
:106D4000CDE900500A224046FDF78AFEEFE7D9F868
:106D500000100A1DC9F8002009680A2206E0D9F8C7
:106D600000100A1DC9F8002009681022CDE9005062
:106D7000404603F001FEDAE7D9F8001000270A1DAB
:106D8000C9F800200E68C00705D112E04046761C05
:106D90007F1CFAF7B9FC31780029F7D104E02021F3
:106DA00040466D1EFAF7B0FCBD42C0D9002DF6D1A9
:106DB000BDE74EB13046F9F7E3FB074604E020217A
:106DC00040466D1EFAF7A0FCBD4206D9002DF6D153
:106DD00003E04046761CFAF797FC31780029F8D199
:106DE000A5E7D9F80000011DC9F800100568302199
:106DF0004046FAF789FC78214046FAF785FC0820DE
:106E00000021CDE90001034610222946B0E7BDE884
:106E1000FC8700002E2E5C2E2E5C2E2E5C2E2E5C0F
:106E20002E2E5C2E2E5C65787465726E616C5C66CD
:106E30007072696E74665C6E72665F667072696E9F
:106E400074665F666F726D61742E63002DE9F84F92
:106E50002E4D0400894628884FF0010C69689A4637
:106E600016460CEB004025D02268002A2DD0002EBB
:106E700035D062684FF010071268531E13EA090FED
:106E800012D1E046724349462046FAF7BAF9002883
:106E90002FD0206853463246056901B04946204646
:106EA000AC46BDE8F04F604700292DD0184B19A221
:106EB000009726E031B10E210091154B1FA221A1B0
:106EC00000F0B9FD0E20BDE8F88F31B10821009126
:106ED0000F4B27A21BA100F0AEFD0820F3E731B154
:106EE000092100910A4B25A216A100F0A4FD09205A
:106EF000E9E7686840B100972988054B204A08EB0C
:106F0000014010A100F097FD1020DCE72C040020C8
:106F100087B00000616464725F69735F7061676568
:106F20005F616C69676E656428705F66732C2070A2
:106F30006167655F6164647229000000705F667359
:106F400000000000257320636865636B206661693B
:106F50006C656420696E2025732829207769746820
:106F60002076616C756520307825782E0000000051
:106F7000705F66732D3E705F617069006C656E00B6
:106F80001CC60000F8B5030010484FF001064FF092
:106F90000E054468008806EB004009D069B119600D
:106FA0000C6801B0A446BDE8F040114618466047A1
:106FB00054B1074B07A2009503E02CB1044B07A284
:106FC000009508A100F037FD0E20F8BD2C0400202C
:106FD0003CB00000705F667300000000705F61707D
:106FE00069000000257320636865636B2066616932
:106FF0006C656420696E2025732829207769746880
:107000002076616C756520307825782E00000000B0
:1070100018B102680AB15269104700207047000099
:107020002DE9F84F414C05008B46208891464FF0E2
:107030000106DDF828A0616898464FF00E0206EBC5
:1070400000401BD0B9F1000F1DD02A68002A23D0C0
:107050000922B8F1000F29D06B685F68B8FBF7FC14
:1070600007FB1C83002B27D029B1314B009231A2A2
:107070003BA100F0E0FC0920BDE8F88F51B100927F
:107080002B4B42A203E029B1294B009241A234A12B
:1070900000F0D1FC0E20EFE731B108210091244B24
:1070A0003EA22FA100F0C7FC0820E5E70029E2D0AE
:1070B00000921F4B3CA2DBE75846FAF79CF81027DA
:1070C00098B14846FAF797F8C8B14246594628465B
:1070D000FAF797F8F8B1CDF800A0286843464A4679
:1070E000C46859462846A047C6E7606800281BD0F8
:1070F000009720880E4B06EB00402CA207E060684A
:1071000090B1009720880A4B06EB00402DA214A1F5
:1071100000F091FC08E0606830B100972088044BD3
:1071200006EB004030A2F2E71020A5E72C04002077
:1071300074B0000021286C656E202520705F667396
:107140002D3E705F666C6173685F696E666F2D3E81
:1071500070726F6772616D5F756E697429000000EF
:10716000257320636865636B206661696C656420C4
:10717000696E202573282920776974682076616CF0
:10718000756520307825782E00000000705F6673EA
:1071900000000000705F737263000000705F667330
:1071A0002D3E705F617069006C656E006164647291
:1071B0005F69735F616C69676E656433322864650B
:1071C00073742900616464725F69735F616C6967DD
:1071D0006E65643332282875696E7433325F7429A2
:1071E000705F737263290000616464725F69735F2A
:1071F00077697468696E5F626F756E647328705F1B
:1072000066732C20646573742C206C656E290000F5
:107210002DE9FF411C46DDE90A7815460E46684611
:1072200000F09CF846EA450141EA840141EA072260
:1072300042EA0841009A00EB8200C0F80017BDE85E
:10724000FF812DE9FF411C46DDE90A7815460E460F
:10725000684600F0A7F846EA450141EA840141EAA0
:10726000072242EA0841009A00EB8200C0F80017AA
:10727000BDE8FF811CB5002100910B460122019160
:10728000FFF7C6FF1CBD1CB5002100910B46012273
:107290000191FFF7D6FF1CBD1CB500220B460092E2
:1072A00011460192FFF7B4FF1CBD1CB500220B462E
:1072B000009211460192FFF7C4FF1CBD1CB50021CE
:1072C00000910B46012201911146FFF7A1FF1CBD61
:1072D0001CB5002100910B46012201911146FFF7D8
:1072E000B0FF1CBD13B50C46684600F013F80099BA
:1072F00000EB8101D1F8002722F44032C1F80027C9
:10730000009900EB8100D0F8001741EA0441C0F871
:1073100000171CBD10B50068202804D303A140F25B
:10732000A110FAF7A1F94FF0A04010BD2E2E5C2E4F
:107330002E5C2E2E5C2E2E5C2E2E5C2E2E5C6D6F07
:1073400064756C65735C6E7266785C68616C2F6ED8
:1073500072665F6770696F2E6800000010B5006884
:10736000202804D303A140F2A110FAF77DF94FF0D1
:10737000A04010BD2E2E5C2E2E5C2E2E5C2E2E5C80
:107380002E2E5C2E2E5C6D6F64756C65735C6E7258
:1073900066785C68616C2F6E72665F6770696F2ECD
:1073A0006800000010B50068202804D303A140F253
:1073B000A110FAF759F94FF0A04010BD2E2E5C2E07
:1073C0002E5C2E2E5C2E2E5C2E2E5C2E2E5C6D6F77
:1073D00064756C65735C6E7266785C68616C2F6E48
:1073E00072665F6770696F2E6800000001B56846BD
:1073F000FFF7B4FF009A01219140C0F8081508BDBD
:1074000001B56846FFF7CEFF009A01219140C0F810
:10741000081508BDF8B504460B48661815460068FF
:107420000090012E04D909A140F2B920FAF71CF905
:10743000694605E051F82400D0F81005641C01C528
:10744000A642F7D8F8BD00005CAD00002E2E5C2EE1
:107450002E5C2E2E5C2E2E5C2E2E5C2E2E5C6D6FE6
:1074600064756C65735C6E7266785C68616C2F6EB7
:1074700072665F6770696F2E68000000034908B587
:107480000844002101600068009008BD00600040D1
:1074900002494058012800D0002070470060004099
:1074A0002DE9F0410E461C4904460025D1F8102470
:1074B000104609E0037AAB4205D16D1C0A2DF7DBBB
:1074C0004FF0FF3525E040680028F3D1681C20D03C
:1074D0002572D1F8100440B140686060D1F8100402
:1074E00044600027DFF834800FE00020C1F810442A
:1074F0006060F6E708EBC700C279B24200D33246BB
:10750000207A394600F090FB7F1C00F05DFBB8420A
:10751000F0D82846BDE8F0814C150020F0D10000DD
:1075200038B54469C0680022694600F05BFF002856
:1075300003D100212046FAF7DDFC38BD10B54469BF
:10754000606801688A680121904718B10420A16829
:10755000087010BD0320FAE72DE9F341466904469F
:10756000B068007804281ED0032807D0002501A9A0
:10757000E06801F06DF885F0010709E00125F6E704
:1075800039463046FAF7B6FC01A9E06801F060F828
:107590000028F5D1019800F040FC002D03D0002117
:1075A0003046FAF7A7FCBDE8FC810000014880687E
:1075B00002F018BB0C02002038B50022164917480B
:1075C000FFF7E0FC164C012108B1217038BD022004
:1075D000207014480025C0F8801101216068FDF773
:1075E000A7FC1149486A0A8DCB6A61F39F200F49B5
:1075F000086090B2C1E901030A4600950C230748D0
:107600002169FFF70DFD20690C302061A068BDE8FD
:1076100038400121FDF78CBCA8B000000403002015
:107620000C02002004E000E02CB200003C1300201B
:1076300070B50B4C0D46207801280FD0084600F09D
:10764000ECFB2946A068FDF787FF2078022805D1CA
:10765000A068BDE870400121FDF76ABC70BD000064
:107660000C02002070B5074D012000232870064849
:107670000122010B09030C460448FFF7E7FB2C61CC
:1076800070BD00000C020020AFE4000004030020E5
:107690003EB50F490B0B0F491B0303F6FF72C1E9FF
:1076A0000332014600220B48FFF76CFC04000DD1A9
:1076B0000025009502AA01A9684600F00FF80028ED
:1076C000F8D0054800990161057020463EBD0000D4
:1076D000AFE40000040300200C02002070B50D464A
:1076E00001681646044611B91248010B09031248F5
:1076F0002160FFF78DFC68B1206828600C30306095
:107700002868006800F00301012905D0022907D08C
:10771000052070BD062070BDC0F38310800002E01C
:10772000800D02F021FC21680C300844206000200C
:1077300070BD0000AFE40000040300200148406871
:1077400002F050BA0C0200207047000070B50E4CD9
:107750000D462078002815D1084600F05EFB29462A
:107760006068FDF7F9FEA1690844A06104F10C000E
:10777000FDF7EFFF002805D16068BDE870400021EB
:10778000FDF7D6BB70BD00000C0200200A4A01299B
:1077900002EBC00007D0022907D0032907D0042933
:1077A00007D00020704702207047042070470079FE
:1077B0007047407970470000F0D100002DE9FF5F6D
:1077C000F9F7B2FF18B1002004B0BDE8F09F874C74
:1077D0000020C4F81804BFF34F8F60680090A668BB
:1077E0004FF00009304004EB800008E02168009869
:1077F000814201D86160E6E7304004EB80000C3044
:107800006946FDF733FA0028F0D101AAA046009995
:1078100001EA060408EB8403491CDB6842F82030C7
:10782000401C00910328F2D3019800F003000228C5
:1078300002D0012850D0BEE00198A022810D8A46D6
:10784000B2EB905F00D8A0210C4664F39F50C0F3C8
:10785000C20701900C31664800F096FA0500EAD0A4
:1078600000F0DBFA4B460C2201A9284600F0F0FAA2
:10787000009909F10C0B3140701A8000001D844200
:1078800023D95A4E0C3630B1C2B208EB8101201A0E
:1078900091460C3104E03146E2B200269146304672
:1078A000C4B25B46284600F0D3FA0BEB09032EB1B5
:1078B000224631464FEA050000F0CAFA00990AF163
:1078C000030001EB900000903DE008EB81015B4676
:1078D000224628460C31EFE70198C0F383100628B2
:1078E00000D30620019960F38911C1F38310C1F31D
:1078F000C207C01C019181003D4800F045FA050017
:1079000059D000F08AFA4B460C2201A9284600F013
:107910009FFA09F10C0900240FE000984B4602463B
:10792000304008EB8001501C0090042228460C31A6
:1079300000F08EFA09F10409641C0198C0F3831069
:10794000A042EAD8B5B3D8F81044D8F8180446468F
:10795000F8B1284600F067FA42E0607A012817D1B2
:10796000BDF80800234A00EB400002EB8000217ABA
:10797000806801EB4101C84000F00700052F00D1ED
:107980000327B84204D3226820462946126890474C
:107990006468002CE1D1284600F045FA0020F9F790
:1079A0007FFDD6F8180408B9009870600020F9F738
:1079B000A5FD15E0FFE7D8F8104404E02168204653
:1079C000896888476468002CF8D10B48416802290F
:1079D00006D30088022101EB004008A100F018F84E
:1079E000F9F7A2FE80F00100EEE600004C15002041
:1079F00018D3000018030020740400204261636B58
:107A0000656E647320666C757368656400000000C1
:107A100000231A4602F000BB08B5012300926A4613
:107A200002F0FAFA08BD1CB5CDE9002302236A462C
:107A300002F0F2FA1CBD3EB5069C8DE81C00032343
:107A40006A4602F0E9FA3EBD7FB5DDE908458DE8FA
:107A50003C0004236A4602F0DFFA7FBD70B586B0B1
:107A60000DF1280C9CE870008DE87C0005236A4627
:107A700002F0D2FA06B070BD2DE9F0470E468046FE
:107A80001C46924608293ED894F80C90002020739A
:107A90001946104602F03CF80025B54206D218F807
:107AA00005201AA12046FFF73BF803E019A1204664
:107AB000FFF736F86D1C082DEFD317A12046FFF70E
:107AC0002FF80025B54210D218F80570F8F7B2FC6F
:107AD0000068C05D10F03E0F01D03A4600E02E2253
:107AE0000EA12046FFF71CF803E00DA12046FFF78A
:107AF00017F86D1C082DE5D301222146504601F0F0
:107B0000E9FF84F80C90BDE8F087000020253032B2
:107B100078000000202020007C0000002563000089
:107B2000200000002DE9F04705001FD0214C4FF048
:107B30000009FF20C4F80090C4E90190C4F818942B
:107B4000C4F8149484F82094084600F00DF91A48FB
:107B5000C4F80C5400F065F9002808D11749DFF883
:107B60006080A1EB0800C70800241EE00720BDE8E4
:107B7000F087002635460CE0AC4209D058F83400B6
:107B800058F835101422F8F719FD002800DD761C8E
:107B90006D1CBD42F0D30B4904EB440001EB8000A7
:107BA000C0F8049004804680641CBC42E1D30020ED
:107BB000DDE700004C15002018D30000E0D20000E3
:107BC000F0D100001803002002480349401AC00801
:107BD00070470000E0D20000F0D100007FB50546FC
:107BE0001146002401A87BB1FDF7E0FCA0B9019883
:107BF0000B4900EB400001EB800005EB450180687C
:107C0000C84000F0070407E0FDF7D0FC20B90548A4
:107C1000019900EBC100847904B0204670BD0000DA
:107C200018030020F0D1000030B50F4B01EB4101EB
:107C300003EB810400EB40000723A56803FA00F181
:107C40008D4302F007018140294300252A46A160A7
:107C500003FA02F00840D040A84200D90546D21CE1
:107C60000A2AF5D3656030BD1803002013B56846B5
:107C7000FDF79CFC08B100201CBD0248009950F89B
:107C800031001CBDF0D1000070B508480125D0F8C6
:107C9000104480F8205405E0657221682046496848
:107CA00088476468002CF7D170BD00004C15002097
:107CB0002DE9FF4781460C9D00200C462F7B287341
:107CC000984616462946184601F022FF072E42D252
:107CD000DFE806F004090F161F2A36004946284639
:107CE000FEF71EFF37E0494628462268FEF718FFD8
:107CF00031E0D4E9002349462846FEF711FF2AE087
:107D0000A0680090D4E9002349462846FEF708FF02
:107D100021E0D4E90201CDE90001D4E9002349467C
:107D20002846FEF7FDFE16E004F1080007C88DE8BE
:107D30000700D4E9002349462846FEF7F1FE0AE091
:107D400004F108000FC88DE80F00D4E9002349466C
:107D50002846FEF7E5FE00222946404601F0BAFE1D
:107D60002F73BDE8FF870000054A0121054B5160D4
:107D700001E0400849009842FBD8C2E90001704781
:107D80007402002040420F002DE9F041058B80462F
:107D90002D1F4819C01CB0FBF5F0C6B24046FDF7D8
:107DA00003FD041E19D00020207101206071E580C0
:107DB00000272546761EC4F800800BE04046FDF7FC
:107DC000F3FC60B16179491C6171286005467F1C34
:107DD000C0F80080B742F1D32046BDE8F0812046CC
:107DE00000F002F80020F8E72DE9F041457901465E
:107DF0006B1E002201E00968521C9A42FBD30F68F7
:107E00000146002605E038460C68FDF733FD2146A3
:107E1000761CAE42F7D3BDE8F0810121001DFDF7CD
:107E20009BBCFDF76DBD10B504460121001DFDF79B
:107E3000B4FC10F0FF0F04D12046BDE81040FFF75E
:107E4000D3BF10BD38B501240094FDF73BFB38BD0E
:107E500038B500240094FDF735FB38BD2DE9F84F07
:107E6000834600F091F90546DBF80800D0F8480396
:107E7000C0F3400030B15846BDE8F84F002211462B
:107E8000FEF75ABA1C4803681CA208215846FEF7A0
:107E9000F5F91948001D03681DA208215846FEF790
:107EA000EDF9DFF85480DFF8509008F1080800245D
:107EB00009F1100908F1040A1AE00020F9F7F0FAB4
:107EC000C8F80040D9F80070DAF800600020F9F72F
:107ED00015FB234613A2082158460096FEF7CEF95B
:107EE000234617A2082158460097FEF7C7F9641CDD
:107EF000AC42E2D3BDE8F88F90ED00E04D50555F05
:107F0000545950453A093078253038580D0A000048
:107F10004D50555F4354524C3A093078253038580B
:107F20000D0A00000D0A4D50555F524241525B252B
:107F3000755D3A093078253038580D0A0000000088
:107F40004D50555F524153525B25755D3A0930786B
:107F5000253038580D0A00002DE9FC41074680689D
:107F6000D0F84803C0F3400038B102B03846BDE84D
:107F7000F04100221146FEF7DFB900F005F9064690
:107F8000009030480068C00701D02FA300E030A364
:107F900032A208213846FEF771F900244EE0002095
:107FA000F9F77EFA2748001D046026480C30056862
:107FB000001FD0F800800020F9F7A0FAE807234658
:107FC00033D032A208213846FEF758F9C5F34401F0
:107FD0000120491C884008EB0001491ECDE9001032
:107FE000434630A208213846FEF748F9284600F0FB
:107FF000D3F8034637A208213846FEF73FF9284652
:1080000000F048F9034637A208213846FEF736F952
:10801000284600F0FBF8034636A208213846FEF752
:108020002DF9E80003D538A302E038A201E03DA312
:108030003DA208213846FEF721F9641CB442AED3B4
:10804000BDE8FC8194ED00E0456E61626C65640002
:1080500044697361626C6564000000004D505520F6
:1080600053746174653A2025732C20257520756E34
:10807000696669656420726567696F6E73206176F1
:108080006961626C652E0D0A0D0A00005265676910
:108090006F6E2025753A20456E61626C65640D0A2D
:1080A00000000000092D204C6F636174696F6E3A07
:1080B000093078253038582D307825303858202828
:1080C00073697A653A202575206279746573290D84
:1080D0000A000000092D204163636573733A092586
:1080E000730D0A00092D20547970653A090925732A
:1080F0000D0A0000092D2043616368696E673A0923
:1081000025730D0A00000000584E00005265676993
:108110006F6E2025753A2044697361626C65640D49
:108120000A0000002D2D0000092D20466C616773A8
:108130003A0925730D0A0D0A0000000008B501294F
:1081400005D08168D1F84813C1F3400129B100225C
:10815000BDE808401146FEF7EFB85168009113687A
:1081600002A20221FEF78AF808BD000025733A201A
:10817000756E6B6E6F776E20706172616D65746580
:10818000723A2025730D0A0002480068C0F30720E8
:108190007047000090ED00E0C0F30260082813D2A1
:1081A000DFE800F00406080A0C0E101007A0704764
:1081B00008A0704709A070470AA070470BA070473D
:1081C0000CA070470DA070470EA070472D2D2F2DCD
:1081D0002D00000052572F2D2D00000052572F5216
:1081E0004F00000052572F52570000003F3F2F3FD3
:1081F0003F000000524F2F2D2D000000524F2F52F4
:108200004F000000556E6B6E6F776E0010B5C0F3B7
:10821000C241C0F34043C0F3004200F47C100404A8
:10822000240C17D10014152814D2DFE800F00B0B32
:108230000D0F0B0B0B0B0B1313110B13130B0B135A
:1082400013130B000A4810BD0AA010BD0BA010BDEF
:108250000CA010BD042908D38807000F40EA430092
:108260000B49104351F8200010BD0148383010BDB3
:10827000CC81000057542F575400000057422F570D
:1082800042000000574257412F574257410000001B
:10829000F400002000F47C100104090C15D1011435
:1082A000152912D2DFE801F00B0D18180B0D161668
:1082B00018111118161111160F1111110F0008A025
:1082C00070470EA0704712A07047C10C042905D357
:1082D000400301D510A0704714A0704715A0704747
:1082E0005374726F6E676C792D6F7264657265641A
:1082F0002C20536861726561626C65004465766923
:1083000063652C20536861726561626C65000000D2
:1083100044657669636500004E6F726D616C2C2058
:10832000536861726561626C650000004E6F726D2A
:10833000616C00005265736572766564206F72200F
:10834000496D706C656D656E746174696F6E204403
:108350006566696E65640000094902220A60BFF320
:108360006F8FBFF34F8F0A1D106006480268002A06
:10837000FCD000200860BFF36F8FBFF34F8F7047B2
:1083800004E5014000E4014070B50E4C0123236078
:10839000BFF36F8FBFF34F8F00230B4D08E000BF7B
:1083A00051F8236040F823602E68002EFCD05B1C3F
:1083B0009342F5D300202060BFF36F8FBFF34F8F40
:1083C00070BD000004E5014000E4014000F180417F
:1083D0000868002210B101200A60704710467047FB
:1083E000704700002DE9F04190460D4604004FF023
:1083F000000703D123A1B320F9F736F91DB921A154
:10840000B420F9F731F90020F9F74AF8204600F0D6
:1084100057F830B105270020F9F770F83846BDE865
:10842000F08120680668B8F1000F05D10168204688
:1084300000F0FCF821680860E268012A0CD0022AEA
:108440000ED0042A11D06068082A13D006FB02015E
:108450002846F8F747F8DEE76068805D2870DAE7BD
:10846000606830F816002880D5E7606850F826006C
:108470002860D0E700EBC601D1E90001C5E90001A1
:10848000C9E700002E2E5C2E2E5C2E2E5C2E2E5C5C
:108490002E2E5C2E2E5C636F6D706F6E656E747326
:1084A0005C6C69627261726965735C717565756532
:1084B0005C6E72665F71756575652E630000000005
:1084C00010B5040004D107A14FF4F270F9F7CCF80D
:1084D000216808684968884201D1012010BD002048
:1084E00010BD00002E2E5C2E2E5C2E2E5C2E2E5CDF
:1084F0002E2E5C2E2E5C636F6D706F6E656E7473C6
:108500005C6C69627261726965735C7175657565D1
:108510005C6E72665F71756575652E6300000000A4
:1085200070B5040003D108A16420F9F79DF8206814
:1085300005684168204600F079F8A84201D1012081
:1085400070BD002070BD00002E2E5C2E2E5C2E2EE5
:108550005C2E2E5C2E2E5C2E2E5C636F6D706F6E0B
:10856000656E74735C6C69627261726965735C716B
:10857000756575655C6E72665F71756575652E6390
:108580000000000010B5040004D104A14FF4F970FC
:10859000F9F76AF82068806810BD00002E2E5C2E66
:1085A0002E5C2E2E5C2E2E5C2E2E5C2E2E5C636F8F
:1085B0006D706F6E656E74735C6C69627261726906
:1085C00065735C71756575655C6E72665F71756506
:1085D00075652E630000000010B5040004D104A1ED
:1085E0004FF4FC70F9F740F821680020886010BD56
:1085F0002E2E5C2E2E5C2E2E5C2E2E5C2E2E5C2EB5
:108600002E5C636F6D706F6E656E74735C6C696207
:108610007261726965735C71756575655C6E7266B1
:108620005F71756575652E630000000070B50C46BE
:10863000050003D105495120F9F716F8A868A042B2
:1086400001D9601C70BD002070BD00009C85000039
:108650002DE9F0410E4604004FF0000803D12CA193
:108660006F20F9F701F81EB929A17020F8F7FCFF77
:108670000020F8F715FF2046FFF752FF070009D04A
:10868000207C38B14FF004080020F8F737FF40464F
:10869000BDE8F0812068456841682046FFF7C6FFC5
:1086A0002168486037B1206801682046FFF7BEFFA7
:1086B00021680860E268012A14D0022A16D0042A30
:1086C00019D0082A1CD06068314605FB0200F7F774
:1086D00009FF204601F098FA21688A688242D3D2C5
:1086E0008860D1E7616830784855F2E76168308882
:1086F00021F81500EDE76168306841F82500E8E7EA
:10870000D6E90001626802EBC502C2E90001E0E7B8
:108710002E2E5C2E2E5C2E2E5C2E2E5C2E2E5C2E93
:108720002E5C636F6D706F6E656E74735C6C6962E6
:108730007261726965735C71756575655C6E726690
:108740005F71756575652E63000000002DE9F04FBF
:108750008046806889B0D0F84803C0F3400038B143
:1087600009B04046BDE8F04F00221146FDF7E4BDD8
:10877000012907D909B04046BDE8F04F1FA20221E8
:10878000FDF77CBD2249DFF88CB0A1EB0B001C216A
:10879000B0FBF1F7002529E0C5EBC5010BEB810427
:1087A0002046D4E9026AFFF7EDFE8146204600F03C
:1087B00041F8642209FB02F14243B1FBF6F1B2FB3E
:1087C000F6F26369247CB4B10FF24C0CCDF81CC0F6
:1087D000CDF800A0CDE90596CDE90120CDE90361F2
:1087E000104A08214046FDF749FD6D1CBD42D3D318
:1087F00009B0BDE8F08F0FF2300CE7E7426164206A
:10880000617267756D656E7420636F756E740000BC
:10881000A4D3000034D300004E6F206F76657266DB
:108820006C6F7700E0C600004F766572666C6F77FC
:108830000000000010B5040004D108A140F2D710D8
:10884000F8F712FF0020F8F72BFE204601F0DCF9C4
:1088500004460020F8F752FE204610BD2E2E5C2E56
:108860002E5C2E2E5C2E2E5C2E2E5C2E2E5C636FCC
:108870006D706F6E656E74735C6C69627261726943
:1088800065735C71756575655C6E72665F71756543
:1088900075652E63000000002DE9F0411F46154666
:1088A0000E00044603D11D491520F8F7DDFE1DB961
:1088B0001A491620F8F7D8FE37B1A068FCF749FF2F
:1088C00010B11120BDE8F081A0686168D0E903C350
:1088D000ACEB0302481C824207D10020286017B18C
:1088E000A068FCF72DFF0020ECE70CEA010003EA8A
:1088F0000102904202D3091A491C01E0A3EB0C01CA
:108900002B688B4200D219462960216808443060E8
:10891000A0682A68C1681144C160E4E75CC7000030
:108920002DE9F04117465FEA0108054603D12149C8
:108930009C20F8F799FE1FB91E499D20F8F794FE78
:10894000A868001DFCF705FF10B11120BDE8F081FB
:10895000A868816800690C1A3868A04200D20446F1
:108960003C60AA6869681069926808400A408242BF
:1089700001D9161A01E00E1A761CB44208D92968EA
:10898000324608444146F7F7ADFDA41B0020B04431
:108990002968224601444046F7F7A4FDA8683A68D2
:1089A000016911440161A868001DFCF7C9FE00209F
:1089B000CCE700005CC700002DE9F04117465FEAF4
:1089C0000108054603D11E494D20F8F74DFE1FB999
:1089D0001B494E20F8F748FEA868FCF7BAFE10B114
:1089E0001120BDE8F081A86881680069081A6968EB
:1089F0000C1A3868641CA04200D204463C60A86887
:108A00006968806808400E1A761CB44208D9296843
:108A1000324608444146F7F765FDA41B0020B044E8
:108A20002968224608444146F7F75CFDA8683A6881
:108A3000816811448160A868FCF782FE0020D0E7BD
:108A40005CC7000010B5826894681369E41AA142FB
:108A500001D9042010BD19441161826851618068F8
:108A6000001DFCF76DFE002010BD00002DE9F04157
:108A70001E4614460F00054603D11D496D20F8F728
:108A8000F3FD1CB91A496E20F8F7EEFD3EB1A86857
:108A9000001DFCF75EFE10B11120BDE8F081A96851
:108AA00088684969421A09D06B68194018408842A1
:108AB0000DD9266896420AD9226010E00020206075
:108AC0001EB1A868001DFCF73BFE0020E5E78842C8
:108AD00005D8581A2268401C824200D920602868B4
:108AE00008443860A8682268416911444161ECE794
:108AF0005CC7000082680021916082681161826811
:108B000051618268D16082685160806801607047FD
:108B100070B58268456894681369E31AEB1A5B1CA8
:108B2000994201D9042070BD214491608268D160CE
:108B30008068FCF708FE08B1002070BD082070BDF9
:108B400070B50D46060003D10BA11420F8F78CFD7B
:108B50001DB909A11520F8F787FD746804E0B26813
:108B60002946904718B1246820680028F7D120686A
:108B70002860256070BD00002E2E5C2E2E5C2E2EEF
:108B80005C2E2E5C2E2E5C2E2E5C636F6D706F6ED5
:108B9000656E74735C6C69627261726965735C7333
:108BA0006F72746C6973745C6E72665F736F7274EB
:108BB0006C6973742E63000010B5040003D103A127
:108BC0003D20F8F751FD206810BD00002E2E5C2ED0
:108BD0002E5C2E2E5C2E2E5C2E2E5C2E2E5C636F59
:108BE0006D706F6E656E74735C6C696272617269D0
:108BF00065735C736F72746C6973745C6E72665FBC
:108C0000736F72746C6973742E63000010B5040086
:108C100003D103A13720F8F727FD6068006810BD75
:108C20002E2E5C2E2E5C2E2E5C2E2E5C2E2E5C2E7E
:108C30002E5C636F6D706F6E656E74735C6C6962D1
:108C40007261726965735C736F72746C6973745C62
:108C50006E72665F736F72746C6973742E6300005A
:108C600010B5040003D105A12B20F8F7FDFC6168C5
:108C70000868002801D002680A6010BD2E2E5C2E04
:108C80002E5C2E2E5C2E2E5C2E2E5C2E2E5C636FA8
:108C90006D706F6E656E74735C6C6962726172691F
:108CA00065735C736F72746C6973745C6E72665F0B
:108CB000736F72746C6973742E63000070B50C4628
:108CC000050003D10BA14320F8F7CEFC1CB909A184
:108CD0004420F8F7C9FC0021686806E0A24203D1ED
:108CE00021680160012103E010460268002AF5D1E5
:108CF000084670BD2E2E5C2E2E5C2E2E5C2E2E5C19
:108D00002E2E5C2E2E5C636F6D706F6E656E7473AD
:108D10005C6C69627261726965735C736F72746CAA
:108D20006973745C6E72665F736F72746C6973746E
:108D30002E6300000C4A10B502F58C730EE0991AF0
:108D4000C91001EBD171491002EBC1010C688442DA
:108D500001D90B4602E005D201F108029A42EED396
:108D6000002010BD486810BD14B1000000B5FFF729
:108D7000E1FF002800D1014800BD000000B1000063
:108D80004058002800D00120704708B5002242500A
:108D90004058009008BDD0F80403084000D00120DE
:108DA00070474058002800D00120704708B50022C5
:108DB00042504058009008BD084810B5007918B9D5
:108DC00007A19520F8F750FC00F0DAF812490120CD
:108DD00008600249091F087010BD0000440100200E
:108DE0002E2E5C2E2E5C2E2E5C2E2E5C2E2E5C2EBD
:108DF0002E5C6D6F64756C65735C6E7266785C6416
:108E00007269766572735C7372635C6E7266785FAA
:108E1000636C6F636B2E63001805004010B504008F
:108E200003D108A17C20F8F71FFC144900200A791F
:108E30000AB1852010BD01220C600A7100224A711E
:108E400010BD00002E2E5C2E2E5C2E2E5C2E2E5C75
:108E50002E2E5C2E2E5C6D6F64756C65735C6E726D
:108E600066785C647269766572735C7372635C6E5B
:108E70007266785F636C6F636B2E63004401002041
:108E800070B54FF480763046FDF780FD114CB50586
:108E900060B13046FDF781FD0120C5F80803607917
:108EA00020B9012060712168002088474FF4827644
:108EB0003046FDF76BFD00280AD03046FDF76DFD0A
:108EC0000220C5F808032168BDE87040012008476A
:108ED00070BD00004401002070B51348007918B936
:108EE00012A1BF20F8F7C0FB4FF48270FDF755FDCB
:108EF00002204107C1F804031A4B196841F0807041
:108F000018601948026842F00104046044684FF494
:108F10000A554668361BAE42FBD3026019601349FE
:108F20000120086070BD0000440100202E2E5C2E40
:108F30002E5C2E2E5C2E2E5C2E2E5C2E2E5C6D6FEB
:108F400064756C65735C6E7266785C647269766574
:108F500072735C7372635C6E7266785F636C6F636E
:108F60006B2E6300FCED00E0001000E00800004004
:108F70000121B1EB507F01D10120704700207047E3
:108F800007480068012110F0010F08D14FF0E020E0
:108F9000E02280F80024C0F88012C0F80011704769
:108FA00000E100E070B54FF08040D0F804531A4C57
:108FB00068070CD54FF48470FFF708FA38B1606881
:108FC00018B916A1E020F8F74FFB60688047A806A3
:108FD0000DD54FF48A70FFF7F9F940B1A06818B9C0
:108FE0000EA1E820F8F740FBA1680020884768063A
:108FF00010D54FF48C70FFF7E9F900280AD0A0686B
:1090000018B906A1EF20F8F72FFBA168BDE8704062
:109010000120084770BD00004C0100202E2E5C2E60
:109020002E5C2E2E5C2E2E5C2E2E5C2E2E5C6D6FFA
:1090300064756C65735C6E7266785C647269766583
:1090400072735C7372635C6E7266785F706F776563
:10905000722E630070B50D46040003D10DA151209E
:10906000F8F702FB204600F0B1FD04000FD000200D
:10907000F8F716FA207920B10020F8F73FFA11200E
:1090800070BD0120256020710020F8F737FA00201C
:1090900070BD00002E2E5C2E2E5C2E2E5C2E2E5CC3
:1090A0002E2E5C2E2E5C6D6F64756C65735C6E721B
:1090B00066785C647269766572735C7372635C7007
:1090C00072735C6E7266785F7072732E630000005C
:1090D00010B5040003D106A17520F8F7C5FA2046A3
:1090E00000F074FD002802D000210160017110BD64
:1090F0002E2E5C2E2E5C2E2E5C2E2E5C2E2E5C2EAA
:109100002E5C6D6F64756C65735C6E7266785C6402
:109110007269766572735C7372635C7072735C6E95
:109120007266785F7072732E630000000149024816
:1091300001F0F4BA14120020002000402DE9F041A3
:1091400017460D00064603D11AA18420F8F78CFAC1
:109150003079264A00EB400101EBC00102EB8104AB
:1091600094F82A1011B10820BDE8F081204951F887
:1091700020103068FFF76EFF08B11120F4E7294690
:109180003046F8F7FBF96760286920601FB1297F36
:109190003046FBF7B9FC30680421C0F80015002008
:1091A000A061E06184F8290044F8140F0121A17541
:1091B000DAE700002E2E5C2E2E5C2E2E5C2E2E5C0E
:1091C0002E2E5C2E2E5C6D6F64756C65735C6E72FA
:1091D00066785C647269766572735C7372635C6EE8
:1091E0007266785F756172742E630000141200203D
:1091F00060AD00002DE9F05F054600790F4600EBF9
:10920000400101EBC0014048164600EB810494F890
:109210002A00012804D03DA140F24310F8F724FAB7
:109220004FF4A27A1FB939A15046F8F71DFA26B9B2
:1092300036A140F24510F8F717FA616800204FF4A4
:10924000017811B12A68C2F80883A1694FF00009BA
:1092500069B1E06938B1606810B12868C0F804836A
:109260001120BDE8F09F27610120E66105E0C4F808
:109270002490E760A661C4F81C9094F8291001437B
:1092800002D1284600F010FE60680028286803D04C
:10929000C0F804830020E4E756465146FFF775FD09
:1092A000B2464FF4927B59462868FFF769FD06469F
:1092B0004FF484712868FFF763FD804651462868A3
:1092C000FFF75EFD074648EA07003043EBD056EA59
:1092D000070007D12146286800F0B6FD616AA06941
:1092E0008842E0D8C4F818900EB10320B9E70FB156
:1092F0000F20B6E794F8291001200029296801D031
:109300000860C7E74860C5E7141200202E2E5C2EC7
:109310002E5C2E2E5C2E2E5C2E2E5C2E2E5C6D6F07
:1093200064756C65735C6E7266785C647269766590
:1093300072735C7372635C6E7266785F756172746F
:109340002E63000001684FF40172C1F80823006821
:1093500001214160704700002DE9F0470546007982
:109360000F4600EB400101EBC0002D49164601EB12
:10937000800494F82A00012803D02AA1EF20F8F7EE
:1093800073F91FB927A1F020F8F76EF91EB925A1CE
:10939000F120F8F769F9284600F060F810B11120C3
:1093A000BDE8F0874FF00008C4F82080A760666130
:1093B00084F828804FF48E76474631462868FFF7B8
:1093C000E4FC28684FF00109C0F80890214628689D
:1093D00001F0E8F8606808BBD5F800A00FE000BF16
:1093E00094F8280008B10F2716E031465046FFF7E1
:1093F000C7FC0028F4D02146504601F0D3F8216A7A
:1094000060698142F1D331462868FFF7B9FC002832
:10941000F9D02868C0F80C90C4F814803846BFE72B
:10942000141200202E2E5C2E2E5C2E2E5C2E2E5C16
:109430002E2E5C2E2E5C6D6F64756C65735C6E7287
:1094400066785C647269766572735C7372635C6E75
:109450007266785F756172742E630000007900EBAC
:10946000400101EBC000044901EB80004069002885
:1094700000D0012070470000141200202DE9F047B1
:10948000044600794FF0000900EB400101EBC000F9
:10949000254901EB80072068C0F80095786880B105
:1094A00020682249C0F8081320680121000B40B24F
:1094B00000F01F0291404009800000F1E020C0F858
:1094C00080112068D0F80C25D0F81485D0F80865F4
:1094D000D0F810554FF0FF31C0F81415C0F80C1536
:1094E0002068C0F80815C0F81015501C02D01046AE
:1094F000FDF7C0FEB8F1FF3F02D04046FDF7BAFECF
:10950000681C02D02846FDF7B5FE701C02D030461C
:10951000FDF7B0FE2068FFF7DBFD87F82A90C7F85B
:109520000490BDE8F08700001412002084020200BD
:109530000149024801F09EB940120020002000407D
:109540002DE9F04117460D00064603D118A19620DB
:10955000F8F78AF83079244A00EBC00102EB810465
:1095600094F8201011B10820BDE8F0811F4951F88E
:1095700020103068FFF76EFD08B11120F4E729468E
:109580003046F8F736F86760286920601FB1297FF8
:109590003046FBF70DFB30680821C0F800150020AD
:1095A000A061E0610121606184F82010DCE7000027
:1095B0002E2E5C2E2E5C2E2E5C2E2E5C2E2E5C2EE5
:1095C0002E5C6D6F64756C65735C6E7266785C643E
:1095D0007269766572735C7372635C6E7266785FD3
:1095E00075617274652E63004012002064AD000046
:1095F0002DE9F05F044600790F46DFF830A100EB5B
:10960000C0010AEB8105164695F82000012804D018
:1096100047A140F23110F8F727F827B944A14FF4D9
:109620009970F8F721F826B941A140F23310F8F704
:109630001BF8207908B9FF2E04D93DA14FF49A7088
:10964000F8F712F83846FFF793FCB0B168684FF0AE
:1096500000084FF4047910B12168C1F80893A86993
:109660004FF0000B80B1E86948B1686810B120681C
:10967000C0F804931120BDE8F09F1020FBE72F6194
:109680004FF00108EE6102E0EF60C5E9066B0025CE
:109690004FF488712068FFF789FB4FF4A2712068AE
:1096A000FFF784FB2068C0F83475C0F8386520687F
:1096B000B8F1000F12D0D0F8001241F02001C0F82C
:1096C00000122079D04600EBC0010AEB810040680F
:1096D00038B12168C1F804932846CCE70121016024
:1096E000EFE74FF4887A4FF4A27951462068FFF7EC
:1096F00058FB074649462068FFF753FB06464FF4E0
:1097000092712068FFF74DFB014647EA06000843C7
:10971000EBD0227902EBC20308EB8302C2F818B047
:1097200001B10325002ED7D00F25D5E74012002028
:109730002E2E5C2E2E5C2E2E5C2E2E5C2E2E5C2E63
:109740002E5C6D6F64756C65735C6E7266785C64BC
:109750007269766572735C7372635C6E7266785F51
:1097600075617274652E6300006801214160704765
:109770002DE9F04704460F4600792D4900EBC00063
:1097800001EB8005164695F82000012803D029A199
:10979000E720F7F769FF1FB926A1E820F7F764FF74
:1097A0001EB924A1E920F7F75FFF207908B9FF2E41
:1097B00003D920A1EA20F7F757FF3846FFF7D8FB77
:1097C00030B1204600F052F820B11120BDE8F087FA
:1097D0001020FBE7AF606E614FF4907600273146B2
:1097E0002068FFF7E3FA4FF4AC7841462068FFF7B2
:1097F000DDFA2068AA686969C0F84425C0F84815F0
:10980000206801218160686878B9B14649462068BE
:10981000FFF7C7FA064641462068FFF7C2FA06433B
:10982000F4D000B10F27002068613846CEE7000071
:10983000401200202E2E5C2E2E5C2E2E5C2E2E5CD6
:109840002E2E5C2E2E5C6D6F64756C65735C6E7273
:1098500066785C647269766572735C7372635C6E61
:109860007266785F75617274652E630000790549D0
:1098700000EBC00001EB80004069002800D001200F
:1098800070470000401200202DE9F047044600799F
:10989000274900EBC00001EB800720684FF000096A
:1098A000C0F80095786880B120682249C0F8081394
:1098B00020680121000B40B200F01F0291404009D6
:1098C000800000F1E020C0F880112068D0F80C255D
:1098D000D0F81485D0F80865D0F810554FF0FF3156
:1098E000C0F80C15C0F814152068C0F80815C0F8A9
:1098F0001015501C02D01046FDF7C5FCB8F1FF3F13
:1099000002D04046FDF7BFFC681C02D02846FDF798
:10991000BAFC701C02D03046FDF7B5FC2068FFF79A
:10992000D7FB87F82090C7F80490BDE8F0870000C7
:10993000401200201003020010B5124C606898B16C
:10994000606840694068042808D360680421406961
:10995000008801EB00400CA1FEF75AF8606800F0A7
:1099600069FC0020606010BD0A4841680229FAD3F2
:109970000088022101EB0040BDE8104006A1FEF77F
:1099800047B8000060010020436F6D706172652070
:1099900045565400FC030020436F6D7061726520D2
:1099A0006576656E7420627574206E6F20616374D5
:1099B0006976652074696D65722028616C726561D5
:1099C00064792073746F707065643F290000000033
:1099D00070B516484168042906D30088042101EBBC
:1099E000004013A1FEF714F81548416829B14168F9
:1099F0004968406821F07F41416000F0CFFA0400DF
:109A000013D04FF080756068A84203D2204600F062
:109A100011FC03E0606820F07F4060602046FFF7A3
:109A2000CBF8002801D00446EDE770BDFC03002010
:109A30004F766572666C6F772045565400000000C3
:109A4000600100202DE9F84317460C0005462BD095
:109A5000DFF870804646D8F80000F8F71BFD384460
:109A600087B23068F8F716FDA968498A081AB0FB72
:109A7000F7F086B22046F8F70DFDA968381A87B2CC
:109A8000088BB0FBF6F206FB1202401C088382B181
:109A900023460DA207212846FCF7F0FB394628464D
:109AA000BDE8F843FAF752B9A96800200883BDE879
:109AB000F883009405A207212846D8F80030FCF767
:109AC000DDFBEBE700020020257300000D0A257383
:109AD0002573000010B50C46017A052908D0407A9C
:109AE00038B1084808A102682046FDF719F800E0DF
:109AF0001AB106A12046FDF713F82046BDE8104034
:109B0000FDF74EB890020020257300000D0A0000FA
:109B100038B5C3880D46044633B116A0009017A28D
:109B200018A12846FCF7FCFF217A052920D0607A8D
:109B300048B1A088FDF72AFE184951F8202018A145
:109B40002846FCF7EDFF2846216800F0E5FCA088D8
:109B50000021FEF78BF803461049207A143951F89A
:109B6000202001B02846BDE830400EA1FCF7D8BF48
:109B700038BD00001B5B306D000000001B5B313BFB
:109B800033316D0025734C6F67732064726F707092
:109B90006564202825642925730D0A0090020020A1
:109BA000257300003C25733E2025733A20000000F9
:109BB000EFF30580C005C00D01D001207047EFF321
:109BC000148040F30000401C7047000003498842A5
:109BD00001D103487047002070470000002000407A
:109BE0005801002008B500226946FEF7FBFB00285B
:109BF00006D104488169491C81610098FEF713F978
:109C000008BD00000C02002001680A684968914202
:109C100001D3881A70478068801A0844401C704736
:109C20002DE9F0479246894604004BD02078212840
:109C300005D05E2803D000270126002035E001274B
:109C4000641CF9E700262F2D02D05C2D04D00CE017
:109C50004FF0FF30BDE8F0875FEACA7006D114F814
:109C6000010B5146FAF7C7FCC5B25DB320782D2829
:109C70002AD160785146FAF7BEFC10F0FF0023D0DD
:109C80005D2821D0A41C5C280AD15FEACA7107D1E3
:109C900014F8010B5146FAF7AEFC10F0FF00D9D0D2
:109CA0004D4503DC814501DC0120804614F8010BA1
:109CB0005146FAF7A0FCC5B25D2DC3D1002EC1D12B
:109CC000B84504D10020C5E74D45EFD1ECE720466B
:109CD000C0E710B510461A46F6F704FC002010BD88
:109CE0000846704710B50446FAF739F908B1FFF78E
:109CF0006FFE00212046FAF74BF808B1FFF71CFE73
:109D0000204600F031FB2046BDE81040AFF3008054
:109D10002DE9F047334C814600264FF0040800BF80
:109D200000F03CF9002854D04768606840686168DA
:109D3000C1B1616800294AD0B84248D96068007E44
:109D400080B1606840694068042807D36068406952
:109D5000018808EB014024A1FDF75AFE61682748FD
:109D6000FEF7EEFE00F020F905464069416804293F
:109D700006D301883A4608EB014021A1FDF74CFECD
:109D80006A6818484FF47A7300210830FAF708F926
:109D900080B10D2811D021499C20F7F765FC686936
:109DA00041680429BCD3018808EB01401CA1FDF7E0
:109DB0002FFEB5E7606820B106E0284600F03AFAC9
:109DC000EDE74846FAF7D0F86560002EA8D1BDE867
:109DD000F08760680028FAD14846BDE8F047FAF7F6
:109DE000D1B800006001002054696D657220707266
:109DF00065656D707465642E0000000070AD000034
:109E000041637469766174696E672074696D657207
:109E1000202843433A2564292E000000D4BB0000CB
:109E200054696D6572206578706972656420626539
:109E3000666F7265207363686564756C6564207411
:109E40006F205254432E000070B5054688690C46B9
:109E500000284FF4847128460AD0FEF796FFD5F803
:109E60001805626AE1688854606A401C606270BDCF
:109E7000FEF78BFFD5F8180570BD1FB501238DF8CF
:109E80000030CDE90121D0E90012684690471FBD9E
:109E90001FB501238DF800308DF808100192D0E92C
:109EA0000012684690471FBD10B5044600684FF485
:109EB0009271FEF76AFF4FF484712068FEF765FF28
:109EC00020680121016010BD7CB50546FF2000908F
:109ED00001236A4601A9E868FEF7DEFC040004D00D
:109EE00010A11A20F7F7C0FB19E0009ABAB168690F
:109EF0001C4C01990378D2B2E35C1BB1001DFFF743
:109F000077FB02E00C30FFF775F9040007D1A86871
:109F10002A4640F6CD410068F7F78CFA0446204601
:109F20007CBD00002E2E5C2E2E5C2E2E5C2E2E5C18
:109F30002E2E5C2E2E5C636F6D706F6E656E74736B
:109F40005C6C69627261726965735C636C695C7593
:109F50006172745C6E72665F636C695F7561727466
:109F60002E63000034010020342800D93420C01CA6
:109F700020F00300704700000022CA604A60054AD2
:109F80008A60052803D2044A52F8200000E000202D
:109F900008607047CCB20000580200200148FEF76C
:109FA00035BE000070AD00000148FEF759BE00004C
:109FB00070AD00002DE9F04107460025F8F76AFA78
:109FC00086B2002F25D0002420E000BFF6F732FA39
:109FD0000168385D085CC00716D0601C06E03A5C7A
:109FE0008A5CD20706D06D1CADB2401C80B2B04274
:109FF000F5D309E045B13918751B38196A1C401CA6
:10A00000F6F770FAAEB20025641CA4B2701E84424A
:10A01000DCDBBDE8F08100002DE9F84FDFF8B0800F
:10A020009246894606461F46012269461846D8F8D8
:10A030000850F7F725FBE8B3009800210446C01C40
:10A040000AE000BF00EA05025AF821C008EB8202CC
:10A05000401C491CC2F80CC0B942F3D3BA46370CB5
:10A06000F9F78CFE8346FDF7AFFDB84204D81949D5
:10A0700040F28310F7F7F8FA601C284008EB8000E4
:10A0800047EA0B41C160D8F80C0447468047A11C41
:10A09000294007EB81012C40C86007EB8401C868A8
:10A0A00066F3C5006AF3891069F39F2020F003006E
:10A0B000401C00E002E020F00400C86098F8200492
:10A0C00002E000BFFDF77AFB0028FBD1BDE8F88F66
:10A0D0004C1500203CCC000070B50C46050003D1A7
:10A0E00007A15420F7F7C0FA1CB905A15520F7F7CE
:10A0F000BBFA21462846BDE87040F6F748BA000092
:10A100002E2E5C2E2E5C2E2E5C64656D6F5F636C54
:10A11000695F636D64732E630000000070B50C46C8
:10A12000050004D108A140F61410F7F79DFA24B9F0
:10A1300005A140F61510F7F797FA21682868BDE8E1
:10A140007040F6F724BA00002E2E5C2E2E5C2E2EC8
:10A150005C2E2E5C2E2E5C2E2E5C636F6D706F6EEF
:10A16000656E74735C6C69627261726965735C635D
:10A170006C695C6E72665F636C692E630000000040
:10A180002DE9F04114460D00064604D11BA140F212
:10A190007A20F7F769FA24B918A140F27B20F7F783
:10A1A00063FA3046F9F702FD78B9B068FA210789F9
:10A1B000B0F80C803046F9F7C9FDFA213046F9F7BE
:10A1C00041FC3046F9F7F2FC10B10620BDE8F08101
:10A1D000B06800892880B068808920802888C01BEA
:10A1E00081B23046F9F7A0FC2188A1EB080081B2CA
:10A1F0003046F9F7B7FD0020E8E700002E2E5C2E70
:10A200002E5C2E2E5C2E2E5C2E2E5C2E2E5C636F12
:10A210006D706F6E656E74735C6C69627261726989
:10A2200065735C636C695C6E72665F636C692E63F8
:10A230000000000070B50446C06818B90F496120DD
:10A24000F7F712FA0E4800250078A0B19CB1207EE5
:10A2500088B1D4E903108847A06850B1217E41B18C
:10A2600061680844606021460648FEF769FC0125E4
:10A2700001E000202076284670BD0000D4BB00001D
:10A280006001002070AD00000948007800280ED061
:10A2900008480268521C026007484168032906D337
:10A2A0000088052101EB004004A1FDF7B5BB704714
:10A2B000000000200400002074040020636F756E0D
:10A2C000746572203D2025640D0A000010B5044617
:10A2D0000020F6F70DFC20B16068D0E900210020D5
:10A2E00090476068D0E9002101209047A06822468D
:10A2F00040F6CD410068F7F79DF8002805D0BDE88D
:10A30000104002A11B20F7F7AFB910BD2E2E5C2E16
:10A310002E5C2E2E5C2E2E5C2E2E5C2E2E5C636F01
:10A320006D706F6E656E74735C6C69627261726978
:10A3300065735C636C695C7274745C6E72665F6397
:10A340006C695F7274742E63000000004069054AF6
:10A350000178515C11B1001DFFF706BA0C30FEF711
:10A36000F1BF0000340100202DE9F84F374D83463E
:10A3700069462868FBF7CEF904464FF00408002729
:10A380004FF00109324EDFF8CCA05BE0207820B11D
:10A39000012828D002284CD138E06068017E0029CD
:10A3A00047D180F818905846F9F7F9FC01466068E3
:10A3B0004268511A284A914203D9416821F07F41ED
:10A3C0004160224861680830FEF7BAFB616848695D
:10A3D0004268042A2DD34A68018808EB01401FA176
:10A3E000FDF71AFB25E061687068814200D1776053
:10A3F00016480830FEF762FC60684069416804292D
:10A4000017D3018808EB01401AA110E0FFF7CCFD3B
:10A4100008B10776FAE786F80090DAF80410032905
:10A4200007D3BAF80000032101EB004015A1FDF7A6
:10A43000EFFA69462868FBF762F969462868FBF776
:10A4400069F90446002CA1D1BDE8F88F68AD000081
:10A4500060010020FC03002017FCFF0053746172B0
:10A46000742072657175657374202843433A2564BE
:10A47000292E000053746F702072657175657374B6
:10A480002E00000053746F7020616C6C2072657137
:10A49000756573742E000000F8B5114C0D46064624
:10A4A00069462068FBF720F9B8B106704560694637
:10A4B0002068FBF73AF918B10A48F9F73FFD0AE0BE
:10A4C00009484168022906D30088022101EB0040B7
:10A4D00006A1FDF79DFA0020F8BD0420F8BD00009C
:10A4E00068AD000068010020FC030020536368652C
:10A4F00064756C696E6720696E74657272757074CC
:10A50000656420616E6F746865722073636865644A
:10A51000756C696E672E0000FEB51A4A6FF0E00593
:10A520005368B1FBF3F411684FF46162B4FBF1F3CB
:10A53000B3FBF2F2554303EB05153C23B5FBF3F3F4
:10A54000A3EB031605EB8606B4FBF1F501FB1544FE
:10A550004FF47A756543B5FBF1F504EB440C05FB4C
:10A5600001F7CCEBC414C7EBC4044FF47A777C43F7
:10A57000B4FBF1F10096CDE9015103A1FCF7D0FA4B
:10A58000FEBD0000740200205B253032643A2530A5
:10A5900032643A253032642E253033642C25303332
:10A5A000645D200070B50C4605464FF48E71FEF7D1
:10A5B000ECFB216AA068415C206A401C2062C5F85F
:10A5C0001C1570BD1FB500228DF800200291816816
:10A5D00001914261D0E90012684690471FBD00001A
:10A5E0007CB5FF260546009600780C46002835D03D
:10A5F000012819D0022802D02CA1652011E0297A67
:10A60000E068FEF785FA28B1042803D027A1392095
:10A61000F7F72AF82046FFF757FC002803D023A1BC
:10A620003B20F7F721F87CBD297AE068FEF770FA45
:10A6300028B1042803D01DA14120F7F715F8287A86
:10A6400020B16068D0E90021002090472046FFF744
:10A650003BFC0028E7D015A14D20E2E7297A2069CC
:10A66000FEF7F0F918B111A15320F6F7FDFF00969F
:10A6700001236A4601A92069FEF7F8F918B10BA178
:10A680005620F6F7F1FF009848B1C2B2606901990F
:10A69000FCF72AFA18B105A15B20F6F7E5FF606820
:10A6A000D0E90021012090477CBD00002E2E5C2EB9
:10A6B0002E5C2E2E5C2E2E5C2E2E5C2E2E5C636F5E
:10A6C0006D706F6E656E74735C6C696272617269D5
:10A6D00065735C636C695C756172745C6E72665FF5
:10A6E000636C695F756172742E6300001FB50A4662
:10A6F00001788DF8001041680191017A8DF80810F9
:10A70000C0680390044850F82210001F50F822201F
:10A71000684690471FBD00003C0100202DE9FF471F
:10A720000C4605464FF40071FEF735FB01274FF448
:10A730000178002618B34FF4927949462846FEF76F
:10A740001FFBE0B149462846FEF71FFBC5F808830A
:10A7500094F8290000B96F6002208DF80000D5F848
:10A760008004C5F880040390A0690290E06801901D
:10A77000A661E661D4E900126846904728E004210A
:10A780002846FEF708FB18B34FF484712846FEF7FD
:10A79000F7FAE8B121462846FFF756FB616AA0693F
:10A7A000884215D1E06938B1E268616AA061206928
:10A7B000E6616662E06008E094F8290000B96F6025
:10A7C000C5F80883A661E268616A2046FFF755FB79
:10A7D0004FF48E7841462846FEF7D2FA78B1206AC7
:10A7E0006169884202D294F8280020B34146284685
:10A7F000FEF7CBFA616911B12046FFF7E3FE4FF493
:10A80000A27841462846FEF7BBFA002818D04146F8
:10A810002846FEF7BAFA94F8290000B12F60A06923
:10A8200000280DD0A661E268616A04B02046BDE848
:10A83000F047FFF722BB21462846FFF7B3FEDEE7CD
:10A84000BDE8FF871FB50A4601788DF80010416802
:10A850000191017A8DF80810C0680390044850F8FF
:10A860002210001F50F82220684690471FBD0000AC
:10A870003C0100202DE9FF410C464FF4927705463C
:10A880003946FEF78EFA0026C0B139462846FEF753
:10A890008DFA02208DF80000D5F88004C5F88004F8
:10A8A0000390D5F83C058DF80800E0680190A6619A
:10A8B000E661D4E900126846904723E04FF48877B8
:10A8C00039462846FEF76DFAE0B139462846FEF7CC
:10A8D0006DFAD5F83C15A069884213D1E06960B1E2
:10A8E000E268D5F8000220F02000C5F80002E06917
:10A8F000A0612069E661E06001E0A661E2682046AF
:10A90000FFF7C6FA4FF4A27739462846FEF749FA10
:10A9100060B139462846FEF749FAA06930B1A66110
:10A92000D5F83C152046E268FFF7B2FA4FF490776D
:10A9300039462846FEF735FA002813D0394628460E
:10A94000FEF734FA606900280CD0D5F84C058DF874
:10A9500000608DF80800A06801906661D4E90012DB
:10A9600068469047BDE8FF8110B50248FAF7E8FE57
:10A97000002010BD080200202DE9F05F8346DDE9CC
:10A980000A4A994690460D460846012703E000BF53
:10A99000B0FBF8F07F1C4045FAD2B94500D94F46CC
:10A9A0005FEACA7012D18CB15FEA8A7002D5B9F140
:10A9B000000F01D0202607E0302605E0314658463A
:10A9C000641EF6F7A1FE0CB1A742F7D35FF00106B3
:10A9D000B9F1010F02D9A9F1010903E0B5FBF6F0C5
:10A9E000404502D306FB08F6F2E7DFF83C9000BFD3
:10A9F000B5FBF6F000FB165519F800105846F6F7AF
:10AA000083FEB6FBF8F6002EF2D15FEACA7009D0D9
:10AA1000002C07D0A74205D220215846641EF6F725
:10AA200073FEF5E7BDE8F09F2CB000001CB50029CF
:10AA300013D08268D27D8A420FD008A3D3E90023C5
:10AA4000CDE9002301F12F028DF803208268D17532
:10AA500000696A4603A1FCF763F81CBD1B5B340068
:10AA60006D000000257300001CB5826899B1927DCD
:10AA70008A420FD00CA2D2E90032CDE9003201F1B6
:10AA80002F028DF805208268917500696A4608A139
:10AA9000FCF746F81CBD9175006902B0054ABDE897
:10AAA000104003A1FCF73CB81B5B313B33006D0049
:10AAB00025730000C0AF000010B50446F7F7EAFCAC
:10AAC000002105E0625C3F2A06D02A2A04D0491CF6
:10AAD0008142F7D3002010BD012010BD0020704737
:10AAE0002DE9FC4180461C4617460E460C48089D41
:10AAF000FAF72FFE10B11120BDE8FC81A2083946FB
:10AB00003046FDF741FC0648FAF71AFE33463A464E
:10AB100001214046CDE90045F9F780FB0020EBE735
:10AB20000802002000B40000DCB3000000000000B8
:10AB3000A5350000000000003CAB00004CB4000054
:10AB40002CB4000000000000CD36000050B400001E
:10AB500008B40000000000000937000000000000F9
:10AB600000000000000000000000000058B40000D9
:10AB700058B4000034AB00001136000060B400008F
:10AB800060B4000000000000413700000000000039
:10AB900094AB0000B8B4000080B4000000000000D6
:10ABA000B92C0000C0B4000098B400000000000000
:10ABB000F12C0000B0B4000068B4000000000000F8
:10ABC000292D00000000000000000000000000002F
:10ABD00000000000ECB40000C8B400008CAB000022
:10ABE000AD2B000001000000E94000000000000063
:10ABF000F4AB000044B600001CB5000000000000EB
:10AC0000D52D000048B60000F4B40000E4AB00000D
:10AC1000712F000050B6000008B50000E4AB000042
:10AC20003D30000058B6000020B6000000000000D3
:10AC300031310000000000000000000000000000B2
:10AC40000000000084B6000060B60000ECAB00001D
:10AC5000612D0000C4BA0000C0BA0000A4BA000010
:10AC600020000020CCBA0000ECAC0000C00700209F
:10AC70007000002058000020E0D200000D0000000D
:10AC8000DCBA000008AD0000B80C0020BC000020B9
:10AC9000A4000020FCD200000A000000FFFFFFFF1C
:10ACA000FFFFFFFFFFFFFFFFFFFFFFFF00000000B0
:10ACB000000000000000D601070100003C00002059
:10ACC000140700203F000000540700206C070020FC
:10ACD0000F0000007C070020000000000020004062
:10ACE00000000000002000400000000018B000003C
:10ACF00094070020BCAC0000CCAC0000C0AC00004D
:10AD0000D8AC000088000020F8AF0000AC0C002098
:10AD100004AD0000000000001CAD000028BB0000D6
:10AD20000CBB0000000000005D7E000020BB0000A6
:10AD3000E8BA000000000000597F00000000000099
:10AD40000000000000000000000000004CBB0000FC
:10AD500030BB000014AD00003D8100000000005039
:10AD60002D910000319500007001002000000700C7
:10AD700000000000840100205D390000B8B400002C
:10AD80001CBC00000000000059370000B0C00000EB
:10AD90002CBC0000000000001532000054BC000074
:10ADA0003CBC000000000000392B00000000000047
:10ADB000B4AD0000B0C000008CBC0000000000007A
:10ADC0005533000060BC000068BC000000000000BB
:10ADD00079340000000000000000000000000000C6
:10ADE00000000000B0BC0000B8BC0000ACAD00002A
:10ADF0000000000000000000000000000000000053
:10AE00000338FDD8704700000000000010AE0000BD
:10AE100064C2000040C2000000000000AD59000004
:10AE20000000000000000000000000000000000022
:10AE30006CC2000074C2000008AE0000AD590000F2
:10AE4000597500003D7500002175000000000000EC
:10AE500054AE000054C300003CC3000000000000DA
:10AE6000B15E000058C3000024C3000000000000D1
:10AE7000DB5E000000000000000000000000000099
:10AE800000000000000000008CAE000054C3000071
:10AE90005CC30000000000009D5F000058C300007C
:10AEA000B8C3000000000000C75F00000000000001
:10AEB0000000000000000000000000000000000092
:10AEC000C4AE0000B8B40000F8C3000000000000E9
:10AED0002D5D000058B60000CCC30000000000004B
:10AEE0005D5D0000000000000000000000000000A8
:10AEF0000000000000000000FCAE000068C400007C
:10AF000048C400004CAE0000E95D000060C40000D1
:10AF100024C4000084AE0000055F000070C400007F
:10AF200038C40000BCAE0000C15C0000000000009E
:10AF30000000000000000000000000000000000011
:10AF400044AF0000BCC4000078C400000000000052
:10AF5000F16100000000000000000000000000009F
:10AF600000000000D4C40000C4C4000000000000C1
:10AF70003D5B000000C50000DCC40000F4AE000032
:10AF8000115C000018C5000004C5000000000000AE
:10AF9000F15F0000C0C5000020C500003CAF00000C
:10AFA000CD60000000000000000000000000000074
:10AFB0001B37001B38001B45002C20001B5B4A0080
:10AFC0001B5B6D00082008001B5B4B00202D200040
:10AFD0001B5B48001B5B366E001B5B324A000000A7
:10AFE0000338FDD870471B5B3F336C002D682C2065
:10AFF0002D2D68656C70000025210000AD2100003A
:10B00000CD200000B5210000492100000000000013
:10B010000338FDD870470000A5280000592900001A
:10B020003928000071290000F12800003031323346
:10B030003435363738394142434445466E72665F8F
:10B040006673746F726167655F696E6974006E72B2
:10B05000665F6673746F726167655F756E696E694E
:10B0600074006E72665F6673746F726167655F729B
:10B07000656164006E72665F6673746F72616765A6
:10B080005F7772697465006E72665F6673746F7263
:10B090006167655F65726173650000000010000004
:10B0A0000400000001000000554A000069A90000EA
:10B0B000D39C0000E1AA0000D5410000E19C000003
:10B0C000DDAA0000C94C000000000000D0B0000064
:10B0D00064C20000B4C60000000000004D870000FC
:10B0E0000000000000000000000000000000000060
:10B0F000D8C6000074C20000C8B000004D87000030
:10B10000556E6B6E6F776E206572726F7220636F13
:10B1100064650000000000000CCB0000010000008E
:10B12000CCC9000002000000C0C7000003000000FE
:10B1300040CA00000400000094CA0000050000009E
:10B1400074C900000600000010C9000007000000DC
:10B150007CCA00000800000088C900000900000047
:10B16000ECC900000A000000F4CA00000B00000057
:10B17000A8C700000C000000A0C900000D000000DE
:10B1800044CB00000E0000006CCA00000F0000005D
:10B19000A8CA000010000000DCCA00001100000076
:10B1A00058CB00008000000028C90000810000008A
:10B1B00064C800008200000024C800008300000072
:10B1C00004C800008400000040C8000085000000A2
:10B1D0004CC900008600000054CA00009000000026
:10B1E000F0C8000091000000E4C7000092000000D9
:10B1F000B4C9000000820000BCCA00000182000047
:10B2000008CA00000282000024CA00000084000076
:10B2100080C800000184000018CB000002840000F8
:10B22000C8C8000003840000A4C800002D2D2D2DE7
:10B230002D2D2D2D2D2D2D43524153484C4F472D53
:10B240002D2D2D2D2D2D2D2D2D2D2D0D0A000000F8
:10B250002900000000000000000000004D77000001
:10B26000497700003D77000031760000B975000095
:10B27000AD750000000000007CB20000D4C40000E6
:10B2800084CB000000000000A942000068CB000051
:10B2900070CB0000000000002543000064C20000E5
:10B2A00090CB00000000000085430000000000007B
:10B2B000000000000000000000000000A4CB00001F
:10B2C000B0CB000074B200000000000001000000DC
:10B2D000E155000001000000799F0000000000001F
:10B2E000E4B2000094CD000020CD0000CCB20000FC
:10B2F000494D00008CCD00009CCC0000D4B2000071
:10B30000494D0000BCCD00009CCD000000000000B5
:10B31000214F0000D0CD0000ACCD000000000000A7
:10B32000294F000064C20000C0CD000000000000F2
:10B330007950000000000000000000000000000044
:10B3400000000000D8CD0000DCCD0000DCB2000021
:10B35000F14C0000004040404040404040404141EE
:10B3600041414140404040404040404040404040DA
:10B370004040404040050202020202020202020274
:10B380000202020202202020202020202020200271
:10B390000202020202029090909090901010101001
:10B3A000101010101010101010101010101010109D
:10B3B0000202020202028888888888880808080831
:10B3C00008080808080808080808080808080808FD
:10B3D000020202024000000055B300005072696E84
:10B3E00074204E6F726469632053656D69636F6E7C
:10B3F000647563746F72206C6F676F2E00000000BD
:10B400006E6F7264696300005072696E74206561CA
:10B41000636820706172616D6574657220696E2069
:10B420006E6577206C696E652E0000005072696E43
:10B430007420616C6C20656E746572656420706147
:10B4400072616D65746572732E000000616C6C0032
:10B45000706172616D0000007072696E74000000AE
:10B46000707974686F6E000053746F702073656339
:10B470006F6E647320636F756E7465722E000000CA
:10B480005265736574207365636F6E647320636FB8
:10B49000756E7465722E000053746172742073654A
:10B4A000636F6E647320636F756E7465722E000037
:10B4B00073746F70000000007265736574000000A3
:10B4C0007374617274000000446973706C61792058
:10B4D0007365636F6E6473206F6E207465726D693F
:10B4E0006E616C2073637265656E0000636F756ECC
:10B4F0007465720045786563757465206120636FBB
:10B500006D6D616E642E000052656D6F7665206111
:10B5100020636F6D6D616E642E00000041646420D5
:10B5200061206E65772064796E616D696320636F59
:10B530006D6D616E642E0A4578616D706C65207565
:10B54000736167653A205B2064796E616D69632081
:10B550006164642074657374205D2077696C6C206D
:10B5600061646420612064796E616D696320636F3A
:10B570006D6D616E64202774657374272E0A496EA1
:10B580002074686973206578616D706C652C206328
:10B590006F6D6D616E64206E616D65206C656E67A8
:10B5A0007468206973206C696D6974656420746FB8
:10B5B0002033322063686172732E20596F752063C7
:10B5C000616E2061646420757020746F20323020B9
:10B5D000636F6D6D616E64732E20436F6D6D616E70
:10B5E000647320617265206175746F6D6174696345
:10B5F000616C6C7920736F7274656420746F206560
:10B600006E7375726520636F727265637420434C4C
:10B610004920636F6D706C6574696F6E2E00000059
:10B6200053686F7720616C6C20616464656420648A
:10B63000796E616D696320636F6D6D616E64732EE9
:10B6400000000000616464006578656375746500DE
:10B6500072656D6F7665000073686F77000000009B
:10B6600044656D6F6E7374726174652064796E6188
:10B670006D696320636F6D6D616E642075736167C2
:10B68000652E000064796E616D6963000D0A2020EB
:10B69000202020202020202020202E636F3A2E20E2
:10B6A000202020202020202020202020202020209A
:10B6B000202027786F2C20202020202020202020D0
:10B6C0000D0A2020202020202020202E2C636F6CAB
:10B6D0006C6C6C632C2E2020202020202020202029
:10B6E00020202027636B4F4F6F3A3A2C2E2E2020BC
:10B6F000202020200D0A2020202020202E3A6F6FAD
:10B700006F6F6F6C6C6C6C6C6C6C6C3A272E2020BD
:10B710002020202E3B644F4F4F4F4F4F6F3A3A3A05
:10B720003B3B3B272E2020200D0A202020276F6B3B
:10B730007864646F6F6F6F6C6C6C6C6C6C6C6C6C41
:10B740006C6C6C3B27636B4F4F4F4F4F4F4F4F4FBE
:10B750006F3A3A3A3B3B3B2C2C2C27200D0A2020F9
:10B76000204F4F4F6B78646F6F6F6F6C6C6C6C6CAD
:10B770006C6C6C6C6C6C6C6C6C6C6C64784F4F4F5C
:10B780004F4F4F4F6F3A3A3A3B3B3B2C2C2C272ED6
:10B790000D0A2020204F4F4F4F4F4F6B646F6F6C3F
:10B7A0006C6C6C6C6C6C6C6C6C6C6C6C6C6C6C6CD9
:10B7B0006C6C6C64784F4F4F6F3A3A3A3B3B3B2C82
:10B7C0002C2C272E0D0A2020204F4F4F4F4F4F4F2C
:10B7D0004F4F6B786F6C6C6C6C6C6C6C6C6C6C6CD5
:10B7E0006C6C6C6C6C6C6C6363636C646C3A3A3A52
:10B7F0003B3B3B2C2C2C272E0D0A2020204F4F4F5B
:10B800004F4F4F4F4F4F4F4F4F4F78646F6C6C6C93
:10B810006C6C6C6C6C6C6C6C6C6C6C636363636395
:10B820003A3A3A3A3B3B3B2C2C2C272E0D0A20204F
:10B83000204F4F4F4F4F4F4F4F4F4F4F4F4F4F4F47
:10B840004F6B78646C6C6C6C6C6C6C6C6C6C6C635B
:10B85000636363633A3A3A3A3B3B3B2C2C2C272EEA
:10B860000D0A2020206B4F4F4F4F4F4F4F4F4F4FE0
:10B870004F4F4F4F4F4F4F4F4F6B646F6C6C6C6C13
:10B880006C6C6C63636363633A3A3A3A3B3B3B2CC0
:10B890002C2C272E0D0A2020206B4F4F4F4F4F4F3F
:10B8A0004F4F4F4F4F4F4F4F4F4F4F4F4F4F4F4FA8
:10B8B0004F78646C6C6C6C63636363633A3A3A3AD6
:10B8C0003B3B3B2C2C2C272E0D0A2020206B4F4F6E
:10B8D0004F4F4F4F4F4F4F4F4F4F4F4F4F4F4F4F78
:10B8E0004F4F4F4F4F4F4F4F6B786F6C6363636396
:10B8F0003A3A3A3A3B3B3B2C2C2C272E0D0A20207F
:10B90000206B4F4F4F4F4F4F4F4F4F4F4F4F4F4F5A
:10B910004F4F4F4F4F4F4F4F4F4F4F4F4F4F4F4F37
:10B920006B646C633A3A3A3A3B3B3B2C2C2C272E07
:10B930000D0A202020784F4F4F4F4F4F4F4F4F4F02
:10B940004F78646B4F4F4F4F4F4F4F4F4F4F4F4FAD
:10B950004F4F4F4F4F4F4F4F786F633A3B3B3B2C0E
:10B960002C2C272E0D0A202020784F4F4F4F4F4F61
:10B970004F4F4F4F4F64633A3A6C646B4F4F4F4F8A
:10B980004F4F4F4F4F4F4F4F4F4F4F4F4F4F4F6BAB
:10B9900064633B2C2C2C27270D0A202020784F4F46
:10B9A0004F4F4F4F4F4F4F4F4F64633A3A3B3B2CF3
:10B9B0003B63646B4F4F4F4F4F4F4F4F4F4F4F4F66
:10B9C0004F4F4F4F4F4F4F786C3B27270D0A20208A
:10B9D000202E6C6B4F4F4F4F4F4F4F4F4F64633A7A
:10B9E0003A3B3B2C2C27272E2E3B6F4F4F4F4F4F70
:10B9F0004F4F4F4F4F4F4F4F4F4F4F4F4F4F782756
:10BA00000D0A2020202020202E3B6F4F4F4F4F4FFC
:10BA10004F64633A3A3B3B2C2E20202020202020EC
:10BA20002E3A784F4F4F4F4F4F4F4F4F4F4F4F641E
:10BA30003B2E20200D0A2020202020202020202006
:10BA40002E3A784F4F64633A2C2E2020202020205D
:10BA5000202020202020202027636B4F4F4F4F6B4A
:10BA60006C272020202020200D0A202020202020AC
:10BA7000202020202020202E6F642720202020201E
:10BA800020202020202020202020202020202027AF
:10BA9000786B2C2020202020202020200D0A0D0A49
:10BAA0000000000064756D6D79206F7074696F6EB1
:10BAB0002068656C7020737472696E670000000006
:10BAC0002D7400002D2D74657374000075617274FF
:10BAD0005F636C693A7E2420000000007274745F1A
:10BAE000636C693A7E2420005072696E7420696E1E
:10BAF000666F726D6174696F6E2061626F7574201C
:10BB00004D50552073746174652E000044756D703E
:10BB1000204D5055207265676973746572732E00ED
:10BB2000696E666F0000000064756D7000000000B3
:10BB3000436F6D6D616E647320666F72204D50555A
:10BB4000206D616E6167656D656E74006D70750066
:10BB50002D2D2F2D2D000000574257412F2D2D0048
:10BB600057422F2D2D00000057542F2D2D0000007F
:10BB70002D2D2F5742574100574257412F574257BB
:10BB80004100000057422F574257410057542F574A
:10BB9000425741002D2D2F57420000005742574178
:10BBA0002F57420057422F574200000057542F573B
:10BBB000420000002D2D2F575400000057425741DE
:10BBC0002F57540057422F575400000057542F57F7
:10BBD000540000002E2E5C2E2E5C2E2E5C2E2E5C31
:10BBE0002E2E5C2E2E5C636F6D706F6E656E74739F
:10BBF0005C6C69627261726965735C74696D6572AF
:10BC00005C6578706572696D656E74616C5C61709D
:10BC1000705F74696D6572322E63000053797374BE
:10BC2000656D2072657365742E000000547269673B
:10BC3000676572206572726F722E00005072696EB5
:10BC400074206170706C69636174696F6E207369D0
:10BC50007A652E006170705F73697A65000000007C
:10BC60007761726E696E67005761726E696E6720E8
:10BC70006C6F67206D6573736167652077697468A1
:10BC800020706172616D6574657273004572726FC8
:10BC900072206C6F67206D657373616765207769CB
:10BCA000746820706172616D657465727300000064
:10BCB0006C6F675F6D7367005472696767657220A8
:10BCC0006C6F67206D657373616765207769746851
:10BCD00020646563696D616C20617267756D656E66
:10BCE000747300002E2E5C2E2E5C2E2E5C2E2E5C8D
:10BCF0002E2E5C2E2E5C636F6D706F6E656E74738E
:10BD00005C6C69627261726965735C74696D65729D
:10BD10005C6578706572696D656E74616C5C647287
:10BD2000765F7274632E6300446174612062757380
:10BD3000206572726F72202872657475726E206150
:10BD400064647265737320696E207468652073740F
:10BD500061636B206672616D65206973206E6F741C
:10BD60002072656C6174656420746F20746865204E
:10BD7000696E737472756374696F6E207468617430
:10BD80002063617573656420746865206572726FE5
:10BD900072290000446174612062757320657272BB
:10BDA0006F72202850432076616C75652073746132
:10BDB000636B656420666F722074686520657863C4
:10BDC000657074696F6E2072657475726E20706F25
:10BDD000696E747320746F2074686520696E737463
:10BDE00072756374696F6E20746861742063617525
:10BDF00073656420746865206661756C7429000041
:10BE000043617573653A204275734661756C7420A1
:10BE10006F6E206120766563746F72207461626C4E
:10BE200065207265616420647572696E672065784B
:10BE300063657074696F6E2070726F636573736988
:10BE40006E672E005468652070726F636573736F40
:10BE5000722068617320657865637574656420611C
:10BE60006E2053444956206F72205544495620692C
:10BE70006E737472756374696F6E2077697468206D
:10BE8000612064697669736F72206F6620300000EC
:10BE90005468652070726F636573736F7220686198
:10BEA0007320617474656D7074656420746F2065AF
:10BEB00078656375746520616E20696E7374727540
:10BEC0006374696F6E2074686174206D616B657353
:10BED00020696C6C6567616C20757365206F6620E6
:10BEE0007468652045505352000000005468652076
:10BEF00070726F636573736F722068617320617411
:10BF000074656D7074656420616E20696C6C656722
:10BF1000616C206C6F6164206F66204558435F52EE
:10BF2000455455524E20746F207468652050432C40
:10BF3000206173206120726573756C74206F6620B8
:10BF4000616E20696E76616C696420636F6E7465E2
:10BF500078742C206F7220616E20696E76616C6936
:10BF600064204558435F52455455524E2076616CCB
:10BF7000756500005468652070726F636573736F38
:10BF80007220617474656D707465642061206C6FDB
:10BF90006164206F722073746F7265206174206118
:10BFA000206C6F636174696F6E20746861742064C3
:10BFB0006F6573206E6F74207065726D6974207484
:10BFC0006865206F7065726174696F6E00000000B3
:10BFD00041204D656D4D616E616765206661756CD0
:10BFE00074206F6363757272656420647572696E24
:10BFF0006720666C6F6174696E672D706F696E740F
:10C00000206C617A79207374617465207072657335
:10C010006572766174696F6E000000004120627580
:10C0200073206661756C74206F63637572726564EA
:10C0300020647572696E6720666C6F6174696E67E3
:10C040002D706F696E74206C617A792073746174DD
:10C050006520707265736572766174696F6E000039
:10C060005468652070726F636573736F72206861C6
:10C070007320617474656D7074656420746F2065DD
:10C0800078656375746520616E20756E6465666998
:10C090006E656420696E737472756374696F6E0087
:10C0A000496E737472756374696F6E206275732064
:10C0B0006572726F720000005468652070726F6361
:10C0C0006573736F722068617320617474656D703D
:10C0D00074656420746F20616363657373206120ED
:10C0E000636F70726F636573736F7200556E7374F4
:10C0F00061636B20666F7220616E20657863657086
:10C1000074696F6E2072657475726E206861732039
:10C11000636175736564206F6E65206F72206D6F4B
:10C120007265206163636573732076696F6C6174F7
:10C13000696F6E7300000000537461636B696E6712
:10C1400020666F7220616E20657863657074696F18
:10C150006E20656E747279206861732063617573F7
:10C160006564206F6E65206F72206D6F726520614F
:10C1700063636573732076696F6C6174696F6E7346
:10C18000000000005468652070726F636573736F00
:10C190007220686173206D61646520616E20756E28
:10C1A000616C69676E6564206D656D6F7279206181
:10C1B0006363657373000000556E737461636B2075
:10C1C000666F7220616E20657863657074696F6E4A
:10C1D0002072657475726E20686173206361757377
:10C1E0006564206F6E65206F72206D6F72652042EE
:10C1F00075734661756C747300000000537461635D
:10C200006B696E6720666F7220616E20657863656A
:10C210007074696F6E20656E747279206861732026
:10C22000636175736564206F6E65206F72206D6F3A
:10C230007265204275734661756C7473000000006E
:10C240005072696E7420737461747573206F662008
:10C2500062616C6C6F6320696E7374616E63657389
:10C260002E000000737461747573000062616C6C61
:10C270006F630000436F6D6D616E647320666F7253
:10C280002042414C4C4F43206D616E6167656D6586
:10C290006E74000025730D0A092D20456C656D65CF
:10C2A0006E742073697A653A092564202B20256411
:10C2B000206279746573206F6620646562756720FB
:10C2C000696E666F726D6174696F6E0D0A092D205B
:10C2D00055736167653A0925752525202825752040
:10C2E0006F7574206F6620257520656C656D656EB1
:10C2F0007473290D0A092D204D6178696D756D3AA9
:10C30000092575252520282575206F7574206F66F1
:10C3100020257520656C656D656E7473290D0A0D99
:10C320000A000000456E61626C6520636F6C6F727D
:10C3300065642073796E7461782E000044697361BE
:10C34000626C6520636F6C6F7265642073796E74C4
:10C3500061782E006F6666006F6E0000446973613D
:10C36000626C6520434C49206563686F2E204172E2
:10C37000726F777320616E6420627574746F6E7370
:10C380003A204261636B73706163652C2044656C75
:10C390006574652C20456E642C20486F6D652C20DB
:10C3A000496E7365727420617265206E6F742068C7
:10C3B000616E646C65642E00456E61626C6520433D
:10C3C0004C49206563686F2E0000000047657420AB
:10C3D000434C492073746174697374696373206694
:10C3E0006F7220746865204C6F67676572206D6F8F
:10C3F00064756C652E000000526573657420434CB3
:10C4000049207374617469737469637320666F7211
:10C4100020746865204C6F67676572206D6F647566
:10C420006C652E00546F67676C6520434C4920652E
:10C4300063686F2E00000000434C492073746174E0
:10C440006973746963732E00546F67676C6520634A
:10C450006F6C6F7265642073796E7461782E000062
:10C460006563686F00000000636F6C6F727300009B
:10C470007374617473000000417373756D652038C7
:10C48000302063686172732073637265656E207714
:10C490006964746820616E642073656E64207468DA
:10C4A00069732073657474696E6720746F20746893
:10C4B00065207465726D696E616C2E0064656661DD
:10C4C000756C7400436C6561722073637265656E90
:10C4D0002E000000636C6561720000005573656694
:10C4E000756C2C206E6F7420556E69782D6C696B9D
:10C4F0006520434C4920636F6D6D616E64732E003F
:10C50000636C6900436F6D6D616E6420686973745C
:10C510006F72792E00000000686973746F72790081
:10C52000436F6E736F6C65206765747320746572FA
:10C530006D696E616C2073637265656E2073697AD4
:10C5400065206F7220617373756D657320383020BC
:10C55000696E20636173652074686520726561642B
:10C560006F7574206661696C732E204974206D7537
:10C5700073742062652065786563757465642061F5
:10C58000667465722065616368207465726D696E9A
:10C59000616C207769647468206368616E676520E8
:10C5A000746F20656E7375726520636F7272656358
:10C5B00074207465787420646973706C61792E00DE
:10C5C000726573697A650000436F6D6D616E6420FA
:10C5D00062756666657220697320746F6F20736878
:10C5E0006F727420746F20657870616E6420616C66
:10C5F0006C20636F6D6D616E6473206D6174636830
:10C60000696E672077696C6463617264207061741D
:10C610007465726E0D0A000020200000616464726F
:10C620005F69735F77697468696E5F626F756E6466
:10C630007328705F66732C20706167655F61646446
:10C64000722C20286C656E202A20705F66732D3E48
:10C65000705F666C6173685F696E666F2D3E6572B0
:10C660006173655F756E6974292900002E2E5C2E3A
:10C670002E5C2E2E5C2E2E5C2E2E5C2E2E5C636F7E
:10C680006D706F6E656E74735C6C696272617269F5
:10C6900065735C6578706572696D656E74616C5FF9
:10C6A0006D656D6F626A5C6E72665F6D656D6F62FF
:10C6B0006A2E63005072696E7420737461747573AE
:10C6C000206F6620717565756520696E7374616E83
:10C6D0006365732E000000007175657565000000CC
:10C6E00025730D0A092D20456C656D656E742073E8
:10C6F000697A653A0925640D0A092D205573616729
:10C70000653A092575252520282575206F75742023
:10C710006F6620257520656C656D656E7473290DD7
:10C720000A092D204D6178696D756D3A09257525C9
:10C730002520282575206F7574206F6620257520AB
:10C74000656C656D656E7473290D0A092D204D6F3A
:10C7500064653A090925730D0A0D0A002E2E5C2E18
:10C760002E5C2E2E5C2E2E5C2E2E5C2E2E5C636F8D
:10C770006D706F6E656E74735C6C69627261726904
:10C7800065735C6578706572696D656E74616C5F08
:10C7900072696E676275665C6E72665F72696E67FB
:10C7A0006275662E630000004E52465F4552524F3E
:10C7B000525F494E56414C49445F44415441000048
:10C7C0004E52465F4552524F525F534F4654444576
:10C7D000564943455F4E4F545F454E41424C454498
:10C7E000000000004E52465F4552524F525F464590
:10C7F00041545552455F4E4F545F454E41424C4562
:10C80000440000004E52465F4552524F525F4D5514
:10C810005445585F554E4C4F434B5F4641494C453C
:10C82000440000004E52465F4552524F525F4D55F4
:10C830005445585F4C4F434B5F4641494C4544007B
:10C840004E52465F4552524F525F4D555445585FC8
:10C85000434F4E445F494E49545F4641494C45441D
:10C86000000000004E52465F4552524F525F4D55F8
:10C870005445585F494E49545F4641494C45440030
:10C880004E52465F4552524F525F424C455F4950AF
:10C8900053505F52585F504B545F5452554E434172
:10C8A000544544004E52465F4552524F525F424CEF
:10C8B000455F495053505F504545525F52454A4588
:10C8C00043544544000000004E52465F4552524FCB
:10C8D000525F424C455F495053505F4C494E4B5F4D
:10C8E000444953434F4E4E454354454400000000D5
:10C8F0004E52465F4552524F525F4150495F4E4F34
:10C90000545F494D504C454D454E54454400000040
:10C910004E52465F4552524F525F4E4F545F5355F1
:10C9200050504F52544544004E52465F4552524F6C
:10C93000525F4D4F44554C455F4E4F545F494E49F1
:10C940005449414C495A4544000000004E52465F4C
:10C950004552524F525F4D4F44554C455F414C52EA
:10C96000454144595F494E495449414C495A45440F
:10C97000000000004E52465F4552524F525F4E4FEC
:10C98000545F464F554E44004E52465F4552524FFB
:10C99000525F494E56414C49445F535441544500FF
:10C9A0004E52465F4552524F525F444154415F538D
:10C9B000495A45004E52465F4552524F525F494FC9
:10C9C0005F50454E44494E47000000004E52465FBE
:10C9D0004552524F525F5356435F48414E444C4577
:10C9E000525F4D495353494E470000004E52465F37
:10C9F0004552524F525F494E56414C49445F4C4557
:10CA00004E475448000000004E52465F4552524F78
:10CA1000525F4452565F5457495F4552525F414EF0
:10CA200041434B004E52465F4552524F525F445273
:10CA3000565F5457495F4552525F444E41434B0045
:10CA40004E52465F4552524F525F494E5445524EE8
:10CA5000414C00004E52465F4552524F525F535474
:10CA60004F524147455F46554C4C00004E52465F81
:10CA70004552524F525F4E554C4C00004E52465F4D
:10CA80004552524F525F494E56414C49445F5041C6
:10CA900052414D004E52465F4552524F525F4E4FEB
:10CAA0005F4D454D000000004E52465F4552524FCB
:10CAB000525F464F5242494444454E004E52465FF3
:10CAC0004552524F525F4452565F5457495F455248
:10CAD000525F4F56455252554E0000004E52465F2F
:10CAE0004552524F525F494E56414C49445F414472
:10CAF000445200004E52465F4552524F525F494EDB
:10CB000056414C49445F464C414753004E52465FA4
:10CB100053554343455353004E52465F4552524F7F
:10CB2000525F424C455F495053505F4348414E4E1F
:10CB3000454C5F414C52454144595F455849535417
:10CB4000530000004E52465F4552524F525F5449C7
:10CB50004D454F55540000004E52465F4552524FCE
:10CB6000525F425553590000726561640000000035
:10CB7000526561642073746F726564206C6F6773B3
:10CB80000000000052656D6F7665206C6F67730062
:10CB9000466C617368206C6F672073746174757381
:10CBA00000000000666C6173686C6F670000000035
:10CBB000436F6D6D616E647320666F722072656184
:10CBC00064696E67206C6F67732073746F7265643D
:10CBD00020696E206E6F6E2D766F6C6174696C6566
:10CBE000206D656D6F7279002E2E5C2E2E5C2E2EC0
:10CBF0005C2E2E5C2E2E5C2E2E5C636F6D706F6E25
:10CC0000656E74735C6C69627261726965735C6590
:10CC100078706572696D656E74616C5F6C6F675C6E
:10CC20007372635C6E72665F6C6F675F6261636B89
:10CC3000656E645F666C6173682E63002E2E5C2ED9
:10CC40002E5C2E2E5C2E2E5C2E2E5C2E2E5C636FA8
:10CC50006D706F6E656E74735C6C6962726172691F
:10CC600065735C6578706572696D656E74616C5F23
:10CC70006C6F675C7372635C6E72665F6C6F675F2C
:10CC800066726F6E74656E642E6300006E6F6E6503
:10CC9000000000006465627567000000276C6F6724
:10CCA00020656E61626C65203C6C6576656C3E202B
:10CCB0003C6D6F64756C655F303E202E2E2E2020FB
:10CCC0003C6D6F64756C655F6E3E2720656E6162BA
:10CCD0006C6573206C6F677320757020746F2067AC
:10CCE0006976656E206C6576656C20696E20737060
:10CCF00065636966696564206D6F64756C65732032
:10CD000028616C6C206966206E6F206D6F64756C95
:10CD1000657320737065636966696564292E000018
:10CD2000276C6F672064697361626C65203C6D6F6E
:10CD300064756C655F303E202E2E203C6D6F6475EF
:10CD40006C655F6E3E272064697361626C65732059
:10CD50006C6F677320696E207370656369666965BF
:10CD600064206D6F64756C65732028616C6C20693C
:10CD700066206E6F206D6F64756C657320737065CF
:10CD8000636966696564292E00000000656E616252
:10CD90006C65000064697361626C6500526573754F
:10CDA0006D65206C6F6767696E67000048616C7421
:10CDB000206C6F6767696E6700000000676F000096
:10CDC0004C6F67676572207374617475730000003F
:10CDD00068616C74000000006C6F6700436F6D6DDC
:10CDE000616E647320666F7220636F6E74726F6C15
:10CDF0006C696E67206C6F67676572001B5B313B07
:10CE000033306D001B5B306D000000001B5B313B5D
:10CE100033316D001B5B313B33326D001B5B313BAB
:10CE200033336D001B5B313B33346D001B5B313B97
:10CE300033356D001B5B313B33366D001B5B313B83
:10CE400033376D006170705F74696D65722E6D5F50
:10CE500074696D65725F30006170705F74696D65D3
:10CE6000722E6D5F636C695F756172745F7472615D
:10CE70006E73706F72745F74696D6572000000008C
:10CE800071756575652E6D5F636C695F7561727430
:10CE90005F6C6F675F6261636B656E645F71756520
:10CEA0007565000062616C6C6F632E6D5F636C6909
:10CEB0005F756172745F636D645F686973745F6DE1
:10CEC000656D6F626A0000006170705F74696D6506
:10CED000722E6D5F636C695F7274745F7472616EE1
:10CEE00073706F72745F74696D65720071756575CA
:10CEF000652E6D5F636C695F7274745F6C6F675FE2
:10CF00006261636B656E645F7175657565000000D5
:10CF100062616C6C6F632E6D5F636C695F727474B9
:10CF20005F636D645F686973745F6D656D6F626A7E
:10CF3000000000006D5F636C695F756172745F6C07
:10CF40006F675F6261636B656E645F717565756560
:10CF5000000000006D5F636C695F7274745F6C6FDA
:10CF6000675F6261636B656E645F717565756500AF
:10CF70006D5F636C695F756172745F636D645F6838
:10CF80006973745F6D656D6F626A00006D5F636CDD
:10CF9000695F7274745F636D645F686973745F6DF9
:10CFA000656D6F626A0000006170705F74696D6525
:10CFB000722E6D5F6273705F6C6564735F746D7207
:10CFC000000000006170705F74696D65722E6D5FA6
:10CFD0006273705F616C6572745F746D72000000E3
:10CFE0006170705F74696D65722E6D5F6273705FE2
:10CFF000627574746F6E5F746D7200006E72665F3E
:10D000006D707500737461636B5F67756172640046
:10D01000636C6F636B000000434C4F434B00000098
:10D020004750494F54450000505253005541525407
:10D030000000000055415254450000006170705FCF
:10D0400074696D65722E6D5F646574656374696F74
:10D050006E5F64656C61795F74696D65725F696448
:10D06000000000006170705F74696D6572000000FF
:10D0700061746669666F2E6D5F7265715F66696661
:10D080006F000000686172646661756C7400000076
:10D09000636C695F75617274000000006E72665F98
:10D0A0006673746F72616765000000007077725F6D
:10D0B0006D676D7400000000736F72746C69737437
:10D0C0000000000071756575652E6D5F666C61739B
:10D0D000686C6F675F717565756500007175657562
:10D0E000652E6D5F63726173686C6F675F717565E4
:10D0F000756500006D5F666C6173686C6F675F716A
:10D1000075657565000000006D5F63726173686C22
:10D110006F675F71756575650000000062616C6C1A
:10D120006F632E6C6F675F6D656D706F6F6C000065
:10D13000617070006C6F675F6D656D706F6F6C0014
:10D14000A4D3000000000020800400002807000095
:10D15000B0D40000800400207837000008110000DF
:10D160000000000024AB0000000000006CAB0000D9
:10D17000000000007CAB000000000000D4AB000009
:10D180000000000044AC0000000000004CAD0000B6
:10D19000000000007CAD0000000000008CAD00002D
:10D1A000000000009CAD000000000000E4AD0000A5
:10D1B0000000000030AE00000000000064AF00007E
:10D1C0000000000074AF00000000000084AF000009
:10D1D0000000000094AF000000000000F0B000006C
:10D1E00000000000BCB200000000000044B30000DA
:10D1F00044CE00000000040358CE000000000403E9
:10D2000080CE000000000003A4CE00000000000358
:10D21000C8CE000000000403ECCE000000000003B4
:10D2200010CF000000000003A8CF0000000004039E
:10D23000C4CF000000000403E0CF0000000004039E
:10D24000FCCF00000000000004D000000000040437
:10D2500010D000000000000018D000000000000006
:10D2600020D000000000000028D0000000000000D6
:10D270002CD000000000000034D0000000000000AE
:10D280003CD000000000040364D00000000004044F
:10D2900070D000000000000384D0000000000404EF
:10D2A00090D00000000000009CD0000000000404AA
:10D2B000ACD0000000000000B8D00000000000006A
:10D2C000C4D0000000000003DCD000000000000318
:10D2D0001CD100000000000330D100000000040455
:10D2E000DC000020D4000020DC0000202C0B0020FB
:10D2F0003C03002070CF000030000000EC00002054
:10D30000E4000020EC000020241000206003002036
:10D310008CCF0000300000006C020020BC13002005
:10D32000CC130020CC1300206804002034D100006E
:10D3300018000000200B00200C0B0020040000004F
:10D34000040000000100000034CF00003003002082
:10D350001810002004100020040000000400000049
:10D360000100000054CF00005403002000130020EF
:10D37000DC12002008000000040000000100000092
:10D38000F4D0000050040020301300200C130020C3
:10D3900008000000040000000100000008D10000A7
:10D3A0005C04002081A35CB29A680C01141318037A
:10D3B0000218205A241C13E00AB320172364AC235C
:10D3C0001968A340AE031E34D35A484CCBD80F4C37
:10D3D0000A11804C0A1D504CC12350BB1A58041A24
:10D3E00068041A60041A70041A78041A8C041A84E7
:10D3F000041AB4041ABC041ACC041AC4041A9404FF
:10D400001A9C041AAC041AA4040135151001401129
:10D410000211044B0804E401102360C06374BF1AB6
:10D42000EC0C2338C15AD010411AA0142394BD1A11
:10D4300028041AB81C1AFC041A1C14A9401B90BE1C
:10D440003C19049AB818811A84301A441CE318C68F
:10D45000236CD31A88040114137C1373203F320108
:10D4600013280224202928238CCC1AB0642360BC02
:10D470001B20BB9819102904291429102920291CC4
:10D480000114E9381B04CECC22CD1A0C081A14045E
:10D490001A1C041A24041A2C041A34041A3C041109
:10D4A000045490D003630D4703FFFF0F016B00008E
:0400000500000201F4
:00000001FF
